:020000040000fa
:080000000002040000000000f2
:020000040000fa
:040008004c030000a5
:020000040000fa
:04000c004c030000a1
:020000040000fa
:040010004c0300009d
:020000040000fa
:040014004c03000099
:020000040000fa
:040018004c03000095
:020000040000fa
:04001c004c03000091
:020000040000fa
:040020004c0300008d
:020000040000fa
:040024004c03000089
:020000040000fa
:040028004c03000085
:020000040000fa
:04002c004c03000081
:020000040000fa
:040030004c0300007d
:020000040000fa
:040034004c03000079
:020000040000fa
:040038004c03000075
:020000040000fa
:04003c004c03000071
:020000040000fa
:040040004c0300006d
:020000040000fa
:040044004c03000069
:020000040000fa
:040048004c03000065
:020000040000fa
:04004c004c03000061
:020000040000fa
:040050004c0300005d
:020000040000fa
:04005400f25c00005a
:020000040000fa
:04005800145d000033
:020000040000fa
:04005c004c03000051
:020000040000fa
:040060004c0300004d
:020000040000fa
:040064004c03000049
:020000040000fa
:040068004c03000045
:020000040000fa
:04006c004c03000041
:020000040000fa
:040070004c0300003d
:020000040000fa
:040074004c03000039
:020000040000fa
:040078004c03000035
:020000040000fa
:04007c004c03000031
:020000040000fa
:040080004c0300002d
:020000040000fa
:040084004c03000029
:020000040000fa
:040088004c03000025
:020000040000fa
:04008c004c03000021
:020000040000fa
:040090004c0300001d
:020000040000fa
:040094004c03000019
:020000040000fa
:040098004c03000015
:020000040000fa
:04009c004c03000011
:020000040000fa
:0400a0004c0300000d
:020000040000fa
:0400a4004c03000009
:020000040000fa
:0400a8004c03000005
:020000040000fa
:0400ac004c03000001
:020000040000fa
:0400b0004c030000fd
:020000040000fa
:0400b4004c030000f9
:020000040000fa
:0400b8004c030000f5
:020000040000fa
:0400bc004c030000f1
:020000040000fa
:0400c0004c030000ed
:020000040000fa
:0400c4004c030000e9
:020000040000fa
:0400c8004c030000e5
:020000040000fa
:0400cc004c030000e1
:020000040000fa
:0400d0004c030000dd
:020000040000fa
:0400d4004c030000d9
:020000040000fa
:0400d8004c030000d5
:020000040000fa
:0400dc004c030000d1
:020000040000fa
:0400e0004c030000cd
:020000040000fa
:0400e4004c030000c9
:020000040000fa
:0400e8004c030000c5
:020000040000fa
:0400ec004c030000c1
:020000040000fa
:0400f0004c030000bd
:020000040000fa
:0400f4004c030000b9
:020000040000fa
:0400f8004c030000b5
:020000040000fa
:0400fc004c030000b1
:020000040000fa
:040100004c030000ac
:020000040000fa
:040104004c030000a8
:020000040000fa
:040108004c030000a4
:020000040000fa
:04010c004c030000a0
:020000040000fa
:040110004c0300009c
:020000040000fa
:040114004c03000098
:020000040000fa
:040118004c03000094
:020000040000fa
:04011c004c03000090
:020000040000fa
:040120004c0300008c
:020000040000fa
:040124004c03000088
:020000040000fa
:040128004c03000084
:020000040000fa
:04012c004c03000080
:020000040000fa
:040130004c0300007c
:020000040000fa
:040134004c03000078
:020000040000fa
:040138004c03000074
:020000040000fa
:04013c004c03000070
:020000040000fa
:040140004c0300006c
:020000040000fa
:040144004c03000068
:020000040000fa
:040148004c03000064
:020000040000fa
:040208004c030000a3
:020000040000fa
:04020c004c0300009f
:020000040000fa
:040210004c0300009b
:020000040000fa
:040214004c03000097
:020000040000fa
:040218004c03000093
:020000040000fa
:04021c004c0300008f
:020000040000fa
:040220004c0300008b
:020000040000fa
:040224004c03000087
:020000040000fa
:040228004c03000083
:020000040000fa
:04022c004c0300007f
:020000040000fa
:040230004c0300007b
:020000040000fa
:040234004c03000077
:020000040000fa
:040238004c03000073
:020000040000fa
:04023c004c0300006f
:020000040000fa
:040240004c0300006b
:020000040000fa
:040244004c03000067
:020000040000fa
:040248004c03000063
:020000040000fa
:04024c004c0300005f
:020000040000fa
:040250004c0300005b
:020000040000fa
:040254004c03000057
:020000040000fa
:040258004c03000053
:020000040000fa
:04025c004c0300004f
:020000040000fa
:040260004c0300004b
:020000040000fa
:040264004c03000047
:020000040000fa
:040268004c03000043
:020000040000fa
:04026c004c0300003f
:020000040000fa
:040270004c0300003b
:020000040000fa
:040274004c03000037
:020000040000fa
:040278004c03000033
:020000040000fa
:04027c004c0300002f
:020000040000fa
:040280004c0300002b
:020000040000fa
:040284004c03000027
:020000040000fa
:040288004c03000023
:020000040000fa
:04028c004c0300001f
:020000040000fa
:040290004c0300001b
:020000040000fa
:040294004c03000017
:020000040000fa
:040298004c03000013
:020000040000fa
:04029c004c0300000f
:020000040000fa
:0402a0004c0300000b
:020000040000fa
:0402a4004c03000007
:020000040000fa
:0402a8004c03000003
:020000040000fa
:0402ac004c030000ff
:020000040000fa
:0402b0004c030000fb
:020000040000fa
:0402b4004c030000f7
:020000040000fa
:0402b8004c030000f3
:020000040000fa
:0402bc004c030000ef
:020000040000fa
:0402c0004c030000eb
:020000040000fa
:0402c4004c030000e7
:020000040000fa
:0402c8004c030000e3
:020000040000fa
:0402cc004c030000df
:020000040000fa
:0402d0004c030000db
:020000040000fa
:0402d4004c030000d7
:020000040000fa
:0402d8004c030000d3
:020000040000fa
:0402dc004c030000cf
:020000040000fa
:0402e0004c030000cb
:020000040000fa
:0402e4004c030000c7
:020000040000fa
:0402e8004c030000c3
:020000040000fa
:0402ec004c030000bf
:020000040000fa
:0402f0004c030000bb
:020000040000fa
:0402f4004c030000b7
:020000040000fa
:0402f8004c030000b3
:020000040000fa
:0402fc004c030000af
:020000040000fa
:040300004c030000aa
:020000040000fa
:040304004c030000a6
:020000040000fa
:040308004c030000a2
:020000040000fa
:04030c004c0300009e
:020000040000fa
:040310004c0300009a
:020000040000fa
:040314004c03000096
:020000040000fa
:040318004c03000092
:020000040000fa
:04031c004c0300008e
:020000040000fa
:040320004c0300008a
:020000040000fa
:040324004c03000086
:020000040000fa
:040328004c03000082
:020000040000fa
:04032c004c0300007e
:020000040000fa
:040330004c0300007a
:020000040000fa
:040334004c03000076
:020000040000fa
:040338004c03000072
:020000040000fa
:04033c004c0300006e
:020000040000fa
:040340004c0300006a
:020000040000fa
:040344004c03000066
:020000040000fa
:040348004c03000062
:020000040000fa
:10040000cfa221000e7f22000e0188000000000014
:10041000000020000000e000020032000001200087
:10042000200288000c00070060ec2600010020007c
:1004300011000700000020000000e0000200320070
:100440000000020000000000e07002000000000058
:100450000040da000000fe004440a900002b20000c
:100460000000e0000300320000002000a00188002e
:100470004440a80000000600910188008000780038
:100480000000eb0015003700e280400032a0b4000d
:100490009101ba00e280400032a0b4009102ba009b
:1004a000e280400032a0b4000002eb00472bde00e7
:1004b000f507b200602ce10004003a000059eb009f
:1004c0008301e900fdff3e00040037006128e100e0
:1004d000010032000082eb000b00070011c3ba00dc
:1004e0001101ba000604e00003003a000200e00037
:1004f000e5ff3a0000000600f607b200960188000a
:1005000082007800f5ff37003159ba008301e90015
:100510000c0032002159ba008301e90008003200c2
:100520000400e00003003a00e280400032a0b40082
:10053000f5ff370011d9ba008301e900faff3a004c
:100540008100e800e180400032a0b4000000060015
:10055000000000000000000000000000000000009b
:10056000000000000000000000000000000000008b
:10057000000000000000000000000000000000007b
:10058000000000000000000000000000000000006b
:10059000000000000000000000000000000000005b
:1005a000000000000000000000000000000000004b
:1005b000000000000000000000000000000000003b
:1005c000000000000000000000000000000000002b
:1005d000000000000000000000000000000000001b
:1005e000000000000000000000000000000000000b
:1005f00000000000000000000000000000000000fb
:1006000000000000000000000000000000000000ea
:1006100000000000000000000000000000000000da
:1006200000000000000000000000000000000000ca
:1006300000000000000000000000000000000000ba
:1006400000000000000000000000000000000000aa
:10065000000000000000000000000000000000009a
:10066000000000000000000000000000000000008a
:10067000000000000000000000000000000000007a
:10068000000000000000000000000000000000006a
:1006900000000000000000000040da000000fe0042
:1006a00003f0a200889fbe008a9fbe008c1f7800c6
:1006b0004a010700510133006450e1004f0032004d
:1006c0006420e1005200320003826c0007003b000e
:1006d0000905d0000306d000820f54000c065d000f
:1006e0000200390002003200890178000306780018
:1006f0008582550004003d000003fd008103fd00dc
:100700008502ea008b854200840f720002003b00e4
:1007100060001000e08018006011b8000005eb00d8
:100720007a28e1000a00390006007800c75ddd0084
:10073000f707b200878075002d00370082817100b5
:100740000a017800610560008180d1000080d3003b
:100750008502e900f9ff3b00060440008784480059
:1007600002003b0060041400e0841c000988a30020
:10077000070032008a81710082817100610164008a
:100780008904d1000884d3008b05e80017003700e6
:100790000978a30013003a000b00e00013003400b6
:1007a0008b05e9000804440089844c000a44740065
:1007b0000978a3000d003a000b00e00007003400a8
:1007c0008b05e9000804440089844c0001003a00cc
:1007d0000b0020000978a300f7ff32000001eb00b6
:1007e00002003700828171000a017800c000070012
:1007f0000cf0a70001f0a000090137006420e1001f
:1008000002003a00838f6c00090133000801be002a
:100810000200be0002013700889fbe008a9fbe0012
:100820008c1f7800ed000700f400330003866c0095
:100830006450e1002e0032006420e10033003200f9
:100840006150e1002f0032006120e10031003200f0
:1008500085855500eb07b000090020000804200042
:10086000050037000804440089844c000a00310068
:100870000603430087834b000001530081815b0026
:10088000f8ff33000203be000800a0000804440083
:1008900089844c00f6ff3900c639dd0083017300fe
:1008a00001003200130020008904d1000884d30025
:1008b0000998a300050032000800a7000300a0006b
:1008c0008904d1000884d3008b05e8008904d10095
:1008d0000884d3000001eb000281d20084000700ed
:1008e00001f0a1000cf0a70001f0a000cc0037003f
:1008f0006420e100ce0032000801be000200be000c
:10090000f7ff37006120e100c90032006000b80045
:10091000f3ff37000000200001f82700f0ff370048
:10092000140020000e023700f4ff2f000c023700e5
:100930000003be00940007006011b8000470a70017
:1009400007f0a10007f8a30017003a006509b100fd
:100950000d0032000d003500860220000628e1005f
:1009600003003500030028006000b8000200050005
:100970000000400081804800020149008381490055
:100980008502e900faff3a0000000600f88f4200f5
:10099000050034008100d1000080d3008502e8000a
:1009a000fcff3a00000006006011b8008000eb0078
:1009b000000005000001be00730007000470a700de
:1009c00003f0a10003f8a30013003a006509b10089
:1009d00010003200090035006928e10002003500ee
:1009e0000100280000000500000040008180480050
:1009f0008502e900fcff3a0000000600f88f420083
:100a0000050035008100d1000080d3008502e80098
:100a1000fcff3a00000006008000eb00000005002b
:100a20004f89de0082017800e8013700889fbe0010
:100a30008a9fbe000082700004027100048271006f
:100a4000260032000004be000200be006011b800a3
:100a50006b092000950220000182cf000a003900b6
:100a60000541b1000082cf00070039000541b10007
:100a70000982cf00040039000541b1000882cf008f
:100a8000010039000541b100054252001200320058
:100a90000a003b0082817100610164008100d10085
:100aa0000080d3008984d3000884d3008b05e8003c
:100ab0000442e800f7ff3a0007003700080444004a
:100ac00089844c0000004800818048008b05e900c3
:100ad0000442e900f9ff3a00050007004f05be0097
:100ae0004f04be00000006006011b800cfff3700c1
:100af00081002000618055000b003d000b002000ac
:100b000061fe2f000100e1001d00340082817100b0
:100b1000610164008904d1000884d3000000e8006a
:100b2000faff3a00710020006100640003007000c9
:100b3000020060000900320061044400e0844c00bf
:100b40000988a500050032008b05e8006808e1006f
:100b500002003a008904d1000884d300f20f20007b
:100b60000258e10005003d00c75ddd00f907b20055
:100b70008980750008007800000006000bf8270047
:100b80008b00780000000500c70ade00f107b20004
:100b9000f50fb20008003200e1cf4200020032003f
:100ba0000170a00024000500810f700001003200d8
:100bb0000408050044000500810f700002003a009f
:100bc000140005008502e9000000400081c04800d3
:100bd000fcff3b000170a000240005000004be00e3
:100be000e9ff07000003be000405be000200be00ce
:100bf000e5ff0700844f7500000006000200be00fc
:100c00006450e100050036006420e1000200360077
:100c10000968a30001003a000800be000160a000be
:100c20004f0678004f05be004f04be0000000600ce
:100c3000f0ff2f00f1ff2700f9ff3700889fbe006b
:100c40008a9fbe008c1f7800e4ff0700ebff330093
:100c500003866c006450e100240032006420e1004f
:100c6000270032006150e100220032006120e100e3
:100c7000210032008b854200eb07b1000134b8003f
:100c8000003ab8000804420089844a00013ab800da
:100c90000030b8008880400009014a000400330099
:100ca0000000400081804800020149008b05e900f6
:100cb000c909dd008301700001003200130020002b
:100cc000c814de004814dd004709de001200b2003f
:100cd000c808de000884700085ff070001f0a1004d
:100ce0000cf0a70001f0a000cdff37006120e1006b
:100cf000cfff32000801be000200be00f7ff370040
:100d00006150e100fcff3a00c9ff37006022b800e3
:100d1000060220000000d0008180d2000482d200b0
:100d20008582d2000000a0000202520083825a0095
:100d3000030031000202420083824a000000a10049
:100d40000603e900f3ff3a0000000600efff07008a
:100d50000400be0000000600889fbe008a9fbe00ff
:100d600030044200b0844a0030054b0090854b00af
:100d70006000b1000898be000a90be000440e10087
:100d800005c8e10006d0e10007d8e100020031000b
:100d9000680040001008e8004f05be004f04be0088
:100da00000000600889fbe008a9fbe003004be007f
:100db0002005be000418540005985c0006185d006c
:100dc00007985d00110020000440e10005c8e10023
:100dd00006d0e10007d8e100010039008000eb00f7
:100de000108810004f05be004f04be000000060032
:100df0001200fa00889fbe008a9fbe008c9fbe0032
:100e0000e0b79f00f1b79f0082bf9f0093bf9f0094
:100e10000605be000404be000000eb00d0b79f0032
:100e2000c0b79f00b0b79f00a0b79f0090b79f00ca
:100e30000006eb005fb19700cfb097008201410040
:100e40003fb097000200e00004003d0037000700bb
:100e50007e805700c0ff0700030037003300070003
:100e60007e805700cfff0700dfb697000d00e0003f
:100e70000c0035006fb29700ffb297000fbb9700d0
:100e80009fbb970010002000010020006011b800f7
:100e90000002720081827200020373008383730078
:100ea0001b0007000c06e80001042000810f56001b
:100eb000e0ff3a000d00e00004003d000802be0023
:100ec0000a03be007e805700a3ff07005fa89700bb
:100ed0000000e00005003a001fb29700afb2970093
:100ee0003fb39700cfb39700090007006fb097009a
:100ef000ffb097000fb997009fb997004f06be004b
:100f00004f05be004f04be000080fa00000006003e
:100f10000100070000000600a4b79f00b5b79f00be
:100f2000c6b79f00d7b79f00000006004f09de003c
:100f300082817100b3b79f004f01de0081804000c5
:100f400082807000a1b79f008fb097004f09de002c
:100f5000000040000200700090b79f007fa897003b
:100f60004f01de00818040008280700081b79f00c9
:100f70000d0007004f3ade00000040000400700042
:100f8000f0af9f00080007000402420085824a007b
:100f900006034b0087834b00dfff07000802be00fb
:100fa0000a03be00000006002fb29700bfb29700f0
:100fb0004fb39700dfb3970000000600881f78004a
:100fc00018002000881f780089ff07008f87e9003c
:100fd0004f04780000000600801feb0084ff07002c
:100fe0008f87e90000000600889fbe008a9fbe0030
:100ff000e00f5000e08f5800e00f5900e08f5900db
:101000000c003d006044b8006055b800000054007a
:1010100081805c0002015d0083815d00180020007a
:101020001500070008003d00180007000004eb0051
:10103000050037000004eb000f00070002003d0030
:101040001200070018002000dcff07000800e00085
:10105000060032006022b8006033b8000000520081
:1010600081805a0002015b0083815b004f05be0056
:101070004f04be0000000600e00f5200e08f5a004f
:10108000e00f5b00e08f5b00000006006044b800ea
:101090006055b8000402540085825c0006035d00c0
:1010a00087835d0000000600889fbe008a9fbe0007
:1010b0008c1f7800e00f5000e08f5800e00f5900bf
:1010c000e08f59000d003d006044b8006055b80045
:1010d0000000540081805c0002015d0083815d009e
:1010e0001c0020000820e10009a8e1000ab0e1008e
:1010f0000bb8e1000d003d00080037000006eb00d2
:10110000e00f5200e08f5a00e00f5b00e08f5b00c1
:1011100006003d006044b8006055b8000402540069
:1011200085825c0006035d0087835d00aaff0700df
:101130000c00e000060032006022b8006033b80006
:101140000000520081805a0002015b0083815b0035
:101150004f0678004f05be004f04be000000060099
:10116000889fbe008a9fbe00841f78009bfe0700f8
:101170004f00780011003300f0ff2f00838f6c00c8
:1011800006003b00040565000a00a70008003700c0
:1011900009f0a6001000200008003700820f54005c
:1011a000838f5c00030039001000200001003e0026
:1011b0000000200009f0a7000000ea004f05be0073
:1011c0004f04be000000e00000000600881f780009
:1011d000030478000300e00007003d0060001000f9
:1011e000e080180060011900e081190002003b0056
:1011f00001f02d00030037000cfe070008f0a700e7
:0c12000001f0a0004f0478000000060080
:020000040000fa
:10120c000d0a00002800000078000000293e0000b4
:10121c000008000020080000000000002e20000044
:10122c0000200000004300006c7500007463000097
:10123c006820000064690000736500006e670000a0
:10124c00616700006564000021210000210000009e
:10125c00546f000020660000696e00006973000086
:10126c00682000007365000074750000702c00008d
:10127c00207300007461000072740000207500007f
:10128c00702000007468000065200000706f000082
:10129c00776500007220000073750000707000000c
:1012ac006c69000065730000207700006974000011
:1012bc0068200000636f00006d6d0000616e00001f
:1012cc006420000027570000270d00000a000000d2
:1012dc00427500007320000050690000726100002c
:1012ec0074650000207600003300000020630000cd
:1012fc006c6f00006e650000207700002f6400000a
:10130c006966000066650000726500006e7400007e
:10131c002050000049430000004300006f6d0000a6
:10132c006d7500006e6900007479000020460000a5
:10133c00697200006d77000061720000652000008a
:10134c00763700002e300000202d000020670000b2
:10135c006f6f00002e6700006c2f000067430000c9
:10136c007a5100006e570000200000002028000079
:10137c0032340000464a0000363400004741000079
:10138c00303000000034000020000000322000004b
:10139c000041000033000000423400000042000015
:1013ac003500000042380000005500004e4b000094
:1013bc000029000000490000090000004f0900004e
:1013cc0000480000090000004c0900000045000026
:1013dc006e740000657200002072000061770000de
:1013ec0020760000616c000075650000206600002e
:1013fc006f7200002042000052470000003e0000c7
:10140c00001b00005b440000001b00005b000000a0
:10141c00440000001b5b0000430000001b5b00004d
:10142c00324b00000d000000430000001b5b00006d
:10143c003244000000570000617200006e69000029
:10144c006e6700003a2000006e6f000020760000ee
:10145c006f6c00007461000067650000206f000075
:10146c006e20000056700000756c00006c7500005a
:10147c0070200000706900006e000000203d00002c
:10148c0020000000436c00007574000063680000cd
:10149c00206500006e670000616700006564000055
:1014ac002121000021000000565200004547000099
:1014bc00207400006f6f0000206c00006f7700003c
:1014cc002c20000069730000207400006865000087
:1014dc00726500002061000020730000686f00003e
:1014ec00727400003f0000002e2000003c00000041
:1014fc000041000052540000310000001434000080
:10150c00040d00008206000040030000a001000052
:10151c00cf0000007f0000006700000044000000c6
:10152c002200000000000000000000002c01000060
:10153c00000000005802000000000000b004000091
:10154c00000000006009000000000000c012000054
:10155c000000000080250000000000004038000062
:10156c0000000000004b0000000000008070000034
:10157c00000000000096000000000000c0da00002f
:10158c000000000000e100000000000000c20000ac
:10159c000100000000f400000100000000e8000061
:1015ac000300000014340000040d0000820600004b
:1015bc0040030000a0010000cf0000006700000005
:1015cc0044000000220000007f00000030300000ca
:1015dc00302c0000003000003000000030620000b1
:1015ec000000000014340000040d0000820600000e
:1015fc0040030000a0010000cf00000067000000c5
:10160c00440000002200000030780000303100005f
:10161c003233000034350000363700003839000012
:10162c0041420000434400004546000020480000b1
:10163c007a000000467200006571000075650000bc
:10164c006e63000069650000732000003c20000000
:10165c00314800007a200000617200006520000013
:10166c006e6f000074200000737500007070000035
:10167c006f72000074650000642e00000000000012
:10168c00436f0000756c0000646e0000277400004e
:10169c00206b000065650000702000007570000074
:1016ac000000000053500000493100000000000011
:1016bc00181c00001d0300000b1300001b00000091
:1016cc00181c00001d000000314100004c530000ac
:1016dc0001420000507600003300000021000000a1
:1016ec000010000000230000000f0000424000002a
:1016fc00400500004102000000000000002900002d
:10170c00002000005700000020520000004900009b
:10171c0032430000310000000808000008080000f7
:10172c00080000000000000042420000494f000089
:10173c003100000052410000573100000000000051
:10174c00003500003f620000610000004f430000c4
:10175c004431000000000000000000000000000008
:020000040000fa
:10176c00889fbe008a9fbe008c1f780013c4800027
:10177c0003007800f007b20001802100614078007e
:10178c00f1ccb30081404000e8cf50001a003e007d
:10179c000000fb000003b1008300e800f107b20079
:1017ac000280210062c1780004cdb30004424100e4
:1017bc0011002000e94f520078003e00f80720008d
:1017cc000780210006cdb3006a02b9000200fb00bd
:1017dc00040040000003b1008100e80003814000d8
:1017ec00080161006741790006424100e94f52004f
:1017fc00f5ff36006900370001c3b300814f50007c
:10180c0061003a000300e800f007b20001802100fb
:10181c006141780020c6b300804f51000b003a00a4
:10182c000380e800f007b2000180210061417800dc
:10183c0004cdb300044241000000eb002100200065
:10184c00e14f5200050036005400370020c4b300ad
:10185c00804f510010003a00f1ff3700f7072000cd
:10186c000680210005cdb300000040000201fb0002
:10187c00020040000003b1008100e8000381400039
:10188c00070161006641790005424100e14f5200b9
:10189c00f5ff36004100370080c7b300804f510080
:1018ac000a00320080c5b300804f51001f003a007f
:1018bc00090037004400dd000003b1000201fb0009
:1018cc00020040008100e8000b0037000000eb0034
:1018dc0021002000020037000000eb002100200056
:1018ec00f90720000780210008cdb300facbb30024
:1018fc000bc2b300fcc9b3000382400009026200b2
:10190c0067417a0088424100e9cf5200e9ff360076
:10191c008a424100e5cf5200280036000c434100ba
:10192c00e54f5300250036001c00370004cdb300f2
:10193c00044241000000eb0011002000e94f52006e
:10194c0016003e000200fb000003b100f807200067
:10195c000780210006cdb3006a02b9000200fb002b
:10196c00040040000003b1008100e8000381400046
:10197c00080161006741790006424100e94f5200bd
:10198c00f5ff36000500370011c0b3004088210078
:10199c00014878000000eb000400370012c48000fe
:1019ac0082804000f107b20011c488004f06780015
:1019bc004f05be004f04be00000006000b41710035
:1019cc0082737a004400dd007005b1000201fb0057
:1019dc0002004000bbff3700881f780011c4800054
:1019ec000100e800f007b20002802100e24178001b
:1019fc0010002000a2c3b30082cf510009003a00ae
:101a0c008180e800f80720008880600011c48800fd
:101a1c0053ff070011c480008100e90008846000b6
:101a2c0018c488004f04780000000600881f780056
:101a3c0011c480000100e800f007b2000280210010
:101a4c00e24178000000eb00b2c3b30082cf51003a
:101a5c0009003a008180e800f807200088806000c7
:101a6c0011c488003eff070011c480008100e9000a
:101a7c000884600018c488004f0478000000060039
:101a8c0012c480000201e800f207b20000802100bd
:101a9c00e040790080c7b30080cf500003003a00cb
:101aac0012c4880010c0b3001200370040c6b30047
:101abc0080cf500003003a0012c4880020c0b3004d
:101acc000c00370020c6b30080cf500003003a0052
:101adc0012c4880030c0b300060037000040eb0091
:101aec0073c7b30083cf500002003a0012c48800c1
:101afc0040c0b3000000060010c48000018021002b
:101b0c006141780001c2b300814f510009003a00d5
:101b1c00f407200003802100014178000000e80058
:101b2c0004006000e340780082cf5000fbff3200dd
:101b3c0010c4880000000600f0874700889fbe0094
:101b4c008a9fbe008c9fbe008e1f7800f0b79f004e
:101b5c00e1b79f00d2b79f00030778000acdb3000e
:101b6c00dbc2b3008bf79f008dc7b30060902800d9
:101b7c00325b020000000000ffb097000100e000a3
:101b8c0004003d00a0902800325b02000000000021
:101b9c00030037006fe89700f059020000000000c6
:101bac00c0902800325b0200000000000006eb0031
:101bbc008004eb00c85902000000000000447800cb
:101bcc00ed4f50004000320005003c00e84f500043
:101bdc0008003200ea4f500025003a003a00370066
:101bec008b4f5000150032008d4f500020003a00f2
:101bfc001d0037000900e000050032008904e900ef
:101c0c00f0902800325b020000000000e9ff370072
:101c1c000c00e00005003200f0902800325b02005e
:101c2c00000000000006eb00e2ff370070c0b300bc
:101c3c00da59020000000000deff37000900e00066
:101c4c0005003a000ff09700da590200000000007e
:101c5c001c002000d7ff370070c0b300da59020017
:101c6c0000000000d3ff37000e00e00036003a0001
:101c7c000a404000e94f50000f003e00e38f540033
:101c8c000500340070c0b300da59020000000000f7
:101c9c0049002000c7ff370008407800da590200dd
:101cac0000000000884078007c80570001f07c0028
:101cbc008904e800bfff370070c0b300da59020096
:101ccc0000000000bbff370030912800125b0200bf
:101cdc00000000000900e0001f0032000900e900cc
:101cec008000eb00080033007c8057008904400022
:101cfc006a09b900b000fb000103b100828040000a
:101d0c00890f5000faff3a006fb09700810f500016
:101d1c0008003c005fb09700810f500005003500b3
:101d2c000c00e0000b0032000100ea00f0b79f004d
:101d3c0009003700b101200080ec20000a6e02007f
:101d4c000000000089ff37008080eb00f1b79f0096
:101d5c0001003700f1b79f007fb097004f07780064
:101d6c004f06be004f05be004f04be000f01b10070
:101d7c00000006000e00fa00889fbe008a9fbe007d
:101d8c008c9fbe0010c480000004e900f807b2006c
:101d9c001d002000880f50002a003200098021000d
:101dac00fb07200069407c000004e00020003a00a2
:101dbc000806e8000b06660069407e000004e0009f
:101dcc001b0032000d407800f059020000000000aa
:101ddc0040912800325b02000000000069407e0048
:101dec000004e000080032000885e800da5902001f
:101dfc00000000000b006500694078000a05e8004f
:101e0c000004e000f9ff3a000d8046000c01780058
:101e1c00fa805700823078008d06e800e78f560074
:101e2c000800320030912800125b02000000000014
:101e3c000804e9000b04640010c48000800f5400f7
:101e4c00d8ff3a0070912800125b020000000000dd
:101e5c0071002000107420000a6e020000000000c7
:101e6c00130020000d017800830078000000eb00c7
:101e7c0031ff07008000e800e18f50000b003600b6
:101e8c0000004000fa805700e1027800050078005d
:101e9c00f007b20001802100e14078000000eb0067
:101eac000104e00006003a001200370030912800cf
:101ebc00125b020000000000100020001c00370024
:101ecc0006c480000000eb00f30720000280210014
:101edc00060240000302620001717a000000e80073
:101eec008500400083806000e2c078000104e000bf
:101efc00f7ff3a0002c480000201e900f10720005c
:101f0c000101610012c488000281e8000000410058
:101f1c000100600000c488000000e900810060003e
:101f2c000041eb000080210002f078000000eb0083
:101f3c004f06be004f05be004f04be000080fa00e5
:101f4c0000000600889fbe008a9fbe008c1f780090
:101f5c0010c480000000e800f007b20010c4880034
:101f6c00e5fe0700fefd07000000e00042003a001d
:101f7c000004eb00090320000a8d21000840e80052
:101f8c00f05902000000000040912800325b020072
:101f9c000000000009c0b9008002b0000a00400037
:101fac00125b0200000000000804e800e40f54007b
:101fbc00f2ff3a0071012000606d20000a6e0200f1
:101fcc0000000000408821000048eb0013002000b6
:101fdc00420020008300780003007800d6fe070042
:101fec008004e9000000e800e10f500005003e000d
:101ffc00e1002000d06e20000a6e020000000000fc
:10200c003b003700489e2100180078000b0320008d
:10201c000b80b9002002b0000c8d21006c00780000
:10202c0000000100ca6a020000000000090c7800e0
:10203c000bcdb9007e0545006c007d000000010051
:10204c0090912800125b0200000000000900e000e3
:10205c0004003200c222a800e0922800125b0200a9
:10206c000000000051002000505720000a6e0200b2
:10207c00000000001e0037000004e900e30f5400cc
:10208c0017003c00499e2100190078000a0320002b
:10209c000a80b9002002b0000b8d21006b00780083
:1020ac0000000100ca6a020000000000880c7800e1
:1020bc000ac0b9007e0540006b007d0000000100e5
:1020cc000800e00001003200c222a80051002000ec
:1020dc00505720000a6e0200000000000400370078
:1020ec0051012000c07220000a6e020000000000a6
:1020fc0000c480000000e900f007b20010c48800a2
:10210c004f0678004f05be004f04be0000000600cd
:10211c00889fbe008a9fbe00e0962800325b0200ba
:10212c0000000000e0c2b300da5902000000000019
:10213c00a09e210010407800da5902000000000037
:10214c0031cf8000f0442000808f500003003a0013
:10215c00c0972800325b020000000000309128007c
:10216c00125b02000000000030992800325b020074
:10217c0000000000b0c5b300da59020000000000f6
:10218c00190020000004eb000a0320000b8d210035
:10219c00020037000804e8008904e8000800e000a9
:1021ac006b00320000c2b300da59020000000000dc
:1021bc000ac0b9008002b0000b004000325b020084
:1021cc0000000000e38f5400f2ff3600d0c5b300ce
:1021dc00da59020000000000d1002000a08020008d
:1021ec00ae6d020000000000a1bf2a000000eb0051
:1021fc00de58020000000000000478004840de00b9
:10220c00f059020000000000e0c2b300da590200ed
:10221c000000000008407800f059020000000000a7
:10222c0030912800125b02000000000061002000c9
:10223c0030762000ae6d020000000000689e210088
:10224c0018007800665c020000000000710020009d
:10225c0010ec2000ae6d02000000000040cf8000aa
:10226c00665c020000000000c09b2800325b02008c
:10227c0000000000f0442000980f100004003a0009
:10228c00909c2800325b0200000000000300370025
:10229c00c09c2800325b02000000000040cf800090
:1022ac0021042300810f50001000320004003e0076
:1022bc00f103b100810f500018003a0007003700fd
:1022cc0031042300810f50000c003200e3804000e9
:1022dc00810f500011003a000c003700f09c2800d0
:1022ec00325b0200000000000f003700209d280028
:1022fc00325b0200000000000b003700509d2800ec
:10230c00325b02000000000007003700809d2800af
:10231c00325b02000000000003003700b09d280073
:10232c00325b020000000000f09d2800125b0200ee
:10233c0000000000e1012000907620000a6e0200ef
:10234c00000000004f05be004f04be000000060058
:10235c000ac0b9008002b0000b004000325b0200e2
:10236c00000000008bff3700c802b60004003200ea
:10237c00109e2800325b02000000000003003700b2
:10238c00409e2800325b02000000000000000600a6
:10239c00ca02b60004003200709e2800325b0200b4
:1023ac000000000003003700a09e2800325b0200f2
:1023bc000000000000000600a100200040072100e2
:1023cc000a6e02000000000061042000c00c210015
:1023dc000a6e020000000000a1012000e0072100ad
:1023ec00ae6d0200000000000003200021cf800031
:1023fc000088b9004002b000018d21006100780016
:10240c0000000100a100200080092100ae6d020037
:10241c000000000000402000d3ff07000010200047
:10242c00d1ff070000202000cfff07000004200090
:10243c00cdff070000082000cbff070030912800db
:10244c00125b02000000000041002000201121005e
:10245c00ae6d02000000000021e3a800a0002000e7
:10246c00026b0200000000003c5a02000000000059
:10247c0011002000b0372000ae6d020000000000fb
:10248c0090c0b300da590200000000009000200058
:10249c00026b0200000000003c5a02000000000029
:1024ac0011002000b0372000ae6d020000000000cb
:1024bc0090c0b300da59020000000000c0002000f8
:1024cc00026b0200000000003c5a020000000000f9
:1024dc0011002000b0372000ae6d0200000000009b
:1024ec0090c0b300da59020000000000b0002000d8
:1024fc00026b0200000000003c5a020000000000c9
:10250c0011002000b0372000ae6d0200000000006a
:10251c0090c0b300da5902000000000021e3a900ca
:10252c00004020009aff07000010200098ff0700d1
:10253c000020200096ff07000004200094ff0700f5
:10254c000008200092ff070030912800125b020067
:10255c0000000000000006005100200050922000f6
:10256c00ae6d020000000000c1bf2a000000eb00ad
:10257c00de58020000000000665c02000000000053
:10258c0061002000a0922000ae6d0200000000004f
:10259c00e1bf2a000000eb00de5802000000000042
:1025ac00665c02000000000030912800125b020003
:1025bc0000000000c1002000707820000a6e0200ac
:1025cc00000000007cff0700c202ab0005003200d7
:1025dc0011012000a0622000ae6d0200000000007e
:1025ec000400370021012000b0632000ae6d020012
:1025fc0000000000c0c2b300da5902000000000065
:10260c0000c2b300da59020000000000cb62ab003c
:10261c000500320041012000705d2000ae6d02000b
:10262c00000000000400370051012000205c200055
:10263c00ae6d020000000000c0c2b300da59020007
:10264c000000000000c2b300da59020000000000d4
:10265c00809c210010407800704060000500320022
:10266c0021022000307920000a6e020000000000d8
:10267c0004003700e1012000507b20000a6e0200ac
:10268c0000000000809c2100104078006840600031
:10269c0005003a00b1012000307d2000ae6d020033
:1026ac000000000004003700c1012000e07e200083
:1026bc00ae6d020000000000c0c2b300da59020087
:1026cc000000000000c2b300da5902000000000054
:1026dc00b1012000b01a2100ae6d02000000000014
:1026ec00709b210010407800f0590200000000009f
:1026fc0030912800125b020000000000809c210039
:10270c001040780063406000e14f500005003a0033
:10271c0051012000005920000a6e02000000000048
:10272c000400370061012000a05720000a6e02004f
:10273c00000000000003200021cf80000088b900b9
:10274c006002b000018d21006100780000000100e2
:10275c00c1002000707820000a6e0200000000000a
:10276c000000060010c480000000e800f007b20072
:10277c0010c48800e0fc0700f9fb07008000e900aa
:10278c00e38f500003003e00219e21008008e900e9
:10279c000d003700408821000048eb00210220008a
:1027ac00708120000a6e0200000000008001eb0026
:1027bc00420020001100200010002000defc070069
:1027cc00219e21008008e900210120009083200037
:1027dc000a6e02000000000000000600881f78004e
:1027ec0010c480000000e800f007b20010c488009c
:1027fc00c1fc0700dafb07000040e900e94f50007c
:10280c0003003e00019e2100804878000d00370037
:10281c00408821000048eb00d10820006087200090
:10282c000a6e0200000000008001eb00a2002000f4
:10283c001100200090002000bffc0700019e210029
:10284c008048e9000044eb00009e210091c0b300d9
:10285c0090cf100010003a00a7fc0700c0fb070047
:10286c00004478000804e0000b003a004088210086
:10287c000048eb00d09e2800125b02000000000014
:10288c008001eb00f2ff27008000eb00200220000b
:10289c00a9fc070000447800410120003090200082
:1028ac000a6e02000000000011012000a019210096
:1028bc000a6e020000000000145902000000000023
:1028cc000004e000fcff3200009e210091c0b30028
:1028dc0090cf100003003a0008407800c05c020062
:1028ec0000000000f45802000000000008c2b30011
:1028fc00c859020000000000884f5000fcff3a004d
:10290c004f04780000000600ec874700889fbe004b
:10291c008a9fbe008c9fbe008e1f78000000eb00cb
:10292c0010c4880000c4880020cf88004188210092
:10293c00804878000002eb00568821008002eb00f2
:10294c008041eb000202200007003700836878000a
:10295c000000e800820f5000fcff3a000402e8007f
:10296c00e30f5200050032007820b9008000e90026
:10297c008680400005007800f4ff37000000eb0073
:10298c0070c688000007eb00deb79f00eeb79f0013
:10299c0020c2b30080ef9f000003200022cf8000f4
:1029ac000091b900818f210001004100325b0200cf
:1029bc000000000050a02800325b02000000000064
:1029cc008000eb0081bf9f00598821000b80210003
:1029dc008a9c210070c680000000e0004300320099
:1029ec000000e90070c688007801b900e940790060
:1029fc000104e000130032000004eb0002c480006c
:102a0c00817579007800b9000000440069407800b5
:102a1c00da590200000000000804e80000c480003d
:102a2c000000e800f007b20000c4880070c6800007
:102a3c007801b90082004400e9c078000104e0008c
:102a4c00eeff3a000000eb0070c68800270037004c
:102a5c001a417800644061002700320018007800a9
:102a6c000c80b9007a0040006d0078000000010075
:102a7c000004e00020003200180078000c80b9003f
:102a8c008002b0000d004000325b0200000000002c
:102a9c0050a02800325b02000000000010c480002f
:102aac0001c48000810f500013003200120032006c
:102abc00f0b79f00ffb197006bc07900da590200a4
:102acc00000000007fb29700f507200005006200af
:102adc000000e800f0b79f0000c480007fb39700af
:102aec00800f530004003200f2ff3700489e210093
:102afc000c0320000d8d21001c5902000000000069
:102b0c000004e000d2ff3200c65c020000000000ae
:102b1c000004e00003003200cc5c02000000000066
:102b2c00acff3700c85902000000000000447800d8
:102b3c000880fb008000eb00f2072000820f5000a1
:102b4c00e08f580056023e00006001004c02370036
:102b5c00120237000501370051023700b60037006a
:102b6c0021023700160137004d023700770037007d
:102b7c004b0237002f02370049023700480237005a
:102b8c002c0237007f01370045023700190137004e
:102b9c00430237004202370041023700400237003f
:102bac003f0237003e0237003d0237003c0237003f
:102bbc003b0237003a023700c600370038023700b4
:102bcc00370237003602370035023700340237003f
:102bdc00330237003202370031023700300237003f
:102bec002f0237002e0237002d0237002c0237003f
:102bfc002b0237002a02370029023700280237003f
:102c0c00270237002602370025023700240237003e
:102c1c00230237002202370021023700200237003e
:102c2c001f0237001e0237001d0237001c0237003e
:102c3c001b0237001a02370019023700180237003e
:102c4c00170237001602370015023700140237003e
:102c5c00130237001202370011023700100237003e
:102c6c000f0237000e0237000d0237000c0237003e
:102c7c000b0237000a02370009023700080237003e
:102c8c00070237000602370005023700040237003e
:102c9c00030237000202370001023700000237003e
:102cac00ff013700fe013700fd013700fc01370042
:102cbc00fb013700fa013700f9013700f801370042
:102ccc00f7013700f6013700f5013700f401370042
:102cdc00f3013700f2013700f1013700f001370042
:102cec00ef013700ee013700ed013700ec01370042
:102cfc00eb013700ea013700e9013700e801370042
:102d0c00e7013700e6013700e5013700e401370041
:102d1c00e3013700e2013700e1013700e001370041
:102d2c00df013700de013700dd013700dc01370041
:102d3c00db013700da013700d9013700d801370041
:102d4c00d7013700d60137003b00370010c4800094
:102d5c00800f57003400320000c48000800f5700f1
:102d6c0009003a000e07e900fe07b2000ec4880005
:102d7c008041eb0083757f00f0902800325b0200ed
:102d8c000000000013ff37000e07e900fe07b20039
:102d9c0070a02800325b02000000000000c480001c
:102dac000006eb00800f5700120032008e007800f6
:102dbc00fd0720000104e8006b407c0080f57800e2
:102dcc000004e00003003200da59020000000000a9
:102ddc000300370000c2b300da5902000000000003
:102dec000c06e8008d00640000c48000808f500049
:102dfc00f0ff3a000000e900f007b20000c48800c0
:102e0c00b0a02800325b0200000000000c407800eb
:102e1c00f059020000000000e0a02800325b020024
:102e2c0000000000ebfe370070c0b300da5902005e
:102e3c0000000000e7fe370000c48000800f570040
:102e4c00200032008e0078000006eb00fd07200009
:102e5c000104e8006b407c0080f578000004e00081
:102e6c0003003200da5902000000000003003700b2
:102e7c0000c2b300da590200000000000c06e800a2
:102e8c008d00640000c48000808f5000f0ff3a0079
:102e9c000000e900f007b20000c48800b0a02800d0
:102eac00325b0200000000000c407800f059020078
:102ebc0000000000e0a02800325b020000000000cf
:102ecc00c4fe370070c0b300da59020000000000e5
:102edc00c0fe3700c859020000000000b1c5b300a5
:102eec00814f5000bbfe3a00c859020000000000a0
:102efc0011c4b300814f50003e00320007003e0069
:102f0c00f0c05000814f50000c003200e3c0400074
:102f1c00814f5000affe3a000e00370031c4b300b1
:102f2c00814f500026003200960039008140e800a5
:102f3c00814f5000a7fe3a000c003700c859020020
:102f4c0000000000e1c7b300814f5000a1fe3a0021
:102f5c0012013700c859020000000000e1c7b3009d
:102f6c00814f50009bfe3a001f0137005fb2970063
:102f7c00e40f520005003400866d020000000000d2
:102f8c008002eb00d5b79f0092fe370010c4800082
:102f9c00800f5700060032000e07e900fe07b20052
:102fac0070a02800325b02000000000089fe370090
:102fbc0070c0b300da5902000000000085fe370033
:102fcc0000c48000800f5700060032000e07e80096
:102fdc00fe07b20000a12800325b020000000000d6
:102fec007cfe370070c0b300da590200000000000c
:102ffc0078fe370015c480000504e900f807b2001c
:10300c000806780002c48000820f54005900320078
:10301c000002eb00f00720000fbb9700eb407c0098
:10302c000104e0004e003a008800e9008080600056
:10303c00ebc178000304e000490032000402e80010
:10304c00860f520046003600010078000fbb970037
:10305c000603e80086bf9f00828f520009003200f1
:10306c00f30720000042eb00847579000201e900af
:10307c0003016100828f5200faff3a0002c48800fb
:10308c008475790002c48000820f50001000320059
:10309c006b407800f30720000004e00008003a00c1
:1030ac00030037006bc078000004e00004003a0015
:1030bc008100e800f107b200e1b79f00040037007f
:1030cc008100e90083806000828f5000f5ff3a0098
:1030dc0040a12800325b0200000000000003200029
:1030ec0022cf80000091b900818f210001004100a6
:1030fc00325b02000000000050a02800325b02008e
:10310c0000000000efb29700888f52000e003200d2
:10311c0085067800fe0720006bc07e00da5902009d
:10312c000000000000c480006df07d000000e8008d
:10313c000e00600000c488008d06e8008e866600d4
:10314c00888f5600f4ff3a000ec480000040eb005c
:10315c0080757f008e0f56001efe3a00050037006a
:10316c000804e9000004640008067800820f54008b
:10317c00aaff3a0070c0b300da5902000000000048
:10318c0014fe370016c480000604e900f807b200ec
:10319c000806780002c48000820f54005a003200e6
:1031ac000002eb00f00720008fb897008102e900c5
:1031bc00eb407c000104e0004e003a008800e9007e
:1031cc0080806000ebc178000304e000490032000d
:1031dc000402e800848f520046003a000100780097
:1031ec008fb997008301e90083bf9f00820f5300c2
:1031fc0009003200f30720000042eb0084757900cf
:10320c000201e90003016100820f5300faff3a004a
:10321c0002c488008475790002c48000820f5000bb
:10322c00100032006b407800f30720000004e0002f
:10323c0008003a00030037006bc078000004e0007f
:10324c0004003a008100e800f107b200e1b79f00ea
:10325c00040037008100e90083806000828f5000f9
:10326c00f5ff3a0040a12800325b0200000000008c
:10327c000003200022cf80000091b900818f210033
:10328c0001004100325b02000000000050a0280049
:10329c00325b020000000000efb29700888f5200f2
:1032ac000e00320085067800fe0720006bc07e0001
:1032bc00da5902000000000000c480006df07d00af
:1032cc000000e8000e00600000c488008d06e800d5
:1032dc008e866600888f5600f4ff3a000ec480007c
:1032ec000040eb0080757f008c0f5700b9fd3a0051
:1032fc00050037000804e9000004640008067800a3
:10330c00820f5400aaff3a008fb89700e18f50004b
:10331c001e003a0040a12800325b020000000000b1
:10332c000003200022cf80000091b900818f210082
:10333c0001004100325b02000000000050a0280098
:10334c00325b0200000000000ec4800010c480003c
:10335c00800f570008003200f10720000041eb00fd
:10336c0082757f000e07e90001076700800f570088
:10337c00faff3a000ec488008041eb0083757f0091
:10338c000002eb0084bf9f0092fd370070c0b300b9
:10339c00da590200000000008efd370018c48000ce
:1033ac00880f57000c003200b0a02800325b0200de
:1033bc000000000008005700f007b200f0590200ae
:1033cc0000000000e0a02800325b020000000000ba
:1033dc001ec480007ffd370070c0b300da590200b4
:1033ec00000000007bfd370008c48000880f5700e8
:1033fc000c003200b0a02800325b0200000000007c
:10340c000e005400f007b200f0590200000000005a
:10341c00a0a12800325b0200000000000ec4800056
:10342c006cfd370070c0b300da59020000000000d8
:10343c0068fd370000c480000044eb0001802100cf
:10344c00887078000000e80000077800fe07b200e2
:10345c000ec4880030912800125b020000000000ae
:10346c0005c48000f5b79f001dc480004088210072
:10347c000848780098ef9f00088021005100370021
:10348c005fb397000603e800d6b79f00f40f530014
:10349c0050fd3a00c25e0200000000004dfd3700f6
:1034ac000cc480008c00e800f107b20010c480004e
:1034bc00808f50003f003200ff4f54003d0036001b
:1034cc00e0c7b300804f54003a003e008c0f570009
:1034dc000c003a0008407800da59020000000000a5
:1034ec0000c48000887578000000e80000077800b0
:1034fc00fe07b2000ec488000040eb0080757f0010
:10350c0034fd3700b0a02800325b02000000000040
:10351c000e005600fd0720000d006000f05902005f
:10352c0000000000a0a12800325b02000000000097
:10353c000cc480000e00e9008d0660008d0f560053
:10354c00100032000c804500eb407e0011409800ca
:10355c006b407e000004e00005003200da590200e6
:10356c0000000000c0a12800325b02000000000037
:10357c000c06e900f2072000020666008d0f5600cb
:10358c00f0ff3a0008407800da5902000000000011
:10359c0088757f000e07e800f00720000007670021
:1035ac0001c480008100e8000080600000c4880035
:1035bc0008fd370070c0b300da59020000000000ab
:1035cc0004fd370012c48000684079000080fb00c5
:1035dc008000eb00e3072000830f5000e08f5800c1
:1035ec0035043e0000600100360437003204370019
:1035fc0031043700300437002f0437002e04370015
:10360c002d0437002c0437002b0437002a04370014
:10361c002c0437002804370027043700290437000e
:10362c002504370024043700230437002204370014
:10363c0021043700200437001f0437001e04370014
:10364c001d0437001c0437001b0437001a04370014
:10365c001904370018043700170437001604370014
:10366c00150437001404370016043700f50337002f
:10367c00870237002001370029013700d9013700b4
:10368c00c70137000c043700640237000a04370006
:10369c0009043700080437000a043700aa0337006e
:1036ac00c103370090033700e2023700e102370014
:1036bc00e0023700df023700de023700dd023700a0
:1036cc00dc023700db023700da023700d9023700a0
:1036dc00f9033700f8033700de013700c400370068
:1036ec00f503370046003700330137002901370056
:1036fc00f103370069003700a6013700ee033700ed
:10370c00ed033700ec033700eb033700ea03370017
:10371c00e9033700e80337006a003700e603370097
:10372c00e5033700e40337008c003700e203370071
:10373c00e1033700bc013700df033700de0337003d
:10374c00dd03370030013700db033700da033700c5
:10375c00d9033700980237006f033700a5023700f2
:10376c009f03370084033700d30337000001370071
:10377c002e0037004100370078013700ce033700a8
:10378c003000370032003700160037001f003700ba
:10379c00c9033700c8033700540037002100370035
:1037ac00c5033700230037005a003700c203370027
:1037bc00ff023700c0033700bf033700be033700da
:1037cc001e0037004a013700bb033700ba0337002d
:1037dc00b90337007f0237009e0037008d02370097
:1037ec00b800370063f907000000e000b5033a00a9
:1037fc001dc4800004c48000f4b79f00b1033700df
:10380c00146e020000000000ae03370040fa0700ff
:10381c0020cf80000000e000aa0332004efb07001e
:10382c00a8033700c7f90700a6033700ebfb070016
:10383c00a4033700cbfb0700a2033700defa070016
:10384c00a0033700ee4d0200000000009d0337007e
:10385c0020cf80000000e00005003a00d1012000dc
:10386c00505a20000a6e0200000000009503370039
:10387c007c4b02000000000092033700809c21006a
:10388c00c1cfb30010c8600061012000a057200018
:10389c000a6e0200000000008a033700819c2100a0
:1038ac00114078000000a0000014a10080487800ae
:1038bc0051012000005920000a6e02000000000097
:1038cc0080033700809c21001034a000c10120002f
:1038dc00e07e2000ae6d0200000000003091280058
:1038ec00125b02000000000076033700809c210070
:1038fc001034a100b1012000307d2000ae6d02001b
:10390c000000000030912800125b02000000000053
:10391c006c03370020cf80000000e00005003a0067
:10392c00d1012000505a20000a6e02000000000055
:10393c0064033700cb62a900c962a90051012000c1
:10394c00205c2000ae6d02000000000030912800c9
:10395c00125b0200000000005a03370020cf8000e9
:10396c000000e00005003a00d1012000505a200070
:10397c000a6e02000000000052033700809c2100f8
:10398c00104078007040600004003a0021022000d2
:10399c00f0e920000a6e020000000000c962a800d5
:1039ac00cb62a90041012000705d2000ae6d0200c9
:1039bc000000000030912800125b020000000000a3
:1039cc0021e3a800b0002000026b02000000000000
:1039dc00f1042000810f500003003e0010a22800cb
:1039ec00125b02000000000021e3a9003503370040
:1039fc000200e800f007b20010c488003ef807008f
:103a0c0057f707008004780009007800925c0200e8
:103a1c000000000040a42800325b020000000000ff
:103a2c0009407800f05902000000000040a4280072
:103a3c00325b02000000000009407800145c0200b8
:103a4c000000000030912800125b02000000000012
:103a5c001c0337000200e800f007b20010c4880015
:103a6c0025f807003ef707000080fb00686c020099
:103a7c00000000008004780009007800925c0200cd
:103a8c000000000040a42800325b0200000000008f
:103a9c0009407800f05902000000000040a4280002
:103aac00325b02000000000009407800145c020048
:103abc000000000030912800125b020000000000a2
:103acc000003370020cf80000000e00005003a0022
:103adc0011c0b30001407800a6660200000000008f
:103aec00f8023700a1012000b05e20000a6e02002f
:103afc0000000000f302370051002000506020004d
:103b0c000a6e0200000000001459020000000000c0
:103b1c000004e000fcff32000000fe00e902370068
:103b2c00a06e0200000000000004e000e50232007c
:103b3c00a1002000a06020000a6e0200000000001e
:103b4c00400620003e6c020000000000ca6a020021
:103b5c000000000014590200000000000004e00006
:103b6c00fcff320081bf2a0001400100d502370062
:103b7c0099f70700800478000900e000d1023200b8
:103b8c0042510200000000008904e900fcff3a00e9
:103b9c00cc02370090f70700800478000900e000a1
:103bac00c802320026510200000000008904e9001e
:103bbc00fcff3a00c302370087f707008004780047
:103bcc000900e000bf0232004a6120003b9128004e
:103bdc00610120000a007800ae6d020000000000b8
:103bec005e51020000000000b05c0200000000000a
:103bfc000b007800125b0200000000008904e90051
:103c0c00f3ff3a00af02370020cf80000000e00045
:103c1c0005003a00d1012000505a20000a6e020023
:103c2c0000000000a7023700c002a900c202a800d1
:103c3c0021e3a800200020003e6c020000000000e0
:103c4c00a0002000026b020000000000011b2000fd
:103c5c00810f50001800360090002000026b02000b
:103c6c0000000000712b2000810f50001200360064
:103c7c0011012000a0622000ae6d020000000000c7
:103c8c0030912800125b02000000000000032000ad
:103c9c0021cf80000088b9000002b000018d210006
:103cac00610078000000010080a42800125b020073
:103cbc00000000000c003700c002a900c202a900dd
:103ccc00a0a52800125b02000000000021012000ca
:103cdc00b0632000ae6d020000000000309128009f
:103cec00125b02000000000021e3a90075023700fe
:103cfc0020cf80000000e00005003a00d101200038
:103d0c00505a20000a6e0200000000006d023700bd
:103d1c00010320000180b9002002b000018d2100b8
:103d2c00610078000000010090912800125b0200f5
:103d3c0000000000c002a900c202a900210120005d
:103d4c00b0632000ae6d020000000000309128002e
:103d5c00125b0200000000005a023700f100200044
:103d6c00c0362000ae6d020000000000106b020097
:103d7c000000000011002000b0372000ae6d0200e2
:103d8c000000000030912800125b020000000000cf
:103d9c004c0237001e6b0200000000004902370085
:103dac000df707008004780061002000906520006a
:103dbc00ae6d02000000000009007800645a020099
:103dcc000000000021002000f06520000a6e0200b7
:103ddc000000000009007800106c020000000000d8
:103dec0038023700fcf607008004780061002000e0
:103dfc0090652000ae6d0200000000000900780004
:103e0c00645a0200000000002100200030ee200067
:103e1c000a6e020000000000090078003e6c0200ef
:103e2c00000000002702370020cf80000000e000d7
:103e3c0005003a00d1012000505a20000a6e020001
:103e4c00000000001f023700845102000000000037
:103e5c001c02370011c0b3004088210001487800d3
:103e6c000200e800f007b200e84078000104e0002e
:103e7c001402320014c0b300100020008042eb008a
:103e8c00f3072000e6c3b30086cf500001003a00d0
:103e9c00054278000000e80082004000838060004a
:103eac00e8c078000104e000f6ff3a0041882100e8
:103ebc0084487800fa0f50000400340011c0b3009d
:103ecc004088210001487800fe013700408821001d
:103edc001004e000fb013a0010c480000000e80070
:103eec00fa0720000a00600010c488001cf60700c6
:103efc008004780010c480000a05600068417d00d1
:103f0c00d1c3b300814f510021003a008900e90070
:103f1c00e28f50001a003e000000e800f007b200eb
:103f2c0010c48800010178007811b9004088210084
:103f3c0080004100010178000000eb008041eb00a3
:103f4c00036978000000e800f80f5000fcff3a000d
:103f5c0010c48000f307200003003700826878004b
:103f6c000000e8000300600068417800e4c3b3007f
:103f7c00844f5100f9ff3a0010c48800d10137007a
:103f8c0011c0b3004088210001487800cd013700f2
:103f9c000900e00015003a005a88210019002000a1
:103fac00aba728005ca0280009407800f05902005b
:103fbc00000000000b007800325b020000000000e3
:103fcc000a007800325b0200000000000c00780050
:103fdc00125b0200000000008904e800780545002f
:103fec00e48f5400f0ff3a00b60137000900e900f5
:103ffc00e20f500005003e0030912800125b0200d9
:10400c000000000079c68800ae01370011c0b30073
:10401c004088210001487800aa0137000200e8001e
:10402c00f90720000900600010c48800ccf50700d7
:10403c0000057800b0f6070010c480008904600009
:10404c00e8c07c0090c2b30080cf50000c003a0056
:10405c000003200021cf80000088b9007c004000c4
:10406c00018d2100e10078000a00780001000100b8
:10407c0030912800125b0200000000009101370013
:10408c0011c0b30040882100014878008d01370031
:10409c0011c0b30040882100014878000200e800fc
:1040ac00f007b200684078000004e000850132009f
:1040bc000281e800814178000042eb00f10720000a
:1040cc0025c2b300854f500001003a0084417800ae
:1040dc0001006100684078000201e8000004e00083
:1040ec00f7ff3a0040882100034878000304e00001
:1040fc0074013a007100200010662000ae6d0200c1
:10410c00000000000fe89700da59020000000000e0
:10411c0011c480008100e800f107b20068c078008b
:10412c0026c2b300864f50001b0032008a9c21002f
:10413c00499e21000b0320000c8d210011c4880026
:10414c00da5902000000000010c4800068407800ba
:10415c000000fb001a417800e840610002003200c8
:10416c00686c020000000000190178000b91b90086
:10417c00e8004100ec8078000100010011c48000cf
:10418c008100e800f107b20068c0780023c2b300d8
:10419c00834f5000e9ff3a0011c488000fe89700e4
:1041ac00da5902000000000030912800125b020076
:1041bc0000000000430137000003200021cf8000e5
:1041cc000088b900028d2100620078000000010017
:1041dc003c0137000003200021cf80000088b9008b
:1041ec000080e800018d21006100780000000100d2
:1041fc00340137000003200021cf80000088b90073
:10420c0064004000018d2100610078000000010075
:10421c002c0137000003200021cf80000088b9005a
:10422c0066004000018d2100610078000000010053
:10423c00240137007100200010662000ae6d0200d2
:10424c000000000046f507008005780010c48000cf
:10425c000000e900f007b20010c48800def507008a
:10426c008004e800f1f507000000e000480032008f
:10427c00719b210080487800e80f50000300340047
:10428c00718040001054a00041003700809c210038
:10429c001054a1003e0037000b007800846b020024
:1042ac000000000004c2b3001a40620005003a008e
:1042bc0086c0b300759b2100954f130005003a0092
:1042cc000b00370001c1b300709b210090cf100090
:1042dc0007003200b0c3b300da590200000000003e
:1042ec00729b210012407800f0590200000000007f
:1042fc009a41780068c06100040032000b0078001d
:10430c00686c020000000000800578001c0078003a
:10431c00040320000480b90068004000058d2100d2
:10432c00e50078000b0078000100010080bf9f00c1
:10433c0000c2b300da5902000000000006c4b3004a
:10434c001a406300140032006100200080662000d7
:10435c00ae6d0200000000009a40780068c060005a
:10436c00040032000fb89700686c020000000000d7
:10437c0080bf9f000fb89700846b02000000000004
:10438c0000c2b300da59020000000000020037003e
:10439c008a9c21004c9e21008904e900beff3a0052
:1043ac0030912800125b020000000000c5003700ad
:1043bc006100200080662000ae6d0200000000004d
:1043cc00aff5070080f79f0083f5070080047800a5
:1043dc0096f507000000e00009003200719b2100f7
:1043ec0080487800e80f50000300340071804000d2
:1043fc001054a00002003700809c21001054a10032
:10440c000ff197000204e00005003200209e21000d
:10441c009041780093ef9f008280fb000108e90037
:10442c000900e000260032004a9e21008b9c2100ee
:10443c00718655001a007800040320000480b9002e
:10444c006a004000058d2100650078000000010025
:10445c001b437800e840630002003200686c0200e5
:10446c0000000000846b02000000000001c2b300d9
:10447c001bc0600004003a0082c0b3009c4f1100c6
:10448c0004003a000900370003c1b3009ccf1100af
:10449c0006003200b0c3b300da590200000000007d
:1044ac001c407800f05902000000000000c2b3006c
:1044bc00da590200000000008904e900ddff3a002f
:1044cc000ff297000404e000030032009fea97000b
:1044dc000580fb0010cf880030912800125b020091
:1044ec00000000007700370081002000e06620000b
:1044fc000a6e0200000000000003200021cf8000a3
:10450c000088b9006c004000018d2100610078002a
:10451c00000001006b003700810020006067200064
:10452c000a6e0200000000000003200021cf800072
:10453c000088b9006e004000018d210061007800f8
:10454c00000001005f003700e1002000e067200060
:10455c000a6e0200000000000003200021cf800042
:10456c000088b90070004000018d210061007800c6
:10457c000000010053003700e1002000c06820005b
:10458c000a6e0200000000000003200021cf800012
:10459c000088b90072004000018d21006100780094
:1045ac000000010047003700c1002000d06420004b
:1045bc00ae6d0200000000000003200021cf80003f
:1045cc000088b90074004000018d21006100780062
:1045dc0000000100b05c0200000000003900370050
:1045ec00fdf4070080047800d1002000a06a2000b0
:1045fc00ae6d02000000000009007800846b020020
:10460c00000000000900e0000a0032004a9e210070
:10461c000b8d21009a007800000320000088b9005f
:10462c00760040006b007800000001008904e9006e
:10463c00f8ff3a0030912800125b020000000000e5
:10464c0020003700e4f4070080047800a10020006b
:10465c00706b2000ae6d0200000000000900e0004d
:10466c00100032004a9e21000b8d21009a00780028
:10467c00000320000088b900780040006b0078002f
:10468c00000001000080fb00b05c02000000000094
:10469c0000c2b300da590200000000008904e900ee
:1046ac00f2ff3a0001012000a06920000a6e02000e
:1046bc00000000000300370011c0b3004088210047
:1046cc000148780010c480000000e800f007b20038
:1046dc0010c488000001eb00408821001004e000a9
:1046ec001600320051012000106c2000ae6d02004b
:1046fc000000000010c48000808f560004003100c0
:10470c000d405000f0590200000000000500370079
:10471c0001c8b300014040000d405000f0590200a8
:10472c0000000000408821000048eb003091280078
:10473c00125b0200000000001200200000c4800088
:10474c0011c48000808f5000020032000200e00093
:10475c009cfb32007fb3970016c4880006c4880007
:10476c008df83700575249005445200042495400f7
:10477c003a2020002a6e650078742000636c6f006c
:10478c00636b2000285e2900207769006c6c200088
:10479c0075736500207468006973200076616c0085
:1047ac0075654e006f2064006576690063652c00aa
:1047bc002074720079202800414c4100524d290090
:1047cc00205345004152430048206d006163720044
:1047dc006f206600697273007441440044524500b6
:1047ec00535320004d414300524f200020302e00e7
:1047fc004d616300726f20006d656e00754d610038
:10480c0063726f0020202000202031005749520095
:10481c004520610064647200657373000d0a20000a
:10482c0020202a003157490052452000524f4d009c
:10483c0020434f004d4d41004e4420004d4143005c
:10484c00524f73003a0d0a00203531002e524500ac
:10485c0041442000524f4d00202830007833330063
:10486c0029202a00666f7200207369006e676c0045
:10487c0065206400657669006365200062757300cd
:10488c000d0a200038352e004d41540043482000bd
:10489c00524f4d00202830007835350029202a0051
:1048ac00666f6c006c6f7700656420006279200085
:1048bc0036346200697420006164640072657300b0
:1048cc00730d0a0020323000342e53004b49500037
:1048dc0020524f004d2028003078430043292000ff
:1048ec002a666f006c6c6f0077656400206279003b
:1048fc0020636f006d6d61006e640d000a20320044
:10490c0033362e00414c4100524d2000534541009e
:10491c00524348002028300078454300290d0a00f6
:10492c0020323400302e53004541520043482000c1
:10493c00524f4d00202830007846300029414c0061
:10494c0041524d002053450041524300482028005d
:10495c00307845004329530045415200434820001c
:10496c00283078004630290044657600696365007c
:10497c00204944007320610072652000617661005b
:10498c00696c6100626c650020627900204d410009
:10499c0043524f002c2073006565200028302900fd
:1049ac002e52450041442000524f4d00202830002b
:1049bc0078333300293a20004d41540043482000fd
:1049cc00524f4d00202830007835350029534b00cc
:1049dc0049502000524f4d002028300078434300ae
:1049ec0029556e006b6e6f00776e20006d61630051
:1049fc00726f2c002074720079203f00206f7200bf
:104a0c0020283000292066006f72200068656c0039
:104a1c007042550053205200455345005420570016
:104a2c0061726e00696e67003a202a0053686f004d
:104a3c00727420006f7220006e6f200070756c0015
:104a4c006c2d750070202a004e6f20006465760076
:104a5c0069636500206465007465630074656400b7
:104a6c00204453003138530032302000486967002d
:104a7c006820500072657300204469006720540060
:104a8c00686572006d4453003138420032302000aa
:104a9c0050726f00672052006573200044696700f4
:104aac002054680065726d00445331003832320076
:104abc00204563006f6e2000446967002054680035
:104acc0065726d004453320034303400204563006d
:104adc006f6e7200616d200074696d00652043007b
:104aec0068697000445332003433310020314b007c
:104afc002045450050524f004d556e006b6e6f00b7
:104b0c00776e2000646576006963650050574d0030
:104b1c0020646900736162006c656400314b48006d
:104b2c007a2d34002c303000304b48007a20500065
:104b3c00574d46007265710075656e0063792000f3
:104b4c00696e20004b487a00205072006573630038
:104b5c00616c65003a505200323a44007574790029
:104b6c0020637900636c650020696e0020252000ad
:104b7c0050574d0020616300746976006545520002
:104b8c00524f52003a205000574d20006163740080
:104b9c00697665002c20670020746f002064690022
:104bac00736162006c6541005558200046726500c7
:104bbc00717565006e6379003a20410055582000ec
:104bcc00494e500055542f0048492d005a4155006c
:104bdc00582048004947480041555800204c4f0088
:104bec0057564f004c544d004554450052204d0033
:104bfc004f444500564f4c0054414700452050004f
:104c0c00524f4200453a200056457200726f7200b6
:104c1c0028292000406c69006e653a002040700025
:104c2c00676d730070616300653a200062797400ef
:104c3c0065732e00546f6f00206c6f006e6721003f
:104c4c0053796e007461780020657200726f720087
:104c5c004e6f200045455000524f4d00457261008b
:104c6c0073696e0067646f006e655300617669004e
:104c7c006e672000746f2000736c6f007420490005
:104c8c006e7661006c69640020736c006f744c006c
:104c9c006f616400696e6700206672006f6d2000a2
:104cac00736c6f007420450052524f00523a200032
:104cbc00636f6d006d616e0064206800617320008d
:104ccc006e6f200065666600656374002068650081
:104cdc0072654100434b4e0041434b004932430047
:104cec002053540041525400204249005449320090
:104cfc0043205300544f5000204249005449320085
:104d0c0043206d006f6465003a0d0a0020312e00bf
:104d1c0020536f0066747700617265000d0a2000e5
:104d2c00322e200048617200647761007265530076
:104d3c00657420007370650065643a000d0a2000ec
:104d4c00312e20007e354b00487a0d000a203200af
:104d5c002e207e0035304b00487a0d000a2033009f
:104d6c002e207e00313030004b487a000d0a200096
:104d7c00342e20007e343000304b48007a574100ee
:104d8c00524e49004e473a002048410052445700c9
:104d9c0041524500204932004320690073206200d3
:104dac00726f6b00656e20006f6e20007468690076
:104dbc007320500049432100202852004556200002
:104dcc0041332900536574002073700065656400dd
:104ddc003a0d0a0020312e0020313000304b4800b3
:104dec007a0d0a0020322e0020343000304b48005f
:104dfc007a0d0a0020332e0020314d00487a4900ec
:104e0c0032432000286d6f00642073007064290009
:104e1c003d28200020302e004d616300726f200071
:104e2c006d656e00750d0a0020312e003762690029
:104e3c0074206100646472006573730020736500f4
:104e4c0061726300680d0a0020322e004932430063
:104e5c0020736e00696666006572530065617200ae
:104e6c00636869006e67200049324300206164006a
:104e7c0064726500737320007370610063652e00ab
:104e8c0020466f00756e64002064650076696300cf
:104e9c006573200061743a00536e690066666500a4
:104eac007228420041534900432952006561640055
:104ebc0079612f00412f400020636f006e747200e7
:104ecc006f6c73002041550058207000696e6100b2
:104edc002f412f00402063006f6e7400726f6c00c6
:104eec007320430053207000696e43006f6d6d009a
:104efc00616e6400206e6f00742075007365640031
:104f0c0020696e0020746800697320006d6f640066
:104f1c00655075006c6c2d00757020007265730007
:104f2c00697374006f727300204f46004650750011
:104f3c006c6c2d00757020007265730069737400c1
:104f4c006f727300204f4e0053656c00662d740019
:104f5c006573740020696e00204869005a206d004a
:104f6c006f646500206f6e006c79520045534500ec
:104f7c0054424f004f544c004f41440045524100a5
:104f8c0055582000494e500055542f0048492d00cb
:104f9c005a2c200052454100443a2000504f5700f3
:104fac004552200053555000504c490045532000a9
:104fbc004f4e50004f574500522053005550500053
:104fcc004c49450053204f00464644004154410093
:104fdc0020535400415445003a204400454c4100b4
:104fec005920750073575200495445003a2052001d
:104ffc00454144003a2043004c4f43004b2c2000c9
:10500c0031434c004f434b002c20300044415400a2
:10501c0041204f005554500055542c002031440071
:10502c0041544100204f550054505500542c200041
:10503c0030202a0070696e0020697300206e6f00aa
:10504c0077204800695a43004c4f43004b205400d2
:10505c0049434b00533a2000524541004420420042
:10506c0049543a00205379006e7461007820650031
:10507c0072726f00722061007420630068617200ac
:10508c0020782e00206578006974280077697400f8
:10509c00686f75007420630068616e006765290095
:1050ac006e6f20006d6f64006520630068616e0098
:1050bc00676523003a204e006f2073006f66740002
:1050cc0077617200652072006573650074206f0053
:1050dc006e207600342c20007573650020746800f7
:1050ec00652072006573650074206200757474002d
:1050fc006f6e2e004e6f6e006578690073746500dc
:10510c006e74200070726f00746f63006f6c2100fe
:10511c00782e200065786900740d0a00496e7600bf
:10512c00616c690064206300686f690063652c0022
:10513c002074720079206100676169006e4445003b
:10514c00564944003a68740074703a002f2f64007a
:10515c00616e670065726f0075737000726f74001a
:10516c006f747900706573002e636f006d2a2d00cb
:10517c002d2d2d002d2d2d002d2d2d002a4f7000a5
:10518c00656e200064726100696e20006f7574009a
:10519c007075740073202800483d4800692d5a0032
:1051ac002c204c003d474e0044294e006f726d0080
:1051bc00616c20006f75740070757400732028008a
:1051cc00483d33002e3376002c204c003d474e00da
:1051dc0044294d0053422000736574003a204d0061
:1051ec004f535400207369006720620069742000db
:1051fc006669720073744c0053422000736574002e
:10520c003a204c004541530054207300696720003c
:10521c0062697400206669007273740020426f002a
:10522c006f746c006f616400657220007620310031
:10523c002e20480045580d000a2032002e20440034
:10524c0045430d000a2033002e204200494e0d002c
:10525c000a2034002e20520041574400697370001c
:10526c006c61790020666f00726d610074207300b0
:10527c00657456006f6c740061676500206d6f007b
:10528c006e6974006f7273003a203500563a200034
:10529c00207c2000332e3300563a2000207c200046
:1052ac00565055004c4c5500503a20005365740034
:1052bc0020736500726961006c2070006f7274005d
:1052cc0020737000656564003a20280062707300da
:1052dc00290d0a0020312e0020333000300d0a0039
:1052ec0020322e002031320030300d000a203300e5
:1052fc002e203200343030000d0a2000342e2000d5
:10530c0034383000300d0a0020352e00203936009c
:10531c0030300d000a2036002e203100393230009a
:10532c00300d0a0020372e00203338003430300086
:10533c000d0a2000382e20003537360030300d0095
:10534c000a2039002e2031003135320030300d006a
:10535c000a3130002e204200524720007261770043
:10536c00207661006c75650041646a007573740089
:10537c0020796f0075722000746572006d696e0083
:10538c00616c410072652000796f750020737500a7
:10539c0072653f002043460047313a0020434600e7
:1053ac0047323a00285c2d002f5f5c002d29280025
:1053bc005c5f2f002d295300656c65006374200021
:1053cc006f757400707574002074790070653a0004
:1053dc000d0a2000312e20004f7065006e206400f5
:1053ec00726169006e202800483d4800692d5a0002
:1053fc002c204c003d474e0044290d000a20320061
:10540c002e204e006f726d00616c200028483d000c
:10541c00332e3300562c20004c3d47004e442900bf
:10542c0052325700202873007064200068697a009b
:10543c00293d2800202030002e4d610063726f0042
:10544c00206d65006e750d000a2031002e49530049
:10545c004f37380031362d003320410054520d00a7
:10546c000a2032002e4953004f37380031362d00b8
:10547c00332070006172730065206f006e6c7900d0
:10548c0049534f002037380031362d00332041006e
:10549c00545220002852450053455400206f6e0092
:1054ac0020435300290d0a00524553004554200057
:1054bc0048494700482c2000434c4f00434b2000e8
:1054cc00544943004b2c20005245530045542000b6
:1054dc004c4f570049534f002037380031362d00c0
:1054ec003320720065706c0079202800757365009c
:1054fc007320630075727200656e7400204c53004b
:10550c004220730065747400696e6700293a2000ac
:10551c0050726f00746f63006f6c3a0020736500fb
:10552c00726961006c33200077697200653220006b
:10553c00776972006552460055756e006b6e6f0090
:10554c00776e5200656164002074790070653a00d2
:10555c0020746f0020656e006476610072696100d2
:10556c00626c6500206c65006e67740068446100b5
:10557c0074612000756e690074733a00206e6f00c0
:10558c0020696e0064696300617469006f6e440089
:10559c006174610020756e00697420006c656e008a
:1055ac00677468002028620069747300293a20002f
:1055bc0043532000454e4100424c450044435300a8
:1055cc0020444900534142004c454400523357009b
:1055dc00202873007064200063736c0020686900dd
:1055ec007a293d00282029000d0a440069736300c4
:1055fc006f6e6e006563740020616e00792064002c
:10560c0065766900636573000d0a43006f6e6e006a
:10561c00656374002028560070752000746f20009c
:10562c002b355600292061006e642000284144006f
:10563c00432074006f202b00332e33005629430077
:10564c0074726c00415558004d4f440045204c007d
:10565c0045445000554c4c005550200048505500c6
:10566c004c4c550050204c005652450047414400cc
:10567c00432061006e64200073757000706c7900bb
:10568c0035565600505533002e33560041444300d6
:10569c0042757300206869006768420075732000ca
:1056ac0048692d005a20300042757300204869006b
:1056bc002d5a2000314d4f0044452000616e64008e
:1056cc0020565200454720004c454400732073007f
:1056dc00686f75006c642000626520006f6e21009d
:1056ec00466f75006e64200020657200726f720048
:1056fc00732e4d004f534900434c4b004d49530002
:10570c004f435300204f4b0020464100494c53005f
:10571c00657420007370650065643a000d0a200002
:10572c00312e200033304b00487a0d000a20320015
:10573c002e20310032354b00487a0d000a20330000
:10574c002e20320035304b00487a0d000a203400f0
:10575c002e2031004d487a00436c6f00636b2000a3
:10576c00706f6c006172690074793a000d0a200048
:10577c00312e200049646c0065206c006f7720008e
:10578c002a646500666175006c740d000a20320095
:10579c002e204900646c65002068690067684f0022
:1057ac007574700075742000636c6f00636b20005f
:1057bc0065646700653a0d000a2031002e2049000f
:1057cc00646c650020746f0020616300746976005e
:1057dc00650d0a0020322e002041630074697600aa
:1057ec00652074006f206900646c6500202a6400d9
:1057fc0065666100756c7400496e700075742000ec
:10580c0073616d00706c65002070680061736500d9
:10581c003a0d0a0020312e00204d690064646c00a2
:10582c0065202a006465660061756c00740d0a00c1
:10583c0020322e0020456e00645350004920280071
:10584c007370640020636b00702073006b65200024
:10585c00736d7000206373006c206800697a2900f6
:10586c003d28200020302e004d616300726f200017
:10587c006d656e00750d0a0020312e00536e6900a7
:10588c0066662000435320006c6f77000d0a2000e1
:10589c00322e53006e696600662061006c6c20002d
:1058ac007472610066666900632d7000202d6600bd
:1058bc00202a42007974650073206400726f7000b6
:1058cc00706564002a464100494c4500442c200078
:1058dc004e4f20004441540041446100746120004b
:1058ec0062697400732061006e6420007061720044
:1058fc00697479003a0d0a0020312e0020382c00f2
:10590c00204e4f004e4520002a64650066617500ec
:10591c006c7420000d0a2000322e2000382c200040
:10592c00455645004e200d000a2033002e2038002d
:10593c002c204f00444420000d0a2000342e20005f
:10594c00392c20004e4f4e00455374006f702000d0
:10595c0062697400733a0d000a2031002e20310068
:10596c00202a640065666100756c74000d0a2000c5
:10597c00322e200032526500636569007665200086
:10598c00706f6c006172690074793a000d0a200026
:10599c00312e200049646c0065203100202a6400ff
:1059ac0065666100756c74000d0a2000322e2000b3
:1059bc0049646c0065203000554152005420280089
:1059cc0073706400206272006720640062702000b3
:1059dc007362200072787000206869007a293d009b
:1059ec0028202000302e4d00616372006f206d0066
:1059fc00656e75000d0a2000312e540072616e0028
:105a0c007370610072656e007420620072696400cc
:105a1c0067650d000a2032002e4c69007665200067
:105a2c006d6f6e0069746f00720d0a0020332e00ca
:105a3c004272690064676500207769007468200011
:105a4c00666c6f00772063006f6e7400726f6c0071
:105a5c000a0d2000342e410075746f002042610045
:105a6c00756420004465740065637400696f6e0092
:105a7c0055415200542062007269640067655200ff
:105a8c0065736500742074006f206500786974007c
:105a9c00526177002055410052542000696e70000d
:105aac007574550041525400204c49005645200055
:105abc0044495300504c4100592c20007d20540087
:105acc004f205300544f50004c4956004520440081
:105adc00495350004c415900205354004f50500032
:105aec004544570041524e00494e47003a20700041
:105afc00696e7300206e6f0074206f0070656e000d
:105b0c002064720061696e0020284800695a2900df
:105b1c0020524500564944003a0d0a00496e760061
:105b2c00616c690064206300686f690063652c0018
:105b3c002074720079206100676169006e6d7300da
:105b4c00525320004c4f57002c2043004f4d4d001a
:105b5c00414e4400204d4f00444552005320480014
:105b6c00494748002c20440041544100204d4f002f
:105b7c00444541006464720065737300206f6600d5
:105b8c00205043004638350037343f0054686900d4
:105b9c0073206d006f64650020726500717569007b
:105bac007265730020616e00206164006170740086
:105bbc0065724c004344200074797000653a0d0006
:105bcc000a2031002e20480044343400373830008d
:105bdc002028750073696e0067205000434638001a
:105bec003537340020494f002065780070616e0015
:105bfc0064657200294c43004420280074797000bd
:105c0c002061640064722900203d200028202000bf
:105c1c00302e4d00616372006f206d00656e750053
:105c2c000d0a2000312e4c004344200052657300b5
:105c3c0065740d000a2032002e496e006974200034
:105c4c004c4344000d0a2000332e43006c65610068
:105c5c0072204c0043440d000a2034002e43750082
:105c6c0072736f00722070006f73690074696f003b
:105c7c006e206500783a280034292000300d0a0087
:105c8c0020362e005772690074652000746573000d
:105c9c0074206e00756d620065727300206578006b
:105cac003a28360029203800300d0a0020372e0003
:105cbc00577269007465200074657300742063006a
:105ccc00686172006163740065727300206578000e
:105cdc003a283700292038003044690073706c0072
:105cec00617920006c696e0065733a000d0a200022
:105cfc00312e200031200d000a2032002e204d00c4
:105d0c00756c740069706c0065494e004954430011
:105d1c004c4541005243550052534f005220530002
:105d2c0045544e006f204100434b2c00206368000b
:105d3c0065636b00206164006170740065724300e0
:105d4c004c4b09004d4f53004909430053094d007a
:105d5c0049534f0050696e00737461007465730091
:105d6c003a474e00440933002e33560009352e00b5
:105d7c003056090041444300095650005509410072
:105d8c0055580900500950000950090049094900ab
:105d9c00092d09004f574400092d09002d2d09002c
:105dac0054784400092d09005278440053434c00a8
:105dbc000953440041092d00092d500047430900a7
:105dcc0050474400092d09002d312e002842520065
:105ddc00290932002e28520044290900332e2800ac
:105dec004f52290009342e00285957002909350033
:105dfc002e2847004e290900362e2800424c290037
:105e0c0009372e0028505500290938002e28470044
:105e1c0052290900392e28005754290009302e0028
:105e2c0028426c006b2947004e440900474e440041
:105e3c0009414400430935002e30560009332e0029
:105e4c003356090056505500094155005809650054
:105e5c007865630075746500203a20002061750038
:105e6c00746f7200616e670065202b004d487a00dc
:105e7c00292b6b00487a290052617700207661004b
:105e8c006c75650020666f0072204200524720003e
:105e9c00284d490044493d00313237002957410013
:105eac00524e49004e473a0020506f007373690000
:105ebc00626c65002062750066666500726f760024
:105ecc00657266006c6f7700416e7900206b65001f
:105edc00792074006f20650078697400537061003c
:105eec0063652000746f2000636f6e0074696e0030
:105efc0075654e00756d6200657220006f6620003e
:105f0c006269740073207200656164002f777200ff
:105f1c00697465003a204300533a0d000a203100a1
:105f2c002e204300530d0a0020322e00202f430058
:105f3c0053202a006465660061756c0074506f0014
:105f4c0073697400696f6e0020696e0020646500cf
:105f5c006772650065735300657276006f2061008f
:105f6c00637469007665570061697400696e670037
:105f7c002061630074697600697479002e2e2e00fe
:105f8c002a2a2000456172006c792000457869004e
:105f9c0074212a002a42610075643e0031366d007e
:105fac003a20420050204300616e6e006f74200056
:105fbc006d6561007375720065203e0020313600fe
:105fcc0030303000303030002c2044006f6e6500d3
:105fdc002e0a0d0043616c0063756c0061746500e2
:105fec00643a2000090a0d0045737400696d610064
:105ffc00746564003a202000092062007073200050
:10600c0047656e00657261006c0909000909090099
:10601c0050726f00746f63006f6c2000696e7400b7
:10602c0065726100637469006f6e20002d2d2d0068
:10603c002d2d2d002d2d2d002d2d2d002d2d2d0038
:10604c002d2d2d002d2d2d002d2d2d002d2d2d0028
:10605c002d2d2d002d2d2d002d2d2d002d2d2d0018
:10606c002d2d2d002d2d2d002d2d2d002d2d2d0008
:10607c002d2d2d002d2d2d002d2d2d002d2d2d00f8
:10608c002d2d2d002d2d2d002d2d2d002d2d2d00e8
:10609c00203f09005468690073206800656c70002b
:1060ac000909090028302900094c69007374200083
:1060bc006375720072656e0074206d00616372000e
:1060cc006f7320003d582f007c580900436f6e0001
:1060dc007665720074732000582f72006576650027
:1060ec0072736500205809000928780029094d00b1
:1060fc00616372006f207800207e090053656c008c
:10610c00667465007374090009095b000953740017
:10611c0061727400202309005265730065742000bd
:10612c0074686500204250002020200009090900f5
:10613c005d095300746f7000202409004a756d00ce
:10614c00702074006f2062006f6f74006c6f6100c0
:10615c006465720009097b00095374006172740054
:10616c002077690074682000726561006420260045
:10617c002f25090044656c006179200031207500e1
:10618c00732f6d0073090900097d090053746f00aa
:10619c00702061002f412f004009410055585000dc
:1061ac00494e2000286c6f00772f4800492f520071
:1061bc00454144002909090022616200632209005b
:1061cc0053656e0064207300747269006e67200062
:1061dc00620953006574200062617500647261008d
:1061ec00746509000909310032332000632f430024
:1061fc00094155005820610073736900676e6d008a
:10620c00656e74002028610075782f0043532900b7
:10621c000909300078313200332064002f44090022
:10622c004d65610073757200652041004443200088
:10623c00286f6e0063652f00434f4e00542e2900cb
:10624c000930620031313000095365006e64200062
:10625c0076616c007565200066094d006561730000
:10626c00757265002066720065717500656e63005d
:10627c0079090900720952006561640020672f00da
:10628c0053094700656e650072617400652050000b
:10629c00574d2f0053657200766f0900092f0900c6
:1062ac00434c4b002068690020680900436f6d0067
:1062bc006d616e006468690073746f007279090017
:1062cc0009095c0009434c004b206c006f206900ed
:1062dc0009566500727369006f6e69006e666f0017
:1062ec002f7374006174750073696e00666f09001a
:1062fc00095e0900434c4b0020746900636b20005d
:10630c006c2f4c0009426900746f72006465720056
:10631c0020286d0073622f004c534200290909009c
:10632c002d09440041542000686920006d09430088
:10633c0068616e00676520006d6f64006509090077
:10634c00095f090044415400206c6f00206f090064
:10635c0053657400206f75007470750074207400a0
:10636c0079706500090909002e0944004154200088
:10637c0072656100642070002f50090050756c002c
:10638c006c7570002072650073697300746f720015
:10639c00732028006f6666002f4f4e0029092100dc
:1063ac000942690074207200656164002073090061
:1063bc00536372006970740020656e0067696e002b
:1063cc0065090900093a090052657000656174009d
:1063dc0020652e00672e2000723a310030207600a6
:1063ec00095368006f772000766f6c0074732f0070
:1063fc00737461007465730009092e000942690009
:10640c0074732000746f200072656100642f770034
:10641c0072697400652065002e672e0020307800ac
:10642c0035352e00322077002f5709005053550078
:10643c0020286f0066662f004f4e290009093c008a
:10644c00783e2f003c783d00203e2f003c303e0033
:10645c000955730065726d00616372006f207800de
:10646c002f617300736967006e2078002f6c6900d0
:10647c0073742000616c6c00809c21001064a0007f
:10648c0020a2210010407800684060000500320016
:10649c00cac2a900f0c2b300da5902000000000021
:1064ac0001003700cac2a800a100200090ab200058
:1064bc000a6e02000000000000000600809c210013
:1064cc001064a10020a221001040780068406000f8
:1064dc0005003200cac2a900f0c2b300da590200aa
:1064ec000000000001003700cac2a800a100200073
:1064fc0090ab20000a6e02000000000000000600b5
:10650c0020a2210010407800684060000500320095
:10651c00cac2a800f0c2b300da59020000000000a1
:10652c0001003700cac2a900b100200030ac200025
:10653c000a6e02000000000000000600881f7800b0
:10654c000102200000ca2000ae6d02000000000015
:10655c00609b21001040e800f05902000000000090
:10656c0000c2b300da5902000000000028a221008a
:10657c009840780061c06000f059020000000000f3
:10658c0000c2b300da590200000000001800d1006c
:10659c0061406000f05902000000000000c2b3002e
:1065ac00da59020000000000180078004200de00fa
:1065bc0061406000f05902000000000000c2b3000e
:1065cc00da59020000000000180078004300de00d9
:1065dc0061406000f05902000000000000c2b300ee
:1065ec00da59020000000000809c21001080fb00a2
:1065fc004400de0061406000f05902000000000021
:10660c0000c2b300da590200000000003100200083
:10661c0020ae2000ae6d0200000000004f04780098
:10662c0000000600889fbe008a9fbe008c1f780069
:10663c00820d020000000000b60b020000000000fa
:10664c0000047800820d020000000000b60b02006e
:10665c000000000080047800820d020000000000a1
:10666c00b60b02000000000000057800820d02004d
:10667c0000000000b60b020000000000800578004e
:10668c00820d020000000000b60b020000000000aa
:10669c0000067800820d020000000000b60b02001c
:1066ac00000000008800e900e38f500003003e006a
:1066bc00619b21008848e900010037000004eb00d1
:1066cc008900e900e18f500007003e0021a2210063
:1066dc008944e900e1c46400114178000204a1007e
:1066ec0089487100010037000004eb008a00e900c2
:1066fc00e18f500008003e0021a221000a45e9006c
:10670c00614565000a454500114178000214a1005d
:10671c008a487100010037000004eb008b00e9008f
:10672c00e18f500009003e0021a221008b45e900b9
:10673c00e1c5650022002000825ddd00114178007a
:10674c000224a1008b487100010037000004eb000b
:10675c008c00e900e18f500009003e0021a22100cd
:10676c000c46e90061466600320020000266dd003e
:10677c00114178000234a1008c48710001003700ef
:10678c000004eb008000e900e18f500009003e009e
:10679c00819c210061406000420020000200dd006d
:1067ac00114178000244a100804871000800e0000b
:1067bc0062003a00408821000048eb007103200081
:1067cc0000bc20000a6e0200000000008001eb00fb
:1067dc00420020001100200010002000a20d020039
:1067ec0000000000619b21008048e900510320005b
:1067fc0070bf20000a6e0200000000008001eb0058
:10680c00220020001100200010002000a20d020028
:10681c000000000028a221000040e9006140600057
:10682c00984078000104a10000cc700031042000d5
:10683c00c0c220000a6e0200000000008001eb00c4
:10684c00220020001100200020002000a20d0200d8
:10685c00000000000040e900614060000040400082
:10686c00984078000114a10000cc700011032000a6
:10687c00f0c620000a6e0200000000008001eb0050
:10688c00220020001100200010002000a20d0200a8
:10689c00000000000040e900614060002900200079
:1068ac000900dd00984078000124a10000cc7000a4
:1068bc00d1012000601c21000a6e020000000000c3
:1068cc008001eb000901780011002000090078001c
:1068dc00a20d0200000000000040e90061406000d1
:1068ec00310020000100dd00984078000134a10047
:1068fc0000cc7000f1042000e09320000a6e02002e
:10690c00000000008001eb0009017800110020005c
:10691c0010002000a20d020000000000819c21004c
:10692c0061406000420020000200dd00114178004f
:10693c000244a1008048710001003700fffe0700ef
:10694c00809c21001064a1004f0678004f05be000a
:10695c004f04be000000060001012000400621008b
:10696c000a6e0200000000000000060041e2a900cf
:10697c00819c210091407800f0c06000040032003e
:10698c00cf22a800cf02a800cec2a8000300370077
:10699c00cf22a900cf02a900cec2a90001fe2f0070
:1069ac0043358000038160007200b30042358800db
:1069bc00f30f2e00423680008281610002702000ad
:1069cc0003017100423688004336800083806000ea
:1069dc000130a00041368800cac2a800c8c2a90074
:1069ec00c902a900c8e2a800c922a9000080fb00c6
:1069fc001012880042a2a80010d18000e1006000b3
:106a0c00c608dd00f2fb2f001312800003016100a9
:106a1c000281700012128800c700dd000110b20064
:106a2c00f2ef2f001312800003016100028170004d
:106a3c00121288004700dd000020b200f1df2f00a9
:106a4c001212800082806000810070001112880098
:106a5c004422ef004022ef0041e2a80000000600b3
:106a6c00609b21001080fb0051b62800614078002b
:106a7c00beff070010d180004300dd000004b2000f
:106a8c00f1fb2f00521680008280600081007000a4
:106a9c00511688000000060041e2a9004035800034
:106aac00f001b30040358800f00f2e00c826b60068
:106abc0000fe2f00c826b600cf22a900cf02a900e5
:106acc00cec2a90000000600f3ff0700000006007c
:106adc000080fb004012880001402000220480004e
:106aec0002806000fdff3200401280008540a9004a
:106afc0000000600f6ff070000417800819c210091
:106b0c0000c4b300914060000000eb0001003200b3
:106b1c000280fb000000060000c0eb00ecff070049
:106b2c000080fb0000000600c8c2a800c902a80033
:106b3c00c8e2a800c922a80000fe2f005235800030
:106b4c00820060006100b30051358800743580000c
:106b5c00840060006100b300713588004535800009
:106b6c00850060009100b30041358800f20f2e00c3
:106b7c004635800086016100018020008381700011
:106b8c0043358800ac06b6007000b3006035880051
:106b9c006035800000016100028170006235880060
:106bac00609b21001080fb0051b6280061427800e8
:106bbc000482fb001412880010d180006101600077
:106bcc004611dd00f3fb2f0015128000858061005b
:106bdc0081007100111288004700dd000010b20026
:106bec00f1ef2f0016128000868260008502700083
:106bfc00151288004422ef004022ef001413880085
:106c0c0014138000848161008301710013138800c8
:106c1c0015138000858060008100700011138800be
:106c2c006422ef006022ef004822ef006822ef00a0
:106c3c004322a9006322a9004362a80042a2a90032
:106c4c006362a80062a2a90040c2a90060c2a900a8
:106c5c004402a8006402a8000000060041e2a9005a
:106c6c004362a90061e2a9006362a900503580006b
:106c7c00f001b3005035880070358000f001b3008e
:106c8c007035880040358000f001b3004035880035
:106c9c004135800000f021008100700041358800f2
:106cac0061358000f101b3006135880061358000e9
:106cbc00810070006135880000000600889fbe00ce
:106ccc008a9fbe008c9fbe008046780001467800eb
:106cdc0009022000ab9e2100225902000000000096
:106cec006dff070090ff07000d04e00003003a0061
:106cfc0042e2a80062e2a80002003700e1cf560091
:106d0c0002003e0041e2a80061e2a8001ac0b300f4
:106d1c00080037000a04e00006003a00cac2ab00c3
:106d2c0004003200d0c5b3008459020000000000fa
:106d3c001ac0b300011280000180640023003a00e5
:106d4c00011380000180640020003a00481280008a
:106d5c00e14f550004003a00b0c5b300845902005d
:106d6c00000000000045eb000c04e0000e003200b7
:106d7c000880fb00a85902000000000048138000a6
:106d8c0080c2b30084590200000000000880fb00a0
:106d9c00a85902000000000090c2b3008459020000
:106dac000000000009003700c0c5b3008459020080
:106dbc000000000008407800845902000000000028
:106dcc0040138000845902000000000040c2ab0058
:106ddc0006003a0060c2ab0004003a00002020001c
:106dec001b0060001000320005003700002020005e
:106dfc001b00600002003a00525902000000000023
:106e0c004022ef006022ef000c04e000040032008e
:106e1c0060b42800125b020000000000aeff3700d7
:106e2c00c222a9000d0037003059020000000000fa
:106e3c001c59020000000000e14f5000b5ff3a0061
:106e4c00c8590200000000000c04e00003003200ee
:106e5c0070b52800125b0200000000007fff0700e5
:106e6c00609b21001080fb0051b628006140780027
:106e7c00befe07004f06be004f05be004f04be000d
:106e8c00000006008000eb00ef0f5000e08f580070
:106e9c0057003e00006001000f0037001300370060
:106eac001e003700560037005100370050003700e5
:106ebc004f0037004e0037004d0037004c003700b4
:106ecc002200370024003700260037002800370046
:106edc002a0037002c0037004103200000cc200092
:106eec000a6e02000000000045003700710020000f
:106efc00705620000a6e020000000000f100200015
:106f0c00b01821000a6e02000000000011c0b3008e
:106f1c000040eb0069ff07003900370071002000ca
:106f2c00705620000a6e020000000000f1002000e4
:106f3c00b01821000a6e02000000000011c0b3005e
:106f4c00014078005dff07002d00370020a22100d2
:106f5c001004a1000e00370020a221001004a00094
:106f6c000b00370020a221001014a10008003700ec
:106f7c0020a221001014a0000500370020a221003f
:106f8c001024a1000200370020a221001024a00030
:106f9c0010d18000e1006000c608dd00f2fb2f007c
:106fac00131280000301610002817000121288002c
:106fbc00c700dd000110b200f2ef2f0013128000a9
:106fcc000301610002817000121288004700dd008d
:106fdc000020b200f1df2f001212800082806000ce
:106fec00810070001112880054fd07000400370066
:106ffc0041022000e01d20000a6e0200000000008b
:10700c000000060080b52800325b02000000000082
:10701c0000000600ea874700889fbe008a9fbe00da
:10702c008c9fbe008e1f780011c0b300609b2100a6
:10703c000148780021a22100114078000000a10035
:10704c000010a0000020a10080487800809c210046
:10705c001044a00080c1b30044fe0700e9ff070004
:10706c0059a221004aa221006b9b2100c8590200a1
:10707c0000000000804c78000081fb004411de0011
:10708c00024d7800e44f51002701320005003e000c
:10709c000204e00008003200e14f510051013a00b7
:1070ac000d013700e64f510025013200e84f510029
:1070bc004c013a002d013700e54f50000a003e000c
:1070cc00e44f500030003100e14f5000140032000a
:1070dc000c003900e24f500013003200e34f500017
:1070ec00f9003a0015003700ed4f5000180032003f
:1070fc00ee4f50001d003200e64f5000f2003a00f7
:10710c007300370064fe07004f0778004f06be007f
:10711c004f05be004f04be00af00b10000000600da
:10712c00b8ff0700d1ff3700ccc2a90010c0b300d4
:10713c00da59020000000000ccff3700ccc2a800d6
:10714c0010c0b300da59020000000000c7ff37007e
:10715c0010c0b300da590200000000008040eb00c0
:10716c0010c0b300d5fe0700c0ff370010c0b3003d
:10717c00da590200000000008040eb00014078006a
:10718c00cefe0700b9ff3700c8590200000000000e
:10719c004804dd00c8590200000000000086fb0016
:1071ac0008067600c8590200000000000044780070
:1071bc00c85902000000000001002100810f560098
:1071cc000a003e00c846dd000080fb008d06700002
:1071dc0001007800808f560004003e000004eb0094
:1071ec000c00e00005003a000c0037000040eb00fa
:1071fc00da590200000000009cff3700e09d2100de
:10720c0010074400c859020000000000004f78002d
:10721c000804e800880f5600f8ff3e0041c0b30098
:10722c0099cf100001003a00cac2a9000c00e0007e
:10723c00070032000004eb00f0ce800060407c00c0
:10724c0023fe07000804e800880f5600faff3e00f2
:10725c0010002000106c0200000000000d00e00087
:10726c00090032000004eb00ee9d21001e064400d4
:10727c0000c0eb0016fe0700004e78000804e80082
:10728c00888f5600f9ff3e0042c0b300994f1100a1
:10729c0001003a00cac2a80010c0b300da590200bb
:1072ac00000000000d00e00070ff32000004eb0055
:1072bc00f0ce800060407c00da5902000000000033
:1072cc000804e800888f5600f9ff3e0067ff37007e
:1072dc0010c0b300da59020000000000c8590200c7
:1072ec0000000000804c7800e14f50000800320094
:1072fc0003003900e24f50006f003a000e003700d7
:10730c0010c0b300da5902000000000057ff37002c
:10731c0010c0b300da590200000000000040eb007e
:10732c00da5902000000000010c0b300da59020064
:10733c00000000004dff3700480020006022b8001c
:10734c00f4b79f0085bf9f00c859020000000000e1
:10735c00804c78007fb297008fba97004829dd00e7
:10736c00c821de00830171004821dd000080fb0094
:10737c008000eb000202700083827000f4b79f0063
:10738c0085bf9f000804e900efff3a004800200089
:10739c006066b800c859020000000000804c7800fc
:1073ac004869dd00c861de00830171004861dd00c1
:1073bc000086fb008006eb000206760083867600d2
:1073cc000804e900f3ff3a00dcb79f00edb79f001b
:1073dc007fb197008fb99700e10f4100e08f590002
:1073ec0008003e00e10f4600e08f5e0005003e0005
:1073fc000c0041008d804900e10f4000e08f5800e7
:10740c00040036000040eb00da59020000000000d6
:10741c0016ff370010c0b300da590200000000005c
:10742c005fb09700efb09700e00f5000e08f58006e
:10743c000eff32007fb4970000c2b300a4fd07001a
:10744c004840de0000477800a1fd0700e8ef9f00f0
:10745c00084078009efd07000040eb009cfd0700f3
:10746c00da59020000000000120020000300200086
:10747c00820f5600838f5e00fcfe320080c2b30088
:10748c0093fd07000e40780091fd07006fe8970010
:10749c008ffd07000040eb008dfd0700da5902005c
:1074ac000000000062065600e0865e00effe32002f
:1074bc000804e800e0ff37000040eb00da59020056
:1074cc0000000000e9fe37000040eb00da59020032
:1074dc0000000000e5fe37006f406000804ce800c3
:1074ec0010c0b300da5902000000000030a22100e5
:1074fc000048eb001904e000dcfe320000047800c8
:10750c00c85902000000000071fd0700da590200a2
:10751c00000000001840e800004c7800994f100063
:10752c00f7ff3e00d1fe3700de71020000000000c4
:10753c0010c0b300da59020000000000cbfe370087
:10754c0067406000804c7800804d78000080fb0024
:10755c00d1b528006140780004fd070010c0b300cd
:10756c00da59020000000000c0fe370021a2210001
:10757c0082cfb30091486100819c21001144a1008d
:10758c000080fb000028a3000200320021a2210091
:10759c001104a0000018a3000200320021a2210057
:1075ac001114a0000008a3000200320021a2210047
:1075bc001124a0000038a30002003a00809c210096
:1075cc001044a0001b80fb00d1b52800614078005e
:1075dc00e6fc070010c0b300da59020000000000fe
:1075ec00a2fe37000040eb00da5902000000000058
:1075fc009efe3700881f78005470020000000000c7
:10760c000004e000170032003262ab0004003200cc
:10761c003100200040cf2000ae6d020000000000c1
:10762c003242ab00040032003100200070cf200049
:10763c00ae6d0200000000004c7002000000000063
:10764c00000478003222ab000b003200f100200065
:10765c00a0cf2000ae6d0200000000003222a90075
:10766c0005003700f100200090d02000ae6d020024
:10767c00000000000004eb00080078004f047800c4
:10768c000000060040700200000000000000eb004b
:10769c0000000600881f780001022000f0db2000ab
:1076ac00ae6d020000000000689b210018407800bd
:1076bc00f05902000000000000c2b300da590200c9
:1076cc000000000018407800e94f500007003a0015
:1076dc00c0118000645a02000000000000c2b30018
:1076ec00da59020000000000090037000080fb009e
:1076fc000000400081ad280061007800645a02004f
:10770c000000000000c2b300da59020000000000c3
:10771c0028a021009840780063c06000f059020056
:10772c000000000000c2b300da59020000000000a3
:10773c00180078004200de0061406000f059020041
:10774c000000000000c2b300da5902000000000083
:10775c00180078004300de0061406000f059020020
:10776c000000000000c2b300da5902000000000063
:10777c00809c21001080fb004400de006140600012
:10778c00f05902000000000000c2b300da590200f8
:10779c00000000003100200020ae2000ae6d020081
:1077ac00000000004f04780000000600889fbe0017
:1077bc008a9fbe008c1f7800820d02000000000022
:1077cc00b60b02000000000000047800ea0f540021
:1077dc0019003a00820d020000000000b60b0200f6
:1077ec000000000000067800820d0200000000007e
:1077fc00b60b02000000000080047800820d02002d
:10780c0000000000b60b020000000000000578002c
:10781c00820d020000000000b60b02000000000008
:10782c0080057800820d020000000000b60b0200fb
:10783c000000000017003700820d0200000000005d
:10784c00b60b02000000000080047800820d0200dc
:10785c0000000000b60b02000000000000057800dc
:10786c00820d020000000000b60b020000000000b8
:10787c0080057800820d020000000000b60b0200ab
:10788c00000000008800e900e98f500004003e0071
:10789c000006eb00619b21008848e90002003700dc
:1078ac000006eb000004eb008900e900e38f5000b8
:1078bc0007003e0021a021008944e900e3c46400d4
:1078cc00c2cfb3001141610089487100010037003b
:1078dc000004eb008a00e900e18f500009003e0033
:1078ec0021a021000a45e900614565002200200025
:1078fc000255dd00114178000224a1008a48710074
:10790c00010037000004eb008b00e900e18f500010
:10791c0009003e0021a021008b45e900e1c565006e
:10792c0032002000825ddd00114178000234a1009c
:10793c008b487100010037000004eb008000e90067
:10794c00e18f500009003e00819c210061406000e5
:10795c00420020000200dd00114178000244a10029
:10796c00804871000800e00060003a004088210067
:10797c000048eb00d1082000608720000a6e02004e
:10798c00000000008001eb00a2002000110020008c
:10799c0010002000a20d0200000000000040e900d1
:1079ac00619b210080487800e94f50000b003a00a1
:1079bc00c1012000f01421000a6e0200000000003a
:1079cc008001eb00f2ff27001100200020022000b4
:1079dc00a20d020000000000c0118800410520002b
:1079ec0080d12000ae6d0200000000008001eb0091
:1079fc00420020001100200010002000a20d020007
:107a0c000000000028a021000040e9006340600055
:107a1c00c1cfb30098c0600000cc700011022000f0
:107a2c00c0d62000ae6d0200000000008001eb000b
:107a3c00220020001100200010002000a20d0200e6
:107a4c00000000000040e9006140600029002000b7
:107a5c000900dd00984078000124a10000cc7000e2
:107a6c0021032000d0d82000ae6d020000000000e1
:107a7c008001eb00090178001100200010002000ab
:107a8c00a20d0200000000000040e900614060000f
:107a9c00310020000100dd00984078000134a10085
:107aac0000cc7000f1042000e09320000a6e02006c
:107abc00000000008001eb0009017800110020009b
:107acc0010002000a20d020000000000819c21008b
:107adc0061406000420020000200dd00114178008e
:107aec000244a100804871000d003700609b21000a
:107afc0091c0b30090cf100008003a006161b9004a
:107b0c0000902000d1032000860602000000000037
:107b1c0061005000e0805800c0118800ddfe0700b5
:107b2c004f0678004f05be004f04be000000060053
:107b3c00609b210010407800e94f50000e003a0085
:107b4c00c011800013d08000421ade004319de0001
:107b5c0061416100819c21009180fb00c408de0022
:107b6c00e1c0600061426200e3c16100c66f0200c7
:107b7c00000000001000370013d08000421ade0015
:107b8c004319de0061416100819c21009180fb0062
:107b9c00c408de00e1c060000080fb000000400073
:107bac0085ad28006500780061426200e3c1610088
:107bbc00c66f02000000000020a0210010407800d9
:107bcc0063406000e34f500003003a0091c0b300e3
:107bdc00709b210001487800227002000000000018
:107bec00c01180002802e3000400360001022000ce
:107bfc00b01621000a6e0200000000000000060012
:107c0c002c70020000000000000006003222a900c7
:107c1c0020a021001044a000809c21001024a00072
:107c2c00c1012000f0e620000a6e020000000000f6
:107c3c000000060020a021001044a100809c21001f
:107c4c001024a10041012000b0e820000a6e0200bf
:107c5c000000000000000600889fbe008a1f78000c
:107c6c000004eb0029a02100daff2f0029003700c7
:107c7c009940780070c0600023003200e0a7280013
:107c8c00125b0200000000006100200080662000f2
:107c9c00ae6d0200000000003262ab000400320046
:107cac003100200040cf2000ae6d0200000000002b
:107cbc003242ab00040032003100200070cf2000b3
:107ccc00ae6d0200000000004c70020000000000cd
:107cdc00846b0200000000003222ab000600320070
:107cec00f1002000a0cf2000ae6d020000000000cb
:107cfc002023200010086500e0a72800125b02007a
:107d0c0000000000020037004c7002000000000070
:107d1c001800200054700200000000000004e00075
:107d2c00d3ff3a00080078004f0578004f04be00de
:107d3c0000000600b1002000b00a21000a6e02000b
:107d4c0000000000000006001e21ef001021ef00d3
:107d5c0080002000800888000821ef000621ef0039
:107d6c001621ef001421ef00f00888000000060037
:107d7c0011e1a9001fe1a90030348000f001b3002b
:107d8c00303488001e21ef001021ef000621ef0097
:107d9c000821ef00000006000003be00b012200016
:107dac00800f5300e08f5b0007003600c2a928004b
:107dbc00210020005202be00860f5200878f5a000d
:107dcc001400360003003700c41220000500200008
:107ddc00110020008100e900c208dd0080a9280004
:107dec00010040001000be000001520081815a00c9
:107dfc008301d1000281d30002014000838148003d
:107e0c00820f5300838f5b00060036000400be0017
:107e1c00040037008100e800ef8f5000e5ff3a00c6
:107e2c006000b80000000600889fbe008a9fbe005c
:107e3c008c9fbe0080067800cae2a900c8e2a800a8
:107e4c000d00e00004003a00310120002020210048
:107e5c000a6e020000000000cae2ab00090032000a
:107e6c002202ab0007003a000108200000000000cd
:107e7c005216800002806000020032002202ab0029
:107e8c00faff32001b0020006044b8000a082000f2
:107e9c000006eb002202ab0008003200301180001b
:107eac00b3ff0700e1002000502121000a6e020000
:107ebc00000000004f0037008b05e800a2ff070010
:107ecc005116800001006500fdff32001fe1a80083
:107edc0011e1a8005216800002006500fdff3a0077
:107eec0011e1a9001fe1a90030348000f001b300ba
:107efc0030348800fc0888008c088800400880001a
:107f0c008000eb00c000dd00000020003208800083
:107f1c0000004100e0804800e18f5500e6ff320090
:107f2c00e00f5400e08f5c0005003200800f54001d
:107f3c00818f5c00030036000004be000100370096
:107f4c000004be00f88f5500dbff360088ff0700e9
:107f5c000801be0000402200410f200086060200ee
:107f6c00000000000004be000d00e00021003a00fb
:107f7c00009f240021002000800f5400818f5c00a2
:107f8c0005003600f1022000302221000a6e0200aa
:107f9c000000000017003700f10020002025210010
:107fac00ae6d0200000000000800be00aa5a0200dc
:107fbc000000000041002000002721000a6e020092
:107fcc0000000000f100200010262100ae6d020020
:107fdc00000000000800be006fff0700aa5a020054
:107fec000000000041002000002721000a6e020062
:107ffc00000000000800be004f06be004f05be008a
:10800c004f04be0000000600889fbe008a1f780047
:10801c0000047800e20f54004f00320005003e00cf
:10802c000800e00008003200e10f540070003a0034
:10803c000e003700e30f540008003200e40f540028
:10804c006b003a005c003700a1062000f0dd200038
:10805c00ae6d02000000000069003700c062a9008c
:10806c00c082a800c8c2a800c902a900b1002000a3
:10807c0090e420000a6e020000000000d1002000f5
:10808c0040e520000a6e020000000000a06e020015
:10809c00000000000004e000590032003222a90068
:1080ac0009202000faef2f003202ab00050032004d
:1080bc00111180000180640002003a003602f800c1
:1080cc002402f9001c59020000000000e14f50008e
:1080dc0007003a00921180000280640004003a000c
:1080ec00c8590200000000000080fb00a0118800ad
:1080fc003222ab0002003a002222ab000400320014
:10810c00d0ff2f003222b6002222b600c222a900d4
:10811c00e30f5400e4ff3a00101680004400dd0029
:10812c000010b200521680008200650081007000c1
:10813c0051168800501680004300de006800600075
:10814c0071ff2f0012168000828060008100700089
:10815c0011168800d4ff3700e100200010e6200043
:10816c000a6e020000000000f1002000b01821008f
:10817c000a6e0200000000003222a9000820200034
:10818c003202ab00050032001111800001006400c6
:10819c0002003a003602f8002402f9001c590200d1
:1081ac0000000000e14f5000f5ff3a00c8590200f2
:1081bc0000000000120037002c70020000000000cc
:1081cc000000eb0018ff0700227002000000000006
:1081dc00c01180002802e3000900360001022000d3
:1081ec00b01621000a6e02000000000004003700e7
:1081fc0041022000e01d20000a6e02000000000079
:10820c004f0578004f04be0000000600f0a72800c0
:10821c00325b02000000000000000600889fbe00d8
:10822c008a9fbe008c9fbe0022a021009240780045
:10823c000100a100809c21001044a00040412300bb
:10824c0020d0880003ceb30003c960000042eb00cd
:10825c00844178000441780011c0b300c66f02005d
:10826c00000000002270020000000000e7ff070081
:10827c0028a0210089a021007ca021004da8280065
:10828c008b9c210054700200000000000004e000f0
:10829c000a0032009840780070c06000050032007f
:1082ac004c70020000000000da59020000000000cf
:1082bc00020037004c700200000000003222ab00bc
:1082cc00010032003222a9001c59020000000000fb
:1082dc00e14f5000ebff3a00c859020000000000cb
:1082ec00804c78000081fb004411de00024e7800c7
:1082fc00e44f51008700320005003e000204e0000c
:10830c000a003200e14f5100d5003a006a003700f4
:10831c00e64f510085003200d1003900e840510091
:10832c00e1cf5000ce003e009e003700e24f5000df
:10833c001500320005003e000004e0000a00320087
:10834c00e14f500058003a000d003700e74f500045
:10835c001a003200ef4f50003b003200e34f500048
:10836c0051003a00100037002c7002000000000091
:10837c004f06be004f05be004f04be0000000600b5
:10838c00a2ff0700bfff370010c0b300da5902008c
:10839c00000000003222ab00010032003222a900a2
:1083ac001844a000b7ff37001844a10010c0b30058
:1083bc00da59020000000000b2ff370010c0b30011
:1083cc00da590200000000002c70020000000000ce
:1083dc00c8590200000000004800dd0020d08800d1
:1083ec0010c0b300da59020000000000c8590200a6
:1083fc00000000008080fb0020d080000100700095
:10840c0020d0880098017800421ade004319de0063
:10841c00614161009b80fb00c408de00e1c060008c
:10842c0061426200e3c16100c66f020000000000ff
:10843c00227002000000000010c0b300da590200e4
:10844c00000000008fff370010c0b300da590200a3
:10845c00000000003222a900082020003202ab00ec
:10846c0005003200121180000200640002003a0084
:10847c003602f8002402f9001c590200000000002a
:10848c00e14f5000f5ff3a009111800001006400ab
:10849c00f2ff3a00c8590200000000000080fb0007
:1084ac00a0118800edff37000040eb00da59020004
:1084bc000000000073ff37006f406000804ce80044
:1084cc0010c0b300da5902000000000060a02100c7
:1084dc000048eb001904e0006aff32000005780048
:1084ec00c8590200000000000080fb004070020030
:1084fc000000000010c0b300da59020000000000b8
:10850c001a40e800004d7800994f1000f4ff3e002f
:10851c005cff3700de7102000000000010c0b300e9
:10852c00da5902000000000056ff37006f4060006f
:10853c00804c7800ea4f500002003600a0c0b30017
:10854c00804c78001980fb00000040006d00780022
:10855c0020d088002c7002000000000098017800e8
:10856c00421ade004319de00614161009b80fb0072
:10857c00c408de00e1c0600061426200e3c161003a
:10858c0020d08000c66f02000000000022700200a4
:10859c000000000010c0b300da5902000000000017
:1085ac0038ff370001cfb30018cc60001b44a1008a
:1085bc000080fb000038a3000400320098407800d3
:1085cc000100a1000114a000014c78000028a300b8
:1085dc000600320018417800e34061000104a0005d
:1085ec00c2cfb30018416100014c71000018a30008
:1085fc00010032001824a0000008a3000100320082
:10860c001834a0000048a30001003a001b44a0004d
:10861c002c7002000000000098017800421ade0065
:10862c004319de00614161009b80fb00c408de0041
:10863c00e1c0600061426200e3c1610020d08000b3
:10864c00c66f020000000000227002000000000053
:10865c0010c0b300da5902000000000009ff370017
:10866c000040eb00da5902000000000005ff370063
:10867c0000ba2800325b0200000000000000060077
:10868c00889fbe00004478008044eb006140640089
:10869c00c0640200000000000884fb000804d10044
:1086ac008944e800e6cf5400f8ff3a006065020008
:1086bc0000000000da5902000000000060650200b2
:1086cc0000000000da590200000000004f04be0058
:1086dc0000000600889fbe008a9fbe008c1f780099
:1086ec000044780081457800024678000ac8b3003f
:1086fc000a4564008044eb0061406400c0640200e1
:10870c00000000000884fb000804d1008944e80044
:10871c00e6cf5400f8ff3a000a04e00006003a00e5
:10872c000b80fb00de640200000000000c80fb00ec
:10873c00de640200000000004f0678004f05be000a
:10874c004f04be0000000600889fbe008a9fbe003a
:10875c00804478000044eb00084578001bc0b3004f
:10876c000908a300040032000b407800c06402002a
:10877c0000000000030037000a407800c0640200cb
:10878c00000000000844e800e44f540003003200ed
:10879c008984fb008904d100f1ff37006065020079
:1087ac00000000006065020000000000da590200c1
:1087bc00000000004f05be004f04be000000060084
:1087cc00889fbe008a9fbe008c9fbe008e1f7800c3
:1087dc008044780081467800024778000986fb00c7
:1087ec004666de000044eb001ac0b30088457800f2
:1087fc000e003700e34f54000c003a000c04e0006c
:10880c000a00320010c0b300a8640200000000008f
:10881c000c80fb003e6c0200000000000040eb00ee
:10882c00a8640200000000000e0037000908a30035
:10883c00040032000a407800c0640200000000000e
:10884c00030037000b407800c064020000000000f9
:10885c008984fb008904d1000844e800e44f5400eb
:10886c00e4ff3a000d80fb00de6402000000000013
:10887c000e80fb00de640200000000004f07780051
:10888c004f06be004f05be004f04be0000000600a0
:10889c000040eb00c0640200000000000040eb0050
:1088ac00c0640200000000000040eb00c064020045
:1088bc00000000000040eb00c0640200000000005b
:1088cc000000eb00de640200000000000000eb0082
:1088dc00de640200000000000000eb00de64020019
:1088ec000000000000000600889fbe000004780015
:1088fc00814478000040eb00c064020000000000de
:10890c000040eb00c0640200000000000040eb00df
:10891c00c0640200000000000040eb00c0640200d4
:10892c00000000001880fb00de6402000000000064
:10893c00184090000080fb00de6402000000000084
:10894c00284090000080fb00de6402000000000064
:10895c006fc4640003003200cdff07000844e90037
:10896c00fdff3a004f04be0000000600889fbe00c9
:10897c008a1f78000004be00024578000040eb001e
:10898c00c0640200000000000040eb00c064020064
:10899c00000000000040eb00c0640200000000007a
:1089ac000040eb00c06402000000000008007800ea
:1089bc00686c020000000000de6402000000000091
:1089cc004849dd004840de0000007100c848de0068
:1089dc00686c020000000000de6402000000000071
:1089ec004048de0001002000686c0200000000001e
:1089fc00de64020000000000ef4465000500320058
:108a0c000044eb00a2ff07000844e80088cf5400a4
:108a1c00fcff3e004f0578004f04be00000006002e
:108a2c00881f780010c0b300c06402000000000072
:108a3c000040eb00c0640200000000000040eb00ae
:108a4c00c0640200000000000040eb00c0640200a3
:108a5c00000000000000eb00de64020000000000db
:108a6c0060650200000000000004780060650200f0
:108a7c0000000000da5902000000000008407800f5
:108a8c00da5902000000000081ff070080ff070098
:108a9c004f04780000000600889fbe008a9fbe002d
:108aac008c9fbe008e1f7800819c210011407800a5
:108abc000040a0000034a1008048780018c0b3002a
:108acc00728050000848780081c0b3000000e800b4
:108adc000148780020c0b300819d210080487800b7
:108aec0080c0eb006263020000000000c922a900f4
:108afc00c902a900c8e2a800084078009c640200e2
:108b0c0000000000dafe0700cd9d2100bc9d210075
:108b1c008e9c2100c859020000000000804e780095
:108b2c000081fb004411de00024e7800e34f51003f
:108b3c00c800320004003e00e14f510089003200b1
:108b4c00bb003e000b003700e64f510078023200ac
:108b5c0003003e00e44f5100a1023a006e023700c0
:108b6c00e84f510081023200ea4f51009c023a005a
:108b7c00d80037000080fb008000eb00ed0f5000a8
:108b8c00e08f580073003e0000600100980237002f
:108b9c000c0037000d0037001200370017003700ab
:108bac001d003700230037003d003700410037001f
:108bbc00450037004b003700510037005700370095
:108bcc005d003700aafe0700d2ff37003e640200aa
:108bdc000000000010c0b300da59020000000000d1
:108bec00ccff3700226402000000000010c0b3006c
:108bfc00da59020000000000c6ff37000040eb000d
:108c0c009c6402000000000010c0b300da5902009e
:108c1c0000000000bfff370010c0b3009c640200ce
:108c2c000000000010c0b300da5902000000000080
:108c3c00b8ff370021c0b300809d210090cf1000f9
:108c4c0005003a006065020000000000a19d2100b3
:108c5c008048780005003700f00f2000a465020062
:108c6c0000000000a19d2100804878001e41780082
:108c7c006840610005003200a89d21001880fb00af
:108c8c00686c020000000000004c7800a09d2100e0
:108c9c0010407800da590200000000009dff3700f8
:108cac003e65020000000000da59020000000000de
:108cbc0098ff37003865020000000000da59020006
:108ccc000000000093ff370010c0b300fa630200ed
:108cdc000000000010c0b300da59020000000000d0
:108cec008cff37000040eb00a8640200000000007d
:108cfc0010c0b300da5902000000000085ff3700f5
:108d0c0010c0b300a86402000000000010c0b30043
:108d1c00da590200000000007eff37000040eb0033
:108d2c00b46402000000000010c0b300da59020065
:108d3c000000000077ff370010c0b300b4640200dd
:108d4c000000000010c0b300da590200000000005f
:108d5c0070ff37000040eb00da5902000000000001
:108d6c006cff37006f406000804ee80010c0b3000d
:108d7c00da59020000000000a09d21000048eb0021
:108d8c001d04e00063ff3200989d2100000578006f
:108d9c00c859020000000000004c78009e41780089
:108dac00e8c06100040032000080fb00686c020027
:108dbc0000000000004c780021c0b300809d210011
:108dcc0090cf100007003a001880fb00de64020010
:108ddc000000000010c0b300da59020000000000cf
:108dec000e0037001880fb00a46502000000000094
:108dfc00004c78009e417800e8c06100040032000d
:108e0c000080fb00686c020000000000004c780041
:108e1c0018407800da590200000000001a40e800ff
:108e2c00004d78009d4f1000d9ff3e0039ff3700f0
:108e3c006f4060000040e800804e7800fa6302004a
:108e4c000000000010c0b300da590200000000005e
:108e5c0030ff37006f406000804ee80010c0b30058
:108e6c00da59020000000000c8590200000000009e
:108e7c00004e7800a09d21000048eb001d04e0008e
:108e8c0010003200000478001c04e00004003d00d7
:108e9c0010c0b300c06402000000000003003700e3
:108eac000040eb00c0640200000000001c40780091
:108ebc00004e40001840e800004c78009d4f100018
:108ecc00f1ff3e0010c0b300da59020000000000b0
:108edc0010ff370041cab300814f5000140032001c
:108eec0004003e00e4c05000814f500086013a005f
:108efc000700370051cab300814f50009b0032006d
:108f0c0081c0e800814f50007f013a00f10037002a
:108f1c00c85902000000000061a2210080487800be
:108f2c0010c0b300da59020000000000f9fe37004f
:108f3c0060a2210010407800e14f50000300320085
:108f4c00e24f500085003a002d003700c85902004e
:108f5c00000000000080fb006300b900b0ce880068
:108f6c000001eb0082ce8800e00f5000e08f58002b
:108f7c000c0032000004eb00e99d210019044400b0
:108f8c00c859020000000000004c780088ce800018
:108f9c000804e80088ce8800b0ce8000880f50000e
:108fac00f6ff3e000000eb0080ce8800b0ce8000c3
:108fbc000000e0000e0032000000eb00e89d2100f4
:108fcc0098017800808041002141900091409000f0
:108fdc0063407800fafd070080ce800063004000fb
:108fec0080ce8800b1ce8000808f5000f4ff3e0010
:108ffc0010c0b300da59020000000000c5fe3700b3
:10900c00c8590200000000000080fb004200dd0097
:10901c00b0ce88008000eb0081ce88000c003200be
:10902c000004eb00e99d210019044400c85902001a
:10903c0000000000004c780088ce80000804e80096
:10904c0088ce8800b0ce8000880f5000f6ff3e001e
:10905c000000eb0080ce8800b0ce80000000e00065
:10906c003a003200e99d2100a89d21000040eb0050
:10907c00c0640200000000000040eb00c06402006d
:10908c00000000000040eb00c06402000000000083
:10909c000040eb00c06402000000000080ce8000a5
:1090ac00f1ce8000614078000080fb00de6402009d
:1090bc000000000080ce8000f1ce800000804000d7
:1090cc00104090000080fb00de64020000000000f5
:1090dc0080ce8000f1ce80000080400020409000c7
:1090ec000080fb00de6402000000000081ce8000e6
:1090fc006380400019014000924178006fc9610003
:10910c00004ceb00f2ce8000624078000004e000de
:10911c0009003200defd07001840e800004c780022
:10912c0081ce8000f2ce80000101410032419000de
:10913c00804f5100f7ff3e00e480400081ce880054
:10914c00b0ce8000810f5000c8ff3e0010c0b300ad
:10915c00da590200000000006efe37000040eb0000
:10916c00da590200000000006afe370060a22100fc
:10917c0010407800e14f500003003200e24f5000e5
:10918c0064fe3a0030003700c859020000000000ad
:10919c000080fb00b0ce8800c8590200000000001f
:1091ac00004e78000000eb0080ce8800b0ce80002e
:1091bc000000e00057fe3200989d2100aa9d21007e
:1091cc008044eb00894578001c4c78000b4d7800ee
:1091dc001880fb000008a3000400320010c0b3008c
:1091ec00c064020000000000030037000940780052
:1091fc00c0640200000000001880fb000000d100d9
:10920c00004c78001a40e800004d7800e34f500005
:10921c00efff360060650200000000006065020090
:10922c0000000000da5902000000000080ce80002f
:10923c000000e80080ce8800b1ce8000808f500006
:10924c00e1ff3e0033fe3700c85902000000000069
:10925c000080fb00b0ce88008000eb0081ce88003f
:10926c002cfe320068b92000a90b20006abb2d002f
:10927c00ab0b200022c0b3000800be00bbfd0700f2
:10928c00e7fd070022c0b3000a00be00b7fd0700cf
:10929c0022c0b300603d2d00a10b2000b3fd0700e0
:1092ac00dffd070022c0b30060bb2000a10b200033
:1092bc00aefd0700dafd070080ce80000000e8005c
:1092cc0080ce8800b1ce8000808f5000e9ff3e0038
:1092dc0010fe3700c8590200000000000080fb009f
:1092ec00a0ce8800c8590200000000008080fb005e
:1092fc0091ce880060a2210010407800e24f50000f
:10930c0005003a00a2ce80006511b90082804000b1
:10931c00b1ce880014003700e14f500006003a002f
:10932c00a0ce800000004000808040008180400082
:10933c00b1ce88000c003700e34f500006003a0015
:10934c00a0ce800000004000808040008180400062
:10935c00b1ce8800040037000040eb00da5902005f
:10936c0000000000ebfd37000000eb0080ce880011
:10937c00b0ce80000000e0000c0032000004eb00d6
:10938c00e99d210019044400c859020000000000a6
:10939c00004c780088ce80000804e80088ce880055
:1093ac00b0ce8000880f5000f6ff3e0090ce8000bb
:1093bc000000e0000300320010c0b300da590200d4
:1093cc00000000000000eb0080ce8800e89d21002a
:1093dc0069a221004100370018007800e0407900b4
:1093ec00e1cf500022003a0099407800e3cf5000c2
:1093fc0009003a000200400030419000a04090006b
:10940c0010409000b3fc070080ce80006400400048
:10941c0080ce880031003700e1cf500009003a00bf
:10942c000200400030419000a0409000104090009d
:10943c00e3fc070080ce80006400400080ce8800f2
:10944c0026003700e2cf500024003a008200400092
:10945c00c14090000201e8000200400022fd07001c
:10946c0080ce80006500400080ce88001b00370055
:10947c00e2cf500019003a0099407800e3cf500039
:10948c0007003a0002004000104090007cfc0700ee
:10949c0080ce80000080e80080ce88000f0037006e
:1094ac00e1cf500007003a0002004000104090004d
:1094bc00a5fc070080ce80000080e80080ce8800ec
:1094cc0006003700e2cf500004003a0054fd0700bc
:1094dc0080ce80000000e80080ce880082ce800024
:1094ec00b0ce8000800f5100bbff390090ce8000c1
:1094fc000000e00087fd3a0010c0b300da5902000a
:10950c000000000083fd37000040eb00da59020038
:10951c00000000007ffd3700de710200000000003b
:10952c0010c0b300da5902000000000079fd3700ca
:10953c00e3406000814e7800609b21000148780078
:10954c00829d21001240780062630200000000003e
:10955c0010c0b3009c6402000000000010c0b300f7
:10956c00da590200000000006afd37001e44a10019
:10957c000080fb000038a30001003a001e44a0004c
:10958c0021c0b300839d2100814978000028a300ed
:10959c000200320031c0b300814978001e34a100b2
:1095ac000018a300010032001e34a000609b2100b3
:1095bc0090407800829d2100124078006263020086
:1095cc000000000010c0b3009c640200000000000a
:1095dc0010c0b300da590200000000004dfd370046
:1095ec000040eb00da5902000000000049fd370092
:1095fc004f0778004f06be004f05be004f04be005b
:10960c0000000600e30f500004003e0010a1a8006b
:10961c001081a800e003200010003700fe0f50005e
:10962c0004003e0010a1a8001081a900a00f20008a
:10963c000a003700410f2000810f500004003e004b
:10964c0010a1a9001081a800007d200003003700a4
:10965c0010a1a9001081a90000e823000000060059
:10966c001021ef001e21ef009c21ef0080cc800028
:10967c000000e00005003a0000fe2f00ca26b600ec
:10968c000000eb00a0cc880017003700ddff0700be
:10969c0082cc8000110009000280d8000000e90093
:1096ac006008880092cc80000282b900420620003b
:1096bc00110009000282d80001fe2f0052368000f2
:1096cc00828060006101b30051368800d00c8800a4
:1096dc00c00c880060002000e00c880011e1a8009c
:1096ec0020002000a0cc880000000600889fbe004f
:1096fc008a9fbe008c1f78001021ef001e21ef0006
:10970c009c21ef00a0cc8000e20f50000f003a002b
:10971c0000fe2f00ca26b600c1002000e02b20005e
:10972c000a6e0200000000000000eb00a0cc8800d4
:10973c0010c480000000e800f007b2000180210096
:10974c00614078000004e0007100320010c4800019
:10975c000000e800f007b20010c48800820d02007f
:10976c0000000000b60b020000000000800578002d
:10977c00820d020000000000b60b02000000000089
:10978c00cf80de0010050200000000000004be00c7
:10979c008b00e9001a002000e0f92000808f5000b7
:1097ac00010036000005eb006011b8000800be0097
:1097bc0094040200000000000000e00008003400e7
:1097cc0002002000832c24000800be00900402003c
:1097dc00000000000000e00001003d000a05e80068
:1097ec00e20f550025003200408821000048eb00b4
:1097fc0011012000a02c20000a6e020000000000c5
:10980c0011012000b02d2000ae6d02000000000000
:10981c008001eb0002fa2000110020002003200040
:10982c00a20d02000000000000047800080078007f
:10983c0074ff0700110009000880d8000006e90039
:10984c0001012000902f2000ae6d020000000000ee
:10985c008001eb00320620008000eb00200320008a
:10986c00a20d020000000000cf80de0010050200f7
:10987c00000000000004be00050037000b0078005b
:10988c0060ff0700110009000b80d8000006e900fa
:10989c006160b80074050200000000000005be0005
:1098ac0002002000832c24000800be000c040200df
:1098bc00000000000001be000a00be001e060200ef
:1098cc0000000000da0402000000000002fe2f007d
:1098dc0053368000030161006201b30052368800e8
:1098ec00d00c8800c00c880060002000e00c8800c0
:1098fc006c08880011e1a800a10020009030200025
:10990c000a6e02000000000020002000a0cc88009d
:10991c004f0678004f05be004f04be000000060045
:10992c000080eb0070088800600888000821ef00b8
:10993c000621ef001621ef001421ef00800020001b
:10994c00f0088800400f2000e0088800004022004a
:10995c00d00888008780a9001fe1a80011e1a800a9
:10996c00010021003204800002806000fdff320003
:10997c0011e1a9001fe1a90031088000a1cd8800e8
:10998c00420880008001eb00c011dd0002002000c5
:10999c0002804000e080490080cd880091cd880095
:1099ac00000006001e21ef001021ef00c942a800a4
:1099bc0000fe2f008606b600a000b30030348800ed
:1099cc00a003200080088800d5ff07000001be001e
:1099dc00f00f2000800f5100e08f59000500360079
:1099ec00481add00c812de00850272004812dd0044
:1099fc0004003700a000200080088800c8ff070082
:109a0c000002be0031348000f101b3003134880013
:109a1c001e21ef001021ef000400be000000060024
:109a2c00889fbe008a9fbe008c9fbe0000017800fc
:109a3c0084a0a9008420a900f10f2e0070348000ae
:109a4c008080600000a0200001007000703488004d
:109a5c0000fe2f008e06b600a000b3007034880004
:109a6c000821ef000621ef0080002000800888000c
:109a7c0011e1a80030002000300a880030082000d6
:109a8c00100a88004261ab0006003200000a800018
:109a9c008000eb004261ab00fcff3a0050cd880027
:109aac0061cd88004661ab0003003200200a8000c3
:109abc004661ab00fdff3a004261ab00feff320095
:109acc00000a80008000eb0030cd880041cd88007a
:109adc00200a80008000eb00f0cc880001cd8800cb
:109aec006000b800b0cc8800c1cc88000000eb004e
:109afc0070cd88000200e000290032003ccd8000cf
:109b0c004dcd8000facc80000bcd80006044b800b5
:109b1c008000eb00020037000405be000606be0004
:109b2c004261ab00feff3200060a80008003eb00ae
:109b3c00240a80008002eb000c0653008d865b002b
:109b4c000a0552008b855a00c055dd000a00200022
:109b5c000c0545008d854d000804450089844d0099
:109b6c008100e800810f5100ebff3e0056cd8800cc
:109b7c0067cd880036cd880047cd880014cd88008d
:109b8c0025cd8800f4cc880005cd8800dacc88007f
:109b9c00ebcc8800b8cc8800c9cc880072cd88008a
:109bac004221ef004221ef0011e1a9008001eb00fe
:109bbc00b0cc8000c1cc8000860602000000000002
:109bcc004f06be004f05be004f04be00000006004d
:109bdc00889fbe008a9fbe00a0cc8000e20f500080
:109bec0005003a00f1012000303120000a6e02001d
:109bfc000000000083013700f1002000203320001a
:109c0c00ae6d0200000000001e21ef001021ef00dd
:109c1c00c942a80000fe2f008606b600a000b300c3
:109c2c0030348800a0032000800888003cff070027
:109c3c000004be006055b800f2ff2300820f5000f4
:109c4c00e08f58000b003600c85ddd004850de0088
:109c5c008b0570004855dd004848de000a05700091
:109c6c00c84cdd004840de00890470004844dd002b
:109c7c0009003700b1002000a0132100ae6d0200d6
:109c8c0000000000a00020008008880024ff0700ce
:109c9c000004be006055b800f0f92000010020005f
:109cac006011b8000040e10001c8e10002d0e10001
:109cbc0003d8e100070036000800be004a5b020032
:109ccc0000000000c0b12800125b02000000000080
:109cdc0047013700e00f5400e08f5c00e00f5d009f
:109cec00e08f5d003f013200b1002000a013210085
:109cfc00ae6d0200000000000800780048ff07006d
:109d0c006011b80004a82100650020006033b80081
:109d1c000400e1000588e1000690e1000798e100ed
:109d2c004e00360016050200000000000001be00c7
:109d3c00703b2400a13b25000c0402000000000035
:109d4c0098040200000000000205be000004be00e2
:109d5c00046a2800150020006033b800de070200fa
:109d6c00000000004a5b020000000000e0c2b300eb
:109d7c00da59020000000000046a280015002000d7
:109d8c006033b8000800be000a01be00ec070200f8
:109d9c00000000000205be000004be00f0702200ae
:109dac00010020006011b8000040e10001c8e10092
:109dbc0002d0e10003d8e10003003e0000c3b30071
:109dcc00da59020000000000703e20000100200063
:109ddc006011b8000040e10001c8e10002d0e100d0
:109dec0003d8e10003003e0000c3b300da590200bf
:109dfc000000000030062000010020006011b800b7
:109e0c000040e10001c8e10002d0e10003d8e1000c
:109e1c0003003e0000c3b300da590200000000004a
:109e2c0090002000010020006011b8000040e1000b
:109e3c0001c8e10002d0e10003d8e10003003e00bc
:109e4c0000c3b300da590200000000000800be0095
:109e5c00aa5a020000000000de003700b4e12e0018
:109e6c00150020006033b8000400e1000588e10013
:109e7c000690e1000798e100430036001605020049
:109e8c00000000000001be00902f20005121250091
:109e9c000c04020000000000980402000000000006
:109eac000205be000004be00047122000500200063
:109ebc006033b800de070200000000004a5b0200bd
:109ecc0000000000e0c2b300da59020000000000fc
:109edc0004712200050020006033b8000800be00a9
:109eec000a01be00ec070200000000000205be00e3
:109efc000004be00703e2000010020006011b8007c
:109f0c000040e10001c8e10002d0e10003d8e1000b
:109f1c0003003e0000c3b300da5902000000000049
:109f2c0030062000010020006011b8000040e10064
:109f3c0001c8e10002d0e10003d8e10003003e00bb
:109f4c0000c3b300da5902000000000090002000aa
:109f5c00010020006011b8000040e10001c8e100e0
:109f6c0002d0e10003d8e10003003e0000c3b300bf
:109f7c00da5902000000000008007800645a020060
:109f8c00000000009300370004c4290005002000e5
:109f9c006033b8000400e1000588e1000690e100a0
:109fac000798e1003800360016050200000000009a
:109fbc000001be0080b22600e10625000c04020060
:109fcc000000000098040200000000000205be0022
:109fdc000004be00843e2000050020006033b80061
:109fec00de070200000000004a5b020000000000d7
:109ffc00e0c2b300da59020000000000843e2000e9
:10a00c00050020006033b8000800be000a01be0045
:10a01c00ec070200000000000205be000004be00b8
:10a02c0030062000010020006011b8000040e10063
:10a03c0001c8e10002d0e10003d8e10003003e00ba
:10a04c0000c3b300da5902000000000090002000a9
:10a05c00010020006011b8000040e10001c8e100df
:10a06c0002d0e10003d8e10003003e0000c3b300be
:10a07c00da5902000000000008007800645a02005f
:10a08c000000000053003700941623000500200048
:10a09c006033b8000400e1000588e1000690e1009f
:10a0ac000798e1002d0036001605020000000000a4
:10a0bc000001be0000c22b00e1eb24000c040200e6
:10a0cc000000000098040200000000000205be0021
:10a0dc000004be0044062000050020006033b800d8
:10a0ec00de070200000000004a5b020000000000d6
:10a0fc00e0c2b300da590200000000004406200060
:10a10c00050020006033b8000800be000a01be0044
:10a11c00ec070200000000000205be000004be00b7
:10a12c0090002000010020006011b8000040e10008
:10a13c0001c8e10002d0e10003d8e10003003e00b9
:10a14c0000c3b300da590200000000000840780098
:10a15c00f0590200000000001e0037001605020036
:10a16c00000000000001be000068290081d124001d
:10a17c000c04020000000000980402000000000023
:10a18c000205be000004be00a40020000500200053
:10a19c006033b800de070200000000004a5b0200da
:10a1ac0000000000e0c2b300da5902000000000019
:10a1bc00a4002000050020006033b8000800be0099
:10a1cc000a01be00ec07020000000000f05902007a
:10a1dc0000000000c0b12800125b0200000000006b
:10a1ec000300370000b22800125b020000000000e0
:10a1fc0030348000f001b300303488001e21ef00b1
:10a20c001021ef004f05be004f04be0000000600f9
:10a21c00809c2100104078006340600002003a00ee
:10a22c00c942a80001003700c8c2a800e100200004
:10a23c0010342000ae6d020000000000000006008b
:10a24c00809c2100104078006340600003003a00bd
:10a25c00c942a900cb42a80002003700c8c2a9001d
:10a26c00cac2a80081002000f03420000a6e02004f
:10a27c000000000000000600809c210010407800c7
:10a28c006340600003003a00c942a900cb42a90018
:10a29c0002003700c8c2a900cac2a9007100200080
:10a2ac00703520000a6e020000000000000006005d
:10a2bc00809c2100104078006340600007003a0049
:10a2cc00c942a800000000000000000050168000e9
:10a2dc004a00de006140600006003700c8c2a800da
:10a2ec000000000000000000501680004600de0058
:10a2fc00614060000080fb0000000600889fbe00eb
:10a30c008a9fbe008c1f78001021ef001e21ef00e9
:10a31c009c21ef00a0cc8000e20f500010003a000e
:10a32c0010c480000000e800f007b200018021009a
:10a33c00614078000004e00009003a0000fe2f00a4
:10a34c00ca26b600c1002000e02b20000a6e0200d5
:10a35c00000000000000eb00a0cc88005e0037007d
:10a36c0010c480000000e800f007b20010c48800a0
:10a37c00820d020000000000b60b0200000000007d
:10a38c00418821001104e0000b003a00cf80de0070
:10a39c0010050200000000000004be0002002000b6
:10a3ac004333240094040200000000000045eb003d
:10a3bc000000e00011003400408821000048eb0050
:10a3cc0031012000301e21000a6e02000000000046
:10a3dc008001eb00420b20008000eb00a005200068
:10a3ec00a20d020000000000cf80de00100502006c
:10a3fc00000000000004be001ac0b3000bfe2f00ca
:10a40c002c4e200010a1a8001081a80002002c00e6
:10a41c00a35524000800be000c040200000000003c
:10a42c0002002400c34924001e06020000000000a4
:10a43c0002002000832724005203020000000000c9
:10a44c00da0402000000000053368000038165002e
:10a45c006201b30052368800d00c8800c00c880012
:10a46c0060002000e00c88006c08880011e1a80056
:10a47c00c1002000601f21000a6e020000000000d5
:10a48c0020002000a0cc8800e14f550012003a00bb
:10a49c0013002000420b20008000eb000080eb003a
:10a4ac00a20d020000000000cf80de0010050200ab
:10a4bc00000000000004be006011b800900402000f
:10a4cc00000000000000e000ceff3d0050b428006a
:10a4dc00125b0200000000004f0678004f05be0022
:10a4ec004f04be0000000600e0a1210010407800df
:10a4fc000018a300110032000008a30003003a006a
:10a50c000040eb00c06402000000000000c2b30079
:10a51c00da59020000000000310020003041200018
:10a52c00ae6d02000000000000c2b300da59020058
:10a53c0000000000e0a121001014a100e0a1210006
:10a54c0010407800e14060000040eb0002003a004f
:10a55c006065020000000000e1a121001114a000c0
:10a56c000080fb0000000600881f780000047800c3
:10a57c00e0a121001040780062406000120032001f
:10a58c0000c2b300da5902000000000031002000c4
:10a59c0030412000ae6d02000000000000c2b3008c
:10a5ac00da59020000000000e0a121001040780000
:10a5bc006140600002003a00c0640200000000002c
:10a5cc00e0a121001014a100e0a1210010407800ae
:10a5dc006140600006003a0008007800de6402006a
:10a5ec00000000003e650200000000000084fb003b
:10a5fc0000c2b300da590200000000000800e000bd
:10a60c0006003a003100200030412000ae6d0200ff
:10a61c000000000000302000050037004100200041
:10a62c0060412000ae6d0200000000000010200010
:10a63c004f04780000000600e0a1210010407800d3
:10a64c006240600010003200410020006041200098
:10a65c00ae6d02000000000040b82800125b020042
:10a66c0000000000e0a12100104078006140600073
:10a67c0003003a0010c0b300c064020000000000e8
:10a68c00e0a121001014a100e0a1210010407800ed
:10a69c00614060000f003a003e64020000000000c0
:10a6ac000000e0000b00320091002000c0202000d0
:10a6bc00ae6d02000000000051012000502120006e
:10a6cc00ae6d02000000000040b82800125b0200d2
:10a6dc0000000000d1002000a04120000a6e020002
:10a6ec000000000000000600e0a1210010407800ee
:10a6fc0062406000100032004100200060412000e8
:10a70c00ae6d02000000000040b82800125b020091
:10a71c0000000000e0a121001040780061406000c2
:10a72c0003003a0010c0b300c06402000000000037
:10a73c00e0a121001014a100e0a12100104078003c
:10a74c006140600002003a00226402000000000038
:10a75c00c1002000704220000a6e020000000000c0
:10a76c000000060001012000404f2000ae6d0200e9
:10a77c00000000000040eb00f05902000000000057
:10a78c0000c2b300da59020000000000609b2100f7
:10a79c0010407800f05902000000000000c2b30025
:10a7ac00da5902000000000050b82800125b0200c9
:10a7bc000000000000000600e0a121001004a10030
:10a7cc00820d020000000000b60b02000000000029
:10a7dc008000e900e38f500004003e00619b2100e3
:10a7ec008048e9000000e00011003a004088210098
:10a7fc000048eb00e0a121001004a100b1032000ef
:10a80c00804520000a6e0200000000008001eb0071
:10a81c00420020001100200010002000a20d0200b8
:10a82c0000000000619b21008048e9000b0037000c
:10a83c0041cf800030002300808f500004003e0088
:10a84c005103200030492000ae6d020000000000d2
:10a85c00c4ff0700e0a121001014a100809c21007e
:10a86c001044a00000000600e0a121001040780078
:10a87c006140600009003a00c922a800c902a80082
:10a88c00cb02a900cb22a900609b2100904078004c
:10a89c0020c0b3006263020000000000000006004c
:10a8ac00e1a12100114078000010a100804878003f
:10a8bc000008a3000100320007e2a9000000060016
:10a8cc00b1002000600b21000a6e020000000000a5
:10a8dc0000000600e4874700889fbe008a9fbe00e8
:10a8ec008c9fbe008e1f7800804678002259020093
:10a8fc0000000000c922a800c902a800cb02a900d0
:10a90c00cb22a90062a0a80062c0a8008660a900a2
:10a91c005b168000c95dde0059168000c84cde0055
:10a92c00e1c46400e1c565000040eb0080f79f00c6
:10a93c00004778000e4678000e00370088447800f7
:10a94c008a4578000b003700884478008a457800e7
:10a95c0008003700884478008a45780005003700e5
:10a96c00884478008a4578000200370088447800d3
:10a97c008a4578008660ab000d003a003059020021
:10a98c00000000001c590200000000000004e00060
:10a99c00f8ff3200c85902000000000062a0a900b4
:10a9ac0062c0a9000d04e0005500320051003700d0
:10a9bc008660a9005a1680004955de006145650085
:10a9cc00581680004844de00614464000c04e0002a
:10a9dc002e0032000904e0002e003a000804e000ca
:10a9ec00d6ff3200e74f57000b003e008ff0970068
:10a9fc0081c0400081f79f000a04e0000200320091
:10aa0c000104a00081f79f000e47e80088447800fd
:10aa1c008a457800d7ff37000d04e00005003200ae
:10aa2c008ff097000180fb00a85902000000000085
:10aa3c0006003700c0c5b3008459020000000000b6
:10aa4c000ff0970084590200000000000a04e00097
:10aa5c0007003200d0c2b30084590200000000008d
:10aa6c00884478008a4578000047eb00c1ff370026
:10aa7c00b0c2b30084590200000000008844780082
:10aa8c000047eb008e457800baff37000904e00060
:10aa9c00adff32000804e000aeff32000b04e00012
:10aaac000a0032000a04e000adff3a00b0c5b30062
:10aabc008459020000000000884478000047eb0035
:10aacc001cc0b3008e457800aaff37000a04e000d2
:10aadc00a6ff3200d0c5b30084590200000000006c
:10aaec00884478008a4578000047eb000e467800d1
:10aafc00a0ff370040b82800125b020000000000e5
:10ab0c004f0778004f06be004f05be004f04be0035
:10ab1c004f00b10000000600889fbe008a9fbe0057
:10ab2c0000057800e10f55000900320003003900e0
:10ab3c00e20f55006a003a0059003700510320001b
:10ab4c0040502000ae6d020000000000680037008d
:10ab5c008040eb0000302000d263020000000000b7
:10ab6c00e1022000905320000a6e02000000000059
:10ab7c00cb02ab00030032000004eb00cb22ab0095
:10ab8c000c003a0091002000c0202000ae6d0200a5
:10ab9c00000000005101200050212000ae6d020089
:10abac000000000040b82800125b0200000000000a
:10abbc004f003700e9a121000b10200099407800cc
:10abcc0061c0600008003a003e6402000000000012
:10abdc0008007800de640200000000003e65020000
:10abec00000000000085fb000a00e00020003a0095
:10abfc0008007800846b02000000000080c2b300e3
:10ac0c00da590200000000000880d100846b0200b9
:10ac1c00000000000808a30004003a0070b82800e7
:10ac2c00325b0200000000000b00370099407800f6
:10ac3c0061c0600005003a00606502000000000081
:10ac4c0010c0b300c064020000000000a0b82800cf
:10ac5c00325b02000000000050b82800325b02009a
:10ac6c000000000000c2b300da590200000000002e
:10ac7c009940780061c0600002003a002264020032
:10ac8c00000000000804e8008b0f5400cbff3a00d2
:10ac9c0040b82800125b02000000000014003700ce
:10acac00e0a12100104078006140600001003200fa
:10acbc0007e2a90071002000705620000a6e020005
:10accc0000000000f1002000b01821000a6e020004
:10acdc000000000010c0b300fefe070004003700a7
:10acec0041022000e01d20000a6e0200000000005e
:10acfc004f05be004f04be0000000600d0b828006f
:10ad0c00325b02000000000000000600889fbe00bd
:10ad1c008a9fbe008c9fbe008e1f7800c922a8009f
:10ad2c00c902a800cb02a900cb22a900c8c2a90065
:10ad3c00819c2100114078000040a0000034a1004b
:10ad4c008048780080c0eb0020c0b3006263020032
:10ad5c0000000000e9ff070019a221000aa221004f
:10ad6c00ed9d2100c859020000000000804c7800c5
:10ad7c000081fb004411de00024d7800e14f5100d0
:10ad8c00d200320005003900e44f5100f0003200cf
:10ad9c00e64f5100f4003a00e40037000080fb005d
:10adac008000eb00ef0f5000e08f5800c3003e0016
:10adbc0000600100f90037000e0037000f0037006b
:10adcc001400370019003700bc0037001c00370096
:10addc0022003700280037007b003700b70037000f
:10adec00b6003700b5003700b4003700b3003700a9
:10adfc00ac003700c1ff0700daff37003e640200e9
:10ae0c000000000010c0b300da590200000000007e
:10ae1c00d4ff3700226402000000000010c0b30011
:10ae2c00da59020000000000ceff37006065020016
:10ae3c0000000000da59020000000000c9ff3700d2
:10ae4c000040eb00c06402000000000010c0b30022
:10ae5c00da59020000000000c2ff370010c0b30036
:10ae6c00c06402000000000010c0b300da590200f8
:10ae7c0000000000bbff3700c859020000000000b2
:10ae8c004804dd00c8590200000000008085fb006a
:10ae9c0088857500c8590200000000000044780045
:10aeac00c85902000000000001002100818f5500ec
:10aebc0009003e004847dd000080fb000e077000d3
:10aecc00810f570004003e000004eb000b00e00073
:10aedc0005003a00a80037000040eb00da590200e8
:10aeec00000000009fff37001d064400c8590200f7
:10aefc0000000000004e78000804e800888f550020
:10af0c00f9ff3e003e640200000000000004eb006c
:10af1c00f0ce800060407c000080fb00de6402000c
:10af2c00000000003e65020000000000e14f5000f0
:10af3c00e9ff32000804e800888f5500f4ff3e005a
:10af4c000e06e9000e00e0008e0032000004eb005b
:10af5c009d0544006065020000000000804d7800f3
:10af6c008c0f5400040031000040eb00c064020060
:10af7c00000000000300370010c0b300c0640200e2
:10af8c00000000000804e800880f5700f0ff3e00a6
:10af9c00226402000000000010c0b300da59020065
:10afac00000000000004eb00f0ce800060407c004c
:10afbc00da590200000000000804e800880f57006e
:10afcc00f9ff3e0067ff370010c0b300da590200ea
:10afdc00000000002202ab00feff320031118000a5
:10afec0001407800814c7800e2cf5000160032000e
:10affc0005003e000104e0000b003200e1cf5000e0
:10b00c0024003a000c003700f0cf5000150032003d
:10b01c0001c2b300814f500017003200e34f5000c3
:10b02c001c003a000c0037004251020000000000e6
:10b03c00100020001800370026510200000000000c
:10b04c0010002000140037000e5102000000000018
:10b05c0010002000100037005e51020000000000bc
:10b06c000d003700c0cfb300829c21001249600054
:10b07c001000200008003700819c2100114078004e
:10b08c000000a0000014a1008048780010002000ef
:10b09c000100370010002000da5902000000000007
:10b0ac0030ff37000040eb000afe070010c0b30071
:10b0bc00da590200000000002aff37000040eb00c4
:10b0cc00da5902000000000026ff37006f406000d4
:10b0dc00804ce80010c0b300da59020000000000f8
:10b0ec00f0a121000048eb001904e0001dff320024
:10b0fc0000047800c8590200000000000080fb002a
:10b10c00de640200000000003e650200000000004a
:10b11c00da590200000000001840e800004c7800ea
:10b12c00994f1000f3ff3e000eff3700e340600024
:10b13c00814c780020c0b300626302000000000064
:10b14c0010c0b300da5902000000000005ff370000
:10b15c00de7102000000000010c0b300da590200da
:10b16c0000000000fffe37000040eb00da5902003f
:10b17c0000000000fbfe37003e64020000000000ef
:10b18c006fff3700226402000000000010c0b30003
:10b19c00da59020000000000f2fe37004f07780079
:10b1ac004f06be004f05be004f04be000000060057
:10b1bc00220320001241780032e0b7001180ba005f
:10b1cc009100ba00024278002303200084497800e1
:10b1dc004800dd000080700000000600009e210089
:10b1ec0010407800e94f5000050032000080fb0051
:10b1fc000000400081af2800e10078004111880078
:10b20c002022ef002062a8002222ef0021e2a800f9
:10b21c002342a8008560a9000000060010118000e0
:10b22c004800de0061406000000006001011800044
:10b23c0061406000000006000000eb00c0d08800f8
:10b24c0010002000b0d08800a09e21001090a1001a
:10b25c00000006002322ab000e003a00c0d0800094
:10b26c000000e80001002100810f500001003a00ad
:10b27c000000eb00b1d08000810f500005003200bf
:10b28c00c0d08800f1ce8000614078000080fb00c7
:10b29c002011880000000600889fbe00b5d08000f9
:10b2ac00f8ce8000c7d08000040021008001eb00a4
:10b2bc00062020000701e80003007800840f5100ed
:10b2cc000100320002007800850f500008003200a7
:10b2dc001911800089006300f7ff3a00e8407800fc
:10b2ec008180fb002111880080037800f1ff37007a
:10b2fc00c7d088004f04be0000000600b1d080000b
:10b30c00c2d08000828f500004003a00c222a900f3
:10b31c00a09e21001090a00009003700f2ce800002
:10b32c0000f178008100e800b1d088000000210015
:10b33c00808f500002003a000000eb00b0d0880073
:10b34c0000000600889fbe000004780000c3b30014
:10b35c00eaff070080c7b300e8ff07004440de00a7
:10b36c006f006000c9b0280069407800e3ff070057
:10b37c006f04640069407c00e0ff07004f04be00ce
:10b38c00000006002202ab00feff320030118000ec
:10b39c0000000600011020001211800002806000e5
:10b3ac00fdff32000000060001102000a29e2100cb
:10b3bc009280600006003a000220200013118000e9
:10b3cc0083006100fdff3a000000fb0020118800a3
:10b3dc0000000600889fbe00004478008884fb00b3
:10b3ec0042062000110009008284d80080447800b5
:10b3fc000904e0001500320001c3b30001c0440091
:10b40c00e9ff07004006200000c8b90000445400c2
:10b41c008884fb00a2002000110009008284d8005f
:10b42c008044780001c3b30001c04400deff070074
:10b43c006a48b9000044540001c3b3000140440001
:10b44c00d9ff07004f04be00000006008884fb00f3
:10b45c00a2002000110009008284d80080447800ea
:10b46c000904e000efff3a00f3ff3700881f780073
:10b47c007d02b900d3022000110009000382d8001c
:10b48c0042062000110009000280d8000104780057
:10b49c00d0ff0700e0c2b300c3ff0700e94f540020
:10b4ac0002003e0000c3b300bfff07000840780055
:10b4bc00c8ff07004f04780000000600889fbe00fc
:10b4cc008a9fbe008c9fbe000005780048c0b30068
:10b4dc000041eb00097122001dc0b300ac0020003c
:10b4ec00110009000985d800800578000204e000ed
:10b4fc0002003a000b00e0000600320001c3b3006a
:10b50c0001c04500a8ff070009d8b9000005550087
:10b51c000d4178000844e9000400320011000900d4
:10b52c008c84d80080047800edff370001c3b30091
:10b53c00014045009cff07004f06be004f05be00b2
:10b54c004f04be0000000600e4874700889fbe0041
:10b55c008a9fbe008c9fbe008e1f78000005be0027
:10b56c008ec0b3000040eb0080f79f0008102e0047
:10b57c00595f20000801be000a00be0086060200ca
:10b58c00000000000006be008ff097000104e000f0
:10b59c0003003a00e00f5600e08f5e000c00320012
:10b5ac0001c3b300014046007fff070008e8b90063
:10b5bc000cc9b900000041000866b8008d064000b7
:10b5cc000c0555008d855d0010c0b30080f79f0001
:10b5dc000e47e90007003200a20020000300200003
:10b5ec000800be0086060200000000000004be0039
:10b5fc00e0ff370001c3b300014045006aff0700bc
:10b60c004f0778004f06be004f05be004f04be002a
:10b61c004f00b10000000600881f7800000478007d
:10b62c00184078000004e000050032000804e8002f
:10b63c005dff0700384078000004e000fcff3a0092
:10b64c00d0c0b30058ff0700a0c0b30056ff0700de
:10b65c004f04780000000600881f78000004780072
:10b66c00184078000004e000050032000804e800ef
:10b67c004dff0700384078000004e000fcff3a0062
:10b68c004f04780000000600889fbe008a9fbe0011
:10b69c008c1f78000005be00f0232400f100200070
:10b6ac00800f5500818f5d001700360002242400a6
:10b6bc00f30020000a00be00860602000000000015
:10b6cc007eff0700c0c2b30037ff0700022424002e
:10b6dc00f30020000a00be00a606020000000000d5
:10b6ec000005be001c002000703e2000800f55009d
:10b6fc00e08f5d000a003e00c0ae2800d6ff0700b8
:10b70c00100020002b0037000000eb00713e2000e1
:10b71c00810f5500e08f5d00260036000006eb001f
:10b72c00823e2000030020000a00be0086060200b4
:10b73c00000000000004be0030062000800f540002
:10b74c00e08f5c0003003600080078005bff070008
:10b75c000f0037000c00e0000b003200e90f540022
:10b76c00e08f5c000300360000c3b3000eff07003f
:10b77c000200370010af2800b7ff07000800780060
:10b78c004eff070002003700080078004bff07004f
:10b79c00c0c2b30004ff0700823e2000030020005b
:10b7ac000a00be00a6060200000000000005be0054
:10b7bc001000200031062000810f5500e08f5d0045
:10b7cc00030036000a0078003cff07000f0037002a
:10b7dc000000e0000b003200e90f5500e08f5d0027
:10b7ec000300360000c3b300effe07000200370071
:10b7fc0010af280098ff07000a0078002fff070001
:10b80c00020037000a0078002cff07004f06780072
:10b81c004f05be004f04be0000000600889fbe000e
:10b82c008a9fbe008c1f78000045780040af28002e
:10b83c0089ff070088c0b30009c8b3000bc3b3006d
:10b84c001cc3b3000ac06400030032000c40780033
:10b85c00d5fe0700020037000b407800d2fe07002f
:10b86c000844e900030032008984fb008904d100fc
:10b87c00f4ff37004f0678004f05be004f04be00a2
:10b88c0000000600889fbe008a1f78000105780022
:10b89c000a00e00007003200800478000004eb008e
:10b8ac0039407800c0fe07000804e800880f5500f6
:10b8bc00fbff3e004f0578004f04be000000060061
:10b8cc00889fbe000004780021002000a0b0280052
:10b8dc00ecff07004c40de00c9b02800694078003e
:10b8ec00b1fe07004840de006f0060006940780040
:10b8fc00adfe07004440de006f0060006940780038
:10b90c00a9fe07006f04640069407c00a6fe0700d6
:10b91c004f04be0000000600889fbe0000047800a3
:10b92c0021002000a0b02800d6ff07004440de0014
:10b93c006f006000c9b02800694078009afe0700cb
:10b94c006f04640069407c0097fe07004f04be0042
:10b95c00000006000000e0000300320010c3b3003a
:10b96c0091fe07000200370000c3b3008efe0700f3
:10b97c00000006000080fb0040118800000006005b
:10b98c002202d50061406000000006002222a900be
:10b99c00000006009580ab000e003a00a2cf80009c
:10b9ac00b0cf8000820f50000a003200012020002e
:10b9bc001311800003806000fdff3a008580a90010
:10b9cc009580a80090cf8000604079000080fb003b
:10b9dc002011880000000600809fbe00821f7800a6
:10b9ec003211800080cf800061cf8000827078009f
:10b9fc0080cf80000000e80080cf880071cf8000ed
:10ba0c00810f500001003a009560a9008560a900e3
:10ba1c004f0178004f00be0000400600809fbe0022
:10ba2c00a0cf80000000e800a0cf8800b1cf80003c
:10ba3c00810f500002003a009580a90004003700e5
:10ba4c0091cf8000614078000080fb0020118800bd
:10ba5c008580a9004f00be0000400600a0b9280058
:10ba6c00325b02000000000000000600c859020012
:10ba7c000000000000000600881f780000447800d9
:10ba8c000880fb00c400de00e1806000ca08dd0015
:10ba9c00f2bf2f0043168000030161000281700089
:10baac0042168800c600dd000120b200f2df2f0034
:10babc004316800003016100028170004216880069
:10bacc00c600dd000110b200f2ef2f00431680001b
:10badc00030161000281700042168800c600dd007f
:10baec000108b200f2f72f00431680000301610039
:10bafc000281700042168800610060004600dd0083
:10bb0c00f1fb2f00421680008280600081007000e3
:10bb1c004116880050002000106c0200000000004c
:10bb2c0000ceb30000406400cb42ab0001003200f9
:10bb3c000044a000cb22ab00010032000034a00076
:10bb4c00cb02ab00010032000024a000cae2ab0023
:10bb5c00010032000014a000cac2ab000100320088
:10bb6c000004a0004f04780000000600881f780035
:10bb7c00004478000880fb000068a300030032003a
:10bb8c00c002a900c202a80002003700c002a9002e
:10bb9c00c202a9000058a30003003200c962a80029
:10bbac00cb62a90002003700cb62a900c962a900d0
:10bbbc00c400de00e1806000ca08dd00f2bf2f0087
:10bbcc005316800003016100028170005216880038
:10bbdc00c600dd000120b200f2df2f0053168000fa
:10bbec00030161000281700052168800c600dd005e
:10bbfc000110b200f2ef2f00531680000301610018
:10bc0c000281700052168800c600dd000108b200e7
:10bc1c00f2f72f00531680000301610002817000bf
:10bc2c0052168800610060004600dd00f1fb2f0019
:10bc3c0052168000828060008100700051168800ce
:10bc4c0050002000106c02000000000000ceb30079
:10bc5c0000406400cb42ab00010032000044a00065
:10bc6c00cb22ab00010032000034a000cb02ab00b1
:10bc7c00010032000024a000cae2ab000100320037
:10bc8c000014a000cac2ab00010032000004a000e6
:10bc9c004f0478000000060000c0eb0076ff0700a0
:10bcac000040eb00b1ff070000000600889fbe00bb
:10bcbc008a1f7800804078000040eb00a6660200e6
:10bccc0000000000004478000804e000010032008d
:10bcdc00c222a80008407800da59020000000000d7
:10bcec008084eb00daff2f001c59020000000000da
:10bcfc000004e0000e003200c859020000000000f1
:10bd0c00e14f40000400320008404000da590200c4
:10bd1c00000000000600370010c0b300da59020022
:10bd2c00000000004f0578004f04be000000060024
:10bd3c000804e000ecff3a00d0d080000000e000e6
:10bd4c0009003a00d9d08800c202d5000080ea0070
:10bd5c006100600000004000121680008200650047
:10bd6c008100700011168800d0d080000000e9001e
:10bd7c00d0d08800dcff3700889fbe008a9fbe00b1
:10bd8c00c222a800c4ff070034ff0700caa121008b
:10bd9c000bfe2f0035ff0700004d78000004e0007b
:10bdac00c100350002003a002cff0700f9ff3700f4
:10bdbc00e14f500006003a00b7ff070010380200b0
:10bdcc0000000000b4ff070024ff0700f1ff37005c
:10bddc00e24f500006003a00afff07008c560200fd
:10bdec0000000000acff07001cff0700e9ff370054
:10bdfc00e34f500006003a00a7ff07001441020071
:10be0c0000000000a4ff070014ff0700e1ff37004b
:10be1c00e44f500004003a009fff07009eff07000c
:10be2c000eff0700dbff3700e54f500006003a001d
:10be3c0099ff0700524502000000000096ff070022
:10be4c0006ff0700d3ff3700e64f500006003a000c
:10be5c0091ff07005e690200000000008eff0700e2
:10be6c00fefe0700cbff3700e74f500004003a00fe
:10be7c0089ff070088ff0700f8fe0700c5ff3700a1
:10be8c00ef4f500008003a0010c0b300da5902001e
:10be9c0000000000c222a900d059020000000000de
:10beac000000fe00bbff3700f04f500003003a00cb
:10bebc000040eb007dff0700b6ff3700f14f50004c
:10becc0003003a0010c0b30078ff0700b1ff370041
:10bedc00f24f500023003a001021ef001e21ef001a
:10beec009c21ef0051368000018065006001b30099
:10befc0050368800ddfe07000080fb000018a30010
:10bf0c000100320010a1a8000008a30001003200bb
:10bf1c001081a800d5fe07004804dd00d3fe070001
:10bf2c000080fb0008047000d80c8800c80c880046
:10bf3c0060002000e00c8800ccfe07004804dd0007
:10bf4c00cafe07000080fb00080070006008880033
:10bf5c0011e1a80010c0b300da5902000000000083
:10bf6c008cff3700f34f500008003a001021ef000f
:10bf7c009c21ef00a26c20001289650010c0b30058
:10bf8c00da5902000000000082ff3700f44f500025
:10bf9c000d003a0021e3a800c0002000026b020053
:10bfac00000000000004780021e3a9004840de00f6
:10bfbc00da5902000000000008407800da5902004b
:10bfcc000000000073ff3700f54f500016003a00d8
:10bfdc0021e3a800c900200009007800026b0200d0
:10bfec000000000000047800d0590200000000009e
:10bffc004840de00da5902000000000008407800da
:10c00c00da590200000000001c5902000000000078
:10c01c00e14f5000f0ff3a00c85902000000000048
:10c02c0021e3a9005bff3700f64f500014003a00e3
:10c03c00d84c0200000000000004be004808de00de
:10c04c00da590200000000004048de000100200028
:10c05c00da590200000000004849dd004840de00cb
:10c06c0000007100c848de00da5902000000000030
:10c07c0008407800da5902000000000045ff370044
:10c08c000068a300040032007bfe0700da590200ae
:10c09c00000000003fff37000040eb00da590200bf
:10c0ac00000000003bff3700b0fe0700da59020029
:10c0bc000000000037ff3700c8e2a800c902a90041
:10c0cc00c922a900c8c2a900cae2a900cb02a900d2
:10c0dc00cb22a900cac2a90000000600501680009d
:10c0ec004700de00614060000000060051d0800077
:10c0fc00c208de00e1c06000014178000204a20029
:10c10c00610161004911dd00f0df2f004416800051
:10c11c00840160008301710043168800e180600097
:10c12c00c908dd00ca02b6000080700050168800f5
:10c13c0040012000106c020000000000000006000e
:10c14c00cb22a900c922a90040012000106c0200da
:10c15c00000000000000060051d08000c208de0084
:10c16c00e1c06000014178000204a200610161009d
:10c17c004811dd00f0ef2f004416800084016000b0
:10c18c008301710043168800e1806000c808dd005f
:10c19c00ca02b600008070005016880040062000cd
:10c1ac00106c02000000000000000600cb02a90089
:10c1bc00c902a90040062000106c0200000000001b
:10c1cc0000000600889fbe00804478000904e0004f
:10c1dc00060032000044eb00dfff0700f3ff07000e
:10c1ec000844e80088cf5400fbff3e004f04be001b
:10c1fc0000000600881f7800d7ff07005816800043
:10c20c004744de0061446400e8ff07000840780002
:10c21c004f04780000000600881f78000004e0003e
:10c22c0002003a00c6ff070001003700afff07000d
:10c23c00c9ff0700581680004744de0061446400c3
:10c24c00daff0700084078004f0478000000060071
:10c25c00889fbe008a1f7800d4ff0700a0a0210091
:10c26c00104078006840600006003200a8a0210051
:10c27c00180078004400de0061406000e6ff070013
:10c28c001834a1000044eb00884478000ac8b300bd
:10c29c00b1ff07000884fb000804d100cae2ab0020
:10c2ac00010032000a444400c0ff07008944e80042
:10c2bc00e8cf5400f6ff3a00084078004f057800ac
:10c2cc004f04be0000000600889fbe008a9fbe007f
:10c2dc008c1f780080447800b4ff0700a0a02100d8
:10c2ec00104078006840600006003200a8a02100d1
:10c2fc00180078004400de0061406000c6ff0700b3
:10c30c001834a1000045eb000a4478000cc8b300b7
:10c31c00aba021000908a30002003a0088ff070027
:10c32c000100370071ff07008bff07008984fb00b9
:10c33c008904d1000a85fb000a05d100cae2ab00d2
:10c34c00010032000c45450098ff07009b40780027
:10c35c0063c06000e24f50000b003a00e64f5400ff
:10c36c0009003a00a0a021001034a0000908a30085
:10c37c0002003a001044a10006003700a0a02100e2
:10c38c001044a000030037000844e800e84f5400b4
:10c39c00e0ff3a000a4078004f0678004f05be00d7
:10c3ac004f04be000000060051d08000c208de0021
:10c3bc00e1c06000014178000204a200610161004b
:10c3cc004611dd00f0fb2f00441680008401600054
:10c3dc008301710043168800e1806000c608dd000f
:10c3ec00ca02b60000807000501688004001200080
:10c3fc00106c02000000000000000600cac2a90078
:10c40c00c8c2a90040012000106c0200000000000e
:10c41c0000000600e4ff0700a0c0b30069ff07009e
:10c42c00f6ff0700a0a02100c1cfb30010c8600028
:10c43c0000000600e24f500010003200e34f5000a5
:10c44c00040032000004e00017003a00f1ff07007e
:10c45c0015003700d4ff070010c0b30059ff0700c8
:10c46c00e6ff070020c0b30056ff0700a0a0210084
:10c47c009040780063c870000b003700caff0700bb
:10c48c0020c0b3004fff0700dcff070020c0b30043
:10c49c004cff0700a1a02100114078000000a10072
:10c4ac000014a000804878000000060050d08000e6
:10c4bc0063006000e20f50000d003200e30f5000eb
:10c4cc00220032000000e0002b003a00cbff0700f6
:10c4dc0010c0b3003bff0700a1a021001140780061
:10c4ec000000a0000014a100804878002200370052
:10c4fc00a0a02100104078000038a30007003200f3
:10c50c000048a30002003200f8fe070001003700cb
:10c51c000bff0700a0a021001034a100a2ff070010
:10c52c0020c0b30027ff0700b4ff070010c0b30002
:10c53c0024ff0700a1a02100114078000000a000fa
:10c54c000014a100804878000b00370096ff07000c
:10c55c0020c0b3001bff0700a8ff070010c0b300ea
:10c56c0018ff0700a1a02100114078000000a000d6
:10c57c000014a1008048780000000600889fbe00cf
:10c58c008a1f7800ccfe0700a0a021001041780083
:10c59c000224a00071ceb30001486100eaa0210082
:10c5ac00f8a02100c859020000000000004d7800de
:10c5bc00e14f500003003200e24f5000f9ff3a0007
:10c5cc000300370093ff0700b8ff0700f5ff3700a3
:10c5dc0090ff0700c5fe0700b4ff070020c0b300a2
:10c5ec0094ff070000c0eb00f6fe070000c0eb0054
:10c5fc00f4fe0700adff070030c0b3008dff07004d
:10c60c000000eb0060d08800990f20000500370077
:10c61c0060d080000000e80060d08800890f5000d6
:10c62c0003003600f3fe07000004e000f8ff3200c0
:10c63c009eff070077ff07009cff070030c0b30088
:10c64c007cff07002000200061d080000008dd0086
:10c65c00da59020000000000004ceb0060d08000b2
:10c66c000000e00012003200f9fe0700da59020067
:10c67c0000000000f6fe0700da590200000000007e
:10c68c00f3fe0700da59020000000000f0fe07007c
:10c69c00da590200000000001840e800004c780055
:10c6ac000080fb0061d08000810f5000eeff39004c
:10c6bc007eff0700bbff3700829f210000497800f6
:10c6cc00e34f500005003a0000202000d0cf880036
:10c6dc0000082000e0cf8800030037000020200075
:10c6ec00d0cf8800e0cf8800e1cf50000e003200a0
:10c6fc0003003900e2cf50001f003a00140037004d
:10c70c0041c1b300e09f21000148780041c6b3004d
:10c71c000000e8000148780021c3b3000000e800e5
:10c72c00014878001b00370021c0b300e09f2100b6
:10c73c0001487800a1c0b3000000e800014878006f
:10c74c0051c0b3000000e800014878001100370028
:10c75c0011c0b300e09f21000148780051c0b30024
:10c76c000000e8000148780021c0b3000000e80098
:10c77c0001487800070037000040eb00e19f2100e2
:10c78c00804878008100e800804878008100e8004b
:10c79c008048780000000600829c2100124178003d
:10c7ac007041610004003a00cc22b7000080ea001e
:10c7bc00c822b60001003700c822b7000180fb0078
:10c7cc00106c020000000000000006000080ea006f
:10c7dc00cc22b600c822b6000180fb00106c02000f
:10c7ec000000000000000600889fbe008a9fbe006b
:10c7fc00804578000b04e0000c0032008044eb0014
:10c80c00f89f21000a102000984078000a00780058
:10c81c00e1ff0700984078000a007800ebff070062
:10c82c008944e80089cf5500f7ff3e004f05be0054
:10c83c004f04be0000000600881f7800f89f2100fe
:10c84c009840780000302000e0ff07009840780006
:10c85c0000102000d0ff0700984078000020200036
:10c86c00cdff07000000eb004f047800000006002d
:10c87c00889fbe00f09f210090407800003020007f
:10c88c00c5ff070019002000cb02ab0005003200e9
:10c89c000920200050168000808464008904e9007f
:10c8ac00cf4cde00f89f210098407800002020003b
:10c8bc00c6ff07009840780000102000c3ff070057
:10c8cc009840780000202000b3ff07000900780092
:10c8dc004f04be00000006000000e00004003a0017
:10c8ec000180ea00cc22b600c822b6000b0037004b
:10c8fc00809c2100104078007040600005003a00d8
:10c90c0001007800cc22b7000180ea00c822b600f2
:10c91c000200370001007800c822b7000280fb003b
:10c92c00106c020000000000000006000080fb00fc
:10c93c00e19f21001141780001042000e6ff07006f
:10c94c00000006000080fb00e19f210011417800ef
:10c95c0001102000e0ff0700000006000080fb0033
:10c96c00e19f210011417800d1cf8000daff070050
:10c97c0000000600881f78000080fb00e19f21006a
:10c98c0011417800d1cf8000d3ff0700f89f210020
:10c99c0098407800001020007fff07009840780036
:10c9ac000010200089ff07004f04780000000600eb
:10c9bc00889fbe008a9fbe008c9fbe00719b210089
:10c9cc00914078008185fb008b05e9001200200066
:10c9dc008b15dd000104e000140032000004780027
:10c9ec008004eb00ec9f21000c05e8007d9b2100ee
:10c9fc000b0064001c41780001202000b6ff0700ea
:10ca0c009a4078000010200063ff07009a407800dd
:10ca1c00001020006dff0700080444008904e800a2
:10ca2c001d80fb00890f5000f1ff3e004f06be0039
:10ca3c004f05be004f04be0000000600c822b70020
:10ca4c00000000000000000000000000ca02b60058
:10ca5c0000f0a7000000ea000000ea004f00de0032
:10ca6c0000000600e0cf8000f4ff07000000060085
:10ca7c00889fbe00c89f210018007800efff0700b8
:10ca8c00e3044400994078000010200042ff0700a6
:10ca9c0018007800e9ff07000044780099407800fe
:10caac000010200049ff0700084078004f04be002a
:10cabc0000000600889fbe008a9fbe008c1f780075
:10cacc0000202000ddff07000004eb00709b21001c
:10cadc001004e000140032008004eb00fa9f2100e7
:10caec00000678009a407800001020002aff07000a
:10cafc0000202000d1ff0700804578009a40780084
:10cb0c000010200031ff0700080444000b04e00073
:10cb1c00010032000804e8008904e8001c80fb00d6
:10cb2c00890f5000efff3e00080078004f06780098
:10cb3c004f05be004f04be0000000600889fbe00db
:10cb4c008a9fbe008c9fbe008e1f7800719b2100b7
:10cb5c00914078008186fb008d06e90012002000d0
:10cb6c008d16dd000004eb000104e0001b00320018
:10cb7c00800478000005eb00ee9f21008e05e80094
:10cb8c000d8064001e4178000120200052ff070038
:10cb9c009b40780000102000fffe070000082000da
:10cbac00a6ff0700004678009b407800001020008c
:10cbbc0006ff070089844400080444000c04e000cc
:10cbcc00010032000804e8000a05e800719b21000e
:10cbdc001180fb008a0f5000e9ff3e00080078002e
:10cbec004f0778004f06be004f05be004f04be0035
:10cbfc0000000600814f500005003a003100200073
:10cc0c0080bb20000a6e0200000000000600370006
:10cc1c0051002000b0bb20000a6e02000000000092
:10cc2c0080a221001048e80000000600881f780050
:10cc3c000044780041002000b0ba2000ae6d020024
:10cc4c0000000000501680004600dd004f00de00a2
:10cc5c0088407800e7ff070031002000f0ba200080
:10cc6c00ae6d020000000000501680004700dd0091
:10cc7c004f00de0088407800deff070041002000f6
:10cc8c0020bb2000ae6d020000000000501680009a
:10cc9c004800dd004f00de0088407800d5ff07001b
:10ccac002100200060bb2000ae6d020000000000df
:10ccbc00501680004900dd004f00de0088407800ef
:10cccc00ccff07004f04780000000600889fbe00d0
:10ccdc008a1f78000004be000205780080c2b300f1
:10ccec00da5902000000000008007800026b020014
:10ccfc000000000000047800080078003c5a020094
:10cd0c000000000090c2b300da59020000000000dd
:10cd1c000000eb00890f54000400360010002000c6
:10cd2c008a0f5400010039000000eb0011c0b30061
:10cd3c00b0ff07004f0578004f04be00000006004e
:10cd4c00889fbe008a9fbe00804478000144780012
:10cd5c0080a221000048eb000904e00003003a0027
:10cd6c00a09e21001080a0000c0037000804e000f9
:10cd7c000a003200f103200050ae20000a6e0200bf
:10cd8c000000000011012000a01921000a6e020011
:10cd9c0000000000c8590200000000004100200003
:10cdac0040b220000a6e020000000000cb42a80036
:10cdbc00c942a9003100200080b22000ae6d0200f3
:10cdcc0000000000501680004500dd004f00de0022
:10cddc0011c0b30087ff0700cb42a900c942a800cd
:10cdec00c222a800c022a90081002000b0b22000fd
:10cdfc00ae6d020000000000c202d50061006000b0
:10ce0c0011c0b3007bff0700c222a900c962a800b1
:10ce1c00cb62a9008100200030b32000ae6d02006f
:10ce2c0000000000501680004400dd004f00de00c2
:10ce3c0011c0b3006fff0700cb62a900c962a90043
:10ce4c0081002000b0b32000ae6d02000000000095
:10ce5c00501680004400dd004f00de008040eb00e7
:10ce6c0064ff0700c002a900c202a8002000200035
:10ce7c003e6c0200000000004100200030b4200095
:10ce8c00ae6d020000000000101680006100600012
:10ce9c0011c0b30057ff0700e100200070b4200060
:10ceac000a6e02000000000021e3a800210020000f
:10cebc0050b52000ae6d020000000000723520005d
:10cecc00712b20009000200080ff07000804e00078
:10cedc00430032003100200070b52000ae6d02001e
:10ceec000000000072352000712b2000b0002000e3
:10cefc0076ff070041002000a0b52000ae6d0200b7
:10cf0c000000000002252000011b2000a0002000d2
:10cf1c006eff070031002000e0b52000ae6d02006e
:10cf2c000000000002252000011b2000c000200092
:10cf3c0066ff070021e3a9008100200010b6200045
:10cf4c000a6e020000000000fac32f00802c2000a3
:10cf5c0010086500601680000b3c200000807500f6
:10cf6c0060168800400620003e6c020000000000a5
:10cf7c0010c0b3002dff0700a100200090b62000c8
:10cf8c000a6e020000000000c02c20001008650092
:10cf9c00c962a800cb62a900400620003e6c0200ca
:10cfac00000000000040eb0020ff0700a100200063
:10cfbc0030b720000a6e020000000000401680000e
:10cfcc00808575004b168800400620003e6c0200e0
:10cfdc000000000010c0b30014ff0700230037004e
:10cfec0041002000a0b52000ae6d02000000000042
:10cffc0002252000011b2000a000200033ff0700a9
:10d00c0021e3a9008100200010b620000a6e020066
:10d01c0000000000fac32f00802c200010086500cf
:10d02c0060168000003cb3006016880040062000ab
:10d03c003e6c02000000000010c0b300fbfe0700b5
:10d04c00a100200090b620000a6e02000000000033
:10d05c00c02c200010086500400620003e6c020029
:10d06c00000000000040eb00f0fe07000904e000a7
:10d07c00120032000804e00010003200c002a900c7
:10d08c00c202a800c422a80001022000d0b72000d0
:10d09c000a6e020000000000f1002000b018210010
:10d0ac000a6e020000000000c859020000000000d7
:10d0bc00c422a900c002a900c202a900ca6a0200c7
:10d0cc000000000061002000d0b92000ae6d02000d
:10d0dc000000000088a2210018407800f0590200de
:10d0ec00000000008100200030ba20000a6e02000f
:10d0fc0000000000a09e21001080a10018407800c4
:10d10c004f05be004f04be0000000600cac2a900b5
:10d11c00cb22a900cb02a900cb42a900ca02a900cc
:10d12c00e24f500006003a00cac2a800cb02a80089
:10d13c00cb22a800cb42a800ca02a80008003700e6
:10d14c00cac2a900cb02a900cb22a900cb42a900dc
:10d15c00ca02a9000040e900e14f500007003e0060
:10d16c00c8c2a900c922a900c902a900c942a900c4
:10d17c00c802a900c8e2a80006003700c8c2a8006f
:10d18c00c922a800c902a800c942a800c802a80068
:10d19c00c8e2a80000000600e44f50002300320053
:10d1ac0005003e00e14f500008003200e24f5000f5
:10d1bc002a003a000d003700e84f500021003200e1
:10d1cc00f04f500025003a0010003700c022a90093
:10d1dc00e180600081804000d0ff2f00c202b600c9
:10d1ec0000807000101688001c0037000104e0005d
:10d1fc0003003200c002a900c202a80017003700c9
:10d20c00c002a900c202a900140037000104e0000a
:10d21c0003003200c962a800cb62a9000f003700de
:10d22c00cb62a900c962a9000c003700e180600044
:10d23c00e0ff2f00ca02b600008070005016880074
:10d24c0006003700e1806000ca08dd00f0bf2f0047
:10d25c00ca02b6000080700050168800000006005c
:10d26c00c0ba2800325b020000000000000006007b
:10d27c00889fbe008a1f7800010578000a00e00034
:10d28c0008003200800478000004eb00394078007c
:10d29c00da590200000000000804e800880f55006d
:10d2ac00faff3e004f0578004f04be000000060058
:10d2bc00889fbe008a9fbe008c9fbe008e1f780088
:10d2cc00f8ce80001000200050d18800e4ff070049
:10d2dc00adcab3000c002200eb9d21004e83200050
:10d2ec00c859020000000000e34f50001200320049
:10d2fc0004003e00e14f50003100320034003e008b
:10d30c0095003700e64f50000900320003003e0044
:10d31c00e54f500089003a0063003700e74f50009a
:10d32c003e003200e84f500084003a0031003700d4
:10d33c00cbff0700eaff370030c0b300004c780089
:10d34c0080c0b3001044980021e3a800c000200066
:10d35c00026b020000000000c800de0021449800af
:10d36c0030449800b0002000026b02000000000066
:10d37c00c800de004144980050449800a0002000f2
:10d38c00026b020000000000c800de00614498003f
:10d39c007044980090002000026b02000000000016
:10d3ac00c800de00014c9800104c980021e3a90045
:10d3bc00a100200008007800adff0700c8ff37006f
:10d3cc00c85902000000000050ff0700c4ff3700de
:10d3dc00c85902000000000080447800c8590200bf
:10d3ec000000000080407800094078006aff0700c8
:10d3fc00bbff3700c85902000000000080447800d1
:10d40c00c859020000000000c84cdd000080fb0081
:10d41c008904700059d18800b1ff3700c859020047
:10d42c000000000080447800e1cf540004003a0072
:10d43c0030c0b300c05c02000000000003003700e5
:10d44c0020c2b300c05c020000000000c8590200fa
:10d45c000000000000457800c859020000000000e0
:10d46c008d4f550005003a0051c5b300814f500057
:10d47c0002003a008984fb000400370020c2b3008c
:10d48c00c05c0200000000008004eb0070c0b30020
:10d49c00004c780019449800210020000800780006
:10d4ac0073ff07008eff3700c85902000000000010
:10d4bc0000457800c8590200000000008560a900f2
:10d4cc00c854dd008080fb00898470008c8f540070
:10d4dc00010036008c04780051c0b300014c780078
:10d4ec001a4498002044980031002000080078006d
:10d4fc005fff07001b00780060cf8800e7804400c6
:10d50c00c308de008180400071cf88000001eb0071
:10d51c0082cf88008e00400091cf8800a2cf880077
:10d52c00b2cf88009560a80053d180000901780023
:10d53c00ea7002000000000069ff37000040eb00b9
:10d54c00004c78001044980011002000080078006e
:10d55c0047ff070062ff37004f0778004f06be00f9
:10d56c004f05be004f04be0000000600809c210049
:10d57c0010417800f20050008048eb0001ceb3005f
:10d58c000148610000000600c922a800c902a800d9
:10d59c00c8e2a800c8c2a800c942a800c222a900bb
:10d5ac00c022a90000fe2f00ca26b600409e210012
:10d5bc000008eb00edff0700cb62a900c962a900cf
:10d5cc00c002a900c202a9002d83a9002d43a90005
:10d5dc002d23a9002d63a90000198000000eb300b3
:10d5ec00001988003023ef0020f02100201988005a
:10d5fc002223ef0000000600401988002023a80019
:10d60c002003a9002003ab00feff320000188000ad
:10d61c000000060021e3a800c0002000f6ff070070
:10d62c003c5a02000000000021e3a90000000600a3
:10d63c00889fbe008a1f7800e1002000e0352000a2
:10d64c000a6e020000000000f1002000b01821005a
:10d65c000a6e020000000000f1002000c03620001d
:10d66c00ae6d0200000000000000eb003c5a02000e
:10d67c000000000011002000b0372000ae6d020049
:10d68c000000000029b92800ba3720000f0037002d
:10d69c0021e3a800c0002000d7ff07000004780099
:10d6ac0021e3a90009007800325b020000000000b1
:10d6bc00080078003c5a0200000000001100200015
:10d6cc000a007800ae6d0200000000001c59020038
:10d6dc00000000000004e000edff3200c859020019
:10d6ec000000000080b92800125b0200000000005e
:10d6fc004f0578004f04be0000000600881f78001c
:10d70c0000047800709b210010407800ef4f50000f
:10d71c0005003e000080fb006f001000f1ff2700a9
:10d72c000088de000004640010cf8000e10f500080
:10d73c001200320005003900e20f50001b003200cd
:10d74c00e30f500031003a0026003700809c210086
:10d75c0001c2b30010c06000040032000800780061
:10d76c00665c02000000000028003700080078000a
:10d77c00925c02000000000024003700809c210015
:10d78c0001c2b30010c06000040032000800780031
:10d79c00645a0200000000001c00370008407800aa
:10d7ac00f05902000000000018003700809c210096
:10d7bc0001c2b30010c060000600320008407800bf
:10d7cc00145c02000000000000c2b300da59020031
:10d7dc000000000008407800145c0200000000000b
:10d7ec000a003700809c210001c2b30010c0600009
:10d7fc00030032004840de00da590200000000004d
:10d80c0008407800da590200000000004f0478004c
:10d81c00000006000000e000140032008000eb0065
:10d82c0000000000000000000000000000000000ec
:10d83c0000000000000000000000000000000000dc
:10d84c0000000000000000000000000000000000cc
:10d85c0000000000000000000000000000000000bc
:10d86c008100e800810f5000edff3e000000060033
:10d87c00889fbe008a1f7800000578000a00e0002f
:10d88c000d0032000004eb00a90f20000900780005
:10d89c00e0ff070009007800deff070009007800b0
:10d8ac00dcff070009007800daff07000804e80035
:10d8bc00880f5500f5ff3e004f0578004f04be0061
:10d8cc000000060000027800020120001100200078
:10d8dc000000eb0000004000848160000100320079
:10d8ec000000a000818040000201e900f9ff3a002d
:10d8fc0000017800719b210091407800f0cf50001e
:10d90c00030032000180fb00700010000010de00ec
:10d91c0000000600c222a9006820ef006a20ef0078
:10d92c006020ef006220ef001e21ef00f0ff2800c6
:10d93c00ac20b6001c21ef0000642000d008880049
:10d94c000000210080d088000000eb0090d08800ff
:10d95c0000000600a1d080000100e00004003200ad
:10d96c000040eb00e28f500037003e0032003700e1
:10d97c00e24f50001000320005003e000004e000b1
:10d98c000a003200e14f500027003a001000370027
:10d99c00f14f50002b003200f34f500029003200a1
:10d9ac00e44f500020003a0019003700d9ff07005f
:10d9bc0010c0b3002400370041002000a0b628009e
:10d9cc00485c0200000000000040eb001e00370025
:10d9dc00c222a8001e21ef001621ef001421ef0037
:10d9ec001e61a8008660a9009660a90060058000f1
:10d9fc0000c0a00000d0a10000e0a10060058800dc
:10da0c001000200090d088000040eb000e00370082
:10da1c0051012000e0b62800485c02000000000024
:10da2c000040eb000800370010002000a0d0880058
:10da3c000040eb00040037000000eb00a0d0880091
:10da4c00010037000040eb0000000600881f780042
:10da5c0090d08000e10f500023003a008660ab00ac
:10da6c0003003a000040eb006200e2001f003a00a5
:10da7c001fe1a8008780a90088d080000800e00082
:10da8c001c0032000001eb00010021005316800045
:10da9c00c619de00f0ce80000370790033048000dc
:10daac0003806000fdff32008780a9000201e800be
:10dabc00880f5100f5ff39006220ef001e21ef00a6
:10dacc00f0ce80000800400070f89700da59020090
:10dadc00000000000804e900f9ff3a008dff070080
:10daec0010c0b300010037000040eb004f04780079
:10dafc00000006006220ef001e21ef00f7ff370048
:10db0c0041168000007c2000010070004016880047
:10db1c0080ff070020c0b3008eff07001c590200d5
:10db2c00000000000004e00005003200c8590200ab
:10db3c000000000087ff07000004e00003003a002b
:10db4c00c2ff07000004e000f4ff320000000600f2
:10db5c00889fbe008a9fbe00008540008a0f50003f
:10db6c002600310000047800390020008b3b220095
:10db7c00110009000984d800e18f50000c0032001c
:10db8c0003003900e28f500019003a0011003700f1
:10db9c00110009000984d800000040000b0040006f
:10dbac001000ba00da590200000000001000370023
:10dbbc00110009000984d800000040000b0040004f
:10dbcc001000ba004800de00da5902000000000024
:10dbdc0007003700110009000984d800000040003c
:10dbec000b0040001080ba00da590200000000005f
:10dbfc000804e8008a0f5400ddff39004f05be0011
:10dc0c004f04be0000000600d1ff070020bb280017
:10dc1c00125b020000000000000006001102200050
:10dc2c0040272100f8ff0700c104200050292100e3
:10dc3c00f5ff070061022000102e2100f2ff070003
:10dc4c008102200070302100efff070051012000fd
:10dc5c00f0322100ecff0700b1012000403421001c
:10dc6c00e9ff070081022000f0352100e6ff0700e4
:10dc7c00b101200070382100e3ff0700e102200011
:10dc8c00203a2100e0ff070051012000003d210057
:10dc9c00ddff070031022000503e2100daff0700b3
:10dcac00e102200080402100d7ff0700c1012000c5
:10dcbc0060432100d4ff0700110220002045210001
:10dccc00d1ff0700c101200030472100ceff070023
:10dcdc0051022000f0482100cbff07001102200068
:10dcec00404b2100c8ff070091012000504d21003e
:10dcfc00c5ff0700f1012000e04e2100c2ff070024
:10dd0c0091022000d0502100bfff070051022000db
:10dd1c0060532100bcff070061032000b0552100b7
:10dd2c00b9ff0700e103200010592100b6ff0700de
:10dd3c0000000600881f7800e10020007091200090
:10dd4c0083ff0700c859020000000000004478005f
:10dd5c0008407800da5902000000000020bb2800bf
:10dd6c00125b020000000000f80db2009885b200b2
:10dd7c000800e9004f00de004f04780000000600a8
:020000040000fa
:10dd8c00901900002600000000000000161a000088
:10dd9c000400000000000000ec1900000c00000062
:10ddac00000000001a1a000004000000000000002f
:10ddbc00261a000002000000020000000300000010
:10ddcc00d01900000e00000000000000f81900003f
:10dddc000a000000000000000a1a00000600000003
:10ddec0000000000de1900000e0000000200000020
:10ddfc00000800000000000000000000000000000f
:10de0c0000000000b61900001a000000000000001d
:10de1c0000080000001000000000000000180000c6
:10de2c00d000000000000000281a000002000000d2
:10de3c0000000000101a00000600000000000000a6
:10de4c001e1a00000400000000000000221a00004e
:10de5c000400000000000000021a0000080000008e
:10de6c00000000002a1a0000020000000000000060
:10de7c00d0180000c000000002000000ce71ce00df
:10de8c0071ce7100ce71bc0071aa7100ce71ce0042
:10de9c0071ce7100ce71aa0071ce7100987198008c
:10deac00718871006a716a00716a71007e71760006
:10debc00714869005a000000000000000c3e0c0084
:10decc003e203e00203e48003b003b00ce71ce0081
:10dedc0071ce7100ce71aa0071ce710098713200b2
:10deec003e0a4000dc3b9e003d063e00a03e50003a
:10defc003b55410052540000000000002253220008
:10df0c00537a53007a53ba00527a5200ce71ce0033
:10df1c0071ce7100ce71aa0071ce7100987198000b
:10df2c0071925500e2533a00545654006654b800ae
:10df3c0053493200430000000000000064324200ec
:10df4c00328632008632800035923500ce71ce009a
:10df5c0071ce7100ce71aa0071ce710098719800cb
:10df6c007148370018333600356a3500b234a400d6
:10df7c00325350004900000000000000287280005d
:020000040000fa
:10df8c00e1806000c908dd00f5df2f007616800007
:10df9c0086826200858270007516880001fe2f0053
:10dfac0035358000858060007100b3003135880004
:10dfbc00f50f2e004636800086826200015020004c
:10dfcc008580700041368800c01188003022ef0037
:10dfdc003062a800610161004410dd00f1fe2f00e9
:10dfec00851180008580600081007000811188009f
:10dffc00e38161008381410090ff2f003002b60065
:10e00c00008071008011880061026200e0ff2f0027
:10e01c003002b60000007200801188003222ef003e
:10e02c004e11dd00f0ff2b003202b6000000710033
:10e03c00901188000000060031e2a8003342a800cd
:10e04c0087c0a900c922a9000000060031e2a9007e
:10e05c003342a90030358000f001b3003035880020
:10e06c00f00f2e00c826b600cf22a900c922a800a6
:10e07c000000060002202000931180008300610044
:10e08c00fdff3a00a0118800000006003202ab0030
:10e09c00feff3200b01180000000060090118000dd
:10e0ac0061406000000006000400fa00881f780040
:10e0bc00f0ff2f0001002000d0bf9f00e1bf9f00a8
:10e0cc004507a9002ca3ef004227a9005fb89700d1
:10e0dc00efb8970061015000e0815800d2bf9f005b
:10e0ec00e3bf9f00e00f5000e08f5800f7ff3a00ad
:10e0fc0000fe2f0023358000830060005100b30028
:10e10c0021358800c406b6003000b30020368800e4
:10e11c0088c0b300009e2100084878000080e80009
:10e12c000008eb00ca6a020000000000f45802006c
:10e13c000000000068c0a80068e0a8008000eb00a8
:10e14c00f00f2000de5802000000000030cf8800e5
:10e15c0021002000f00f2000de580200000000001b
:10e16c0040cf880051168000a09e2100c208de001e
:10e17c00e380600072ba280062c8780068c0a90009
:10e18c0068e0a9001080a100709b2100084878006d
:10e19c003260ef0060ba2800125b02000000000041
:10e1ac008e100200000000004f0478000080fa007e
:10e1bc0000000600bcff07008a14020000000000eb
:10e1cc000000eb0000000600889fbe008a9fbe0086
:10e1dc008c1f78008002eb000203e90080037800ba
:10e1ec000104780003067800a92c20009a00200076
:10e1fc006b00200070cf8000e48242000028e60013
:10e20c0005007800f019e300feff350037017800b7
:10e21c00b70178000280fd0003026900f40fb20020
:10e22c0004016900848169000280fd00f000200077
:10e23c000030e60006007800800078000c800900b1
:10e24c00000000001980a1000281d3001950ad001c
:10e25c008381d3001958ad000c8009000000000028
:10e26c001980a0001970a3000482d3008100e9007a
:10e27c00f2ff3100ef0010000122de00041c7800d8
:10e28c004300de000000e800f639b4009580ab00d6
:10e29c0006003200a0cf8000f619e3000300320024
:10e2ac00f219b4001000780020118800700353009c
:10e2bc00d0ff31004f0678004f05be004f04be0062
:10e2cc00d05c04000000000081c0b300709b2100f2
:10e2dc0001487800710040001054a10000000600b5
:10e2ec0040bb2800125b020000000000000006008a
:10e2fc0001012000400621000a6e0200000000000f
:10e30c000000060011022000203f20000a6e0200cf
:10e31c000000000011c0b3004088210001487800c3
:10e32c000000060011022000203f20000a6e0200af
:10e33c000000000011c0b3004088210001487800a3
:10e34c000040eb000000060011022000203f2000de
:10e35c000a6e02000000000011c0b30040882100ca
:10e36c00014878000000eb000000060011022000bc
:10e37c00203f20000a6e02000000000011c0b30014
:10e38c0040882100014878000010200000000600a1
:10e39c0011022000203f20000a6e02000000000045
:10e3ac0011c0b3004088210001487800000006002d
:10e3bc000080fb000038a30003003200c002a9005b
:10e3cc00c202a80002003700c002a900c202a900c4
:10e3dc000028a30003003200c962a800cb62a90088
:10e3ec0002003700cb62a900c962a9000018a30083
:10e3fc0003003200c942a900cb42a800020037003a
:10e40c00c942a900cb42a9000008a30009003200b0
:10e41c00809c2100104078007040600002003200a7
:10e42c00c8c2a80006003700ccc2a800c8c2a90008
:10e43c0003003700f0fb2f00cc22b600c822b60038
:04e44c0000000600c6
:020000040000fa
:04e4500000000000c8
:020000040000fa
:020000040001f9
:0457f800dff90000d5
:020000040000fa
:020000040001f9
:0457fc007f3f0000eb
:00000001FF
